:100000000C94850A0C94A60A0C94A60A0C94FD0F75
:100010000C9437100C94A60A0C94A60A0C94A60A09
:100020000C94A60A0C94A60A0C94A60A0C94A60A90
:100030000C94A60A0C94A60A0C94A60A0C945213CB
:100040000C94A60A0C94A60A0C94A60A0C94A60A70
:100050000C94A60A0C946D650C94A60A0C94A60A3E
:100060000C94A60A0C94E8650C94A60A0C94A60AB3
:100070000C94A60A0C94A60A0C94A60A0C94A60A40
:100080000C946E790C94A60A0C94A60A0C94A60AF9
:100090000C9417660C94A60A0C94A60A0C94A60A53
:1000A0000C94A60A0C94A60A0C94A60A0C94A60A10
:1000B0000C94A60A0C94A60A0C94A60A0C94A60A00
:1000C0000C94A60A0C94A60A0C94A60A0C94A60AF0
:1000D0000C94A60A0C94A60A0C94A60A0C94A60AE0
:1000E0000C94A60A0C94A86C0C94B26C0C949E6CA4
:1000F0000C945E6C0C94DE6C0C94D46C0C94C86CF8
:100100000C94BC6C0C94A60A0C94A60A0C94A60A37
:100110000C94A60A0C94A60A0C94A60A0C94A60A9F
:100120000C94A60A0C94A60A0C94A60A0C94A60A8F
:100130000C94A60A9C7FBB7F348026814681668111
:100140006E811B81084AD73B3BCE016E84BCBFFD4C
:10015000C12F3D6C74319ABD56833DDA3D00C77F97
:1001600011BED9E4BB4C3E916BAAAABE0000008030
:100170003F07634236B79BD8A71A39685618AEBAFC
:10018000AB558C1D3CB7CC5763BD6DEDFD753EF690
:10019000177231BF000000803F08000000BE9224AB
:1001A00049123EABAAAA2ABECDCCCC4C3E000000E0
:1001B00080BEABAAAAAA3E00000000BF00000080DB
:1001C0003F0000000000084178D3BB4387D1133DB6
:1001D000190E3CC3BD4282AD2B3E68EC8276BED97F
:1001E0008FE1A93E4C80EFFFBE01C4FF7F3F0000BE
:1001F000000000000C945C5B0C949C7F0C94DE85EA
:100200000C9402110C941E780C9457820C94D066B6
:100210000C94F96C0C9436760C948A680C942178C2
:100220000C9481890C9466810C9460740C94111662
:100230000C9465740C9482370C948B0E0C9434805F
:100240000C946A740C94031D0C9440790C943183C3
:100250000C94710E0C9477740C947F860C946F74CC
:100260000C94454C0C9446810C941E150C944569D5
:100270000C94BB6A0C9423740C94006A0C94497916
:100280000C94BB7F0C9478660C94484D0C94EE82D1
:100290000C9439730C941B6E0C94E56B0C94AE8724
:1002A0000C9426810C94A7820C94FC660C942D73FC
:1002B0000C9493680C946E810C9482820C94C067A9
:1002C0000C941B810C94C7730C94CB670C947474BE
:1002D0000C94EA4C0C9419780C94F0730C94686AA2
:1002E0000C94BD780C94D8786E616E00696E6600CF
:1002F000256300496E76616C6964206932632073FE
:100300007065656420696E20454550524F4D2E2022
:1003100053657474696E67203130206B6269742F85
:10032000730025730A005854414C5F5452494D3DA7
:1003300025640025730A0025730A00546573742030
:10034000362025730A005465737420352025730AFE
:10035000005465737420342025730A005465737447
:1003600020332025730A00546573742032202573CE
:100370000A005465737420312025730A0063686194
:100380006E3D25640A0074787077723D25640A001A
:100390003530306B0A003235306B0A003131356B45
:1003A0000A0035366B0A0033386B0A0025730A00E1
:1003B000765F6C6F773D252D332E32660A002573EC
:1003C0000A0073656E743D252D75206475703D259A
:1003D0002D752069676E6F7265643D252D752074DB
:1003E000746C5F7A65726F3D252D750A0025372E76
:1003F00033662025372E33660025352E32662000E1
:100400004572726F72203020566F6C74004E6F749C
:1004100020737570706F727465640A004572726F34
:1004200072203020566F6C74004572726F722030EB
:1004300020566F6C740062756C6B5F64656C6179DB
:100440003D252D750062756C6B3D252D750056613F
:100450006C7565206E6F7420616C6C6F77656400DD
:1004600062756C6B3A206D61783D257520737461FF
:1004700072743D25752C20656E643D25752C2069B0
:100480006E5F7573653D25750A007062323D257398
:100490000A007062313D25730A00256C7500416CBD
:1004A0006C6F77656420737065656420312F31301F
:1004B0002F3130302F343030206B6269742F73004D
:1004C00025630074746C3D252D64200074746C3DAC
:1004D000252D6420004E65772074746C3D252D64B5
:1004E00020002563004D533536313120503D252DF8
:1004F000372E326620252D372E32666D0A00424D8A
:100500005030383520256C642050612020252D374F
:100510002E32666D00256300545F484541545F49A3
:1005200044583D252D352E32662000545F444557F2
:100530003D252D352E3266200041483D252D352E96
:1005400032662000545F53485432583D252D352ED5
:100550003266200052485F53485432583D252D35AD
:100560002E32662000545F52483D252D342E3166D0
:10057000200052483D252D342E3166200025630091
:100580002563002563002563002563007265706F95
:1005900072745F616C6C3D007265706F72743D00C7
:1005A000256300256300256300256300204F534326
:1005B00043414C3D2564200020467573653A206513
:1005C000653D253032782068663D25303278206CD4
:1005D000663D25303278206C623D25303278004D02
:1005E00043553D2530366C780025630074785F6C88
:1005F000656E3D252D6C752C765F6C6F773D252DD6
:100600006C752C73687432783D252D6C752C627571
:100610006C6B3D252D6C75002563004F4B0A002542
:1006200063002563002563002563002563002563BF
:100630000025630025630064656275675F616C6C0B
:100640003D0064656275673D0064656275673D00E5
:1006500025730A00646565700A006E6F6E650A0096
:10066000707772733D007062323D25730A007062CC
:10067000313D25730A00696E74725F7365635F7044
:10068000313D252D372E33660A00696E74725F7016
:10069000313D252D6C640A00696E74725F73656369
:1006A0005F70303D252D372E33660A00696E7472F7
:1006B0005F70303D252D6C640A00765F6D63753D7B
:1006C000252D352E32660A00745F6D63753D252D2C
:1006D000352E32660A00707077723D25730A006409
:1006E000656275673D0072636D643D25730A002580
:1006F000730A006175746F0A006C6F675F6D6F64D9
:10070000653D007573625F7077723D25730A0072F4
:10071000656C61793D25730A0074746C3D252D6408
:100720000A0052494D455F616464723D252D642E77
:10073000252D640A006E65696768626F725F746177
:10074000626C655F73697A653D25640A00765F6C4B
:100750006F773D252D332E32660A00747870773D11
:1007600025640A006368616E3D25640A0069643D82
:10077000006932635F6275733D006932635F737055
:100780006565643D252D6C750A007478743D25738C
:100790000A0053797374656D2053756D6D617279BC
:1007A0000A002530366C780041744D65676132353A
:1007B00036524652320041744D65676131323852CB
:1007C0004652320041744D656761363452465232AA
:1007D0000041744D65676131323852464131004DF8
:1007E00043553D006D61736B3D002C00696E74656F
:1007F0007276616C3D252D750023252D642C0070CB
:1008000062320070623100745F686561745F6964B0
:100810007800745F64657700616800705F6D7335A0
:100820003631310072685F736874327800745F73B8
:100830006874327800706100700061643400616433
:100840003300616432006164310061330061320061
:10085000613100765F696E007268006572720075C2
:100860007074696D650070315F6C73740070315F16
:10087000740070310070305F6C73740070305F749E
:1008800000703000765F6D637500745F6D63750096
:100890007431007400696400653634007478740043
:1008A0002D002B006175746F006E6F6E65006275B0
:1008B0006C6B00706F7765725F736176655F6C65F6
:1008C0006472790072656C61795F6C65647900634C
:1008D0006F6D7061737300616363656C0070726546
:1008E0007300705F707772006165730070315F6CC8
:1008F0006564790070305F6C656472006576656E62
:1009000074006C6564006F7700706B740074785FBE
:100910006C6564790072785F6C656472006F7065F5
:1009200072006E6F6E65002530327800765F61640C
:10093000343D252D382E3666002000765F61643305
:100940003D252D382E3666002000765F6164323DED
:10095000252D382E3666002000765F6164313D25F6
:100960002D382E3666002000765F6C696768743D0E
:10097000252D382E3666002000765F61323D252D0C
:10098000372E3366002000765F61313D252D372EEE
:100990003366002000765F696E3D252D352E326668
:1009A00000204E657665722D7573656420737461E1
:1009B000636B203E2025642062797465730A00759C
:1009C0007074696D653D252D642D646179732D25E5
:1009D0003032643A253032643A253032642D686F03
:1009E0007572730A0074657374205B6F66667C3180
:1009F0007C327C337C347C355D20202020202020FC
:100A0000202D2074657374206D6F6465730A0D006A
:100A10007478205B706B74207061796C6F61645DB9
:100A20002020202020202020202020202D20736521
:100A30006E6420726164696F20706B74206B6579DD
:100A4000626F6172640A0D00776474205B6F6E7C64
:100A50006F66667C746573745D20202020202020E2
:100A6000202020202D207761746368646F670A0D51
:100A700000765F6C6F77205B765F6C6F775D202010
:100A8000202020202020202020202020202D206C0D
:100A90006F77657374207265706F727420766F6CF7
:100AA000746167650A0D0075706772202020202030
:100AB0002020202020202020202020202020202036
:100AC0002020202D207265626F6F7420766961206E
:100AD000626F6F746C6F616465720A0D007561728C
:100AE00074205B33386B7C35366B7C3131356B7CF5
:100AF0003235306B7C3530306B5D202D2073657462
:100B0000207465726D2F75617274207370656564F1
:100B10000A0D00626F6F74202020202020202020EA
:100B20002020202020202020202020202020202DB8
:100B3000207265626F6F740A0D0070777273205BAC
:100B4000646565707C6E6F6E655D202020202020BE
:100B50002020202020202D206D637520736C65657A
:100B600070206D6F64650A0D007265737420656591
:100B700070726F6D20202020202020202020202037
:100B800020202020202D20726573746F72652065EF
:100B90006570726F6D0A0D0070707772205B6F6EFA
:100BA0007C6F66665D2020202020202020202020D1
:100BB000202020202D2070726F6772616D6D616240
:100BC0006C65207077720A0D0070623220205B6FB6
:100BD0006E7C6F66665D2020202020202020202053
:100BE00020202020202D2070726F6772616D6D6152
:100BF000626C652070696E2062320A0D007062318D
:100C000020205B6F6E7C6F66665D20202020202098
:100C10002020202020202020202D2062756C6B2099
:100C20004750494F2070696E0A0D00747874205B3C
:100C3000737472696E675D202020202020202020A0
:100C4000202020202020202D2053657420726570E4
:100C50006F7274207465787420737472696E670A99
:100C60000D0074787077205B31352D305D202020A9
:100C700020202020202020202020202020202D2067
:100C80005458205077722E20486967686573742025
:100C90003020283364426D290A0D0074746C205B87
:100CA000302D31355D2020202020202020202020C4
:100CB000202020202020202D2074696D652D746F48
:100CC0002D6C69766520666F72207061636B657448
:100CD000730A0D0073732020202020202020202064
:100CE0002020202020202020202020202020202004
:100CF0002D2073797374656D2073756D6D617279D4
:100D00000A0D007273202020202020202020202087
:100D10002020202020202020202020202020202DC6
:100D200020726164696F2073746174730A0D0072BC
:100D300069205B236E5D205B696E745D202020203E
:100D400020202020202020202020202D20726570AF
:100D50006F727420696E74657276616C0A0D007230
:100D6000636D64205B6F6E7C6F66665D2020202063
:100D700020202020202020202020202D20616C6C8D
:100D80006F7720636D642066726F6D206E65746F7F
:100D9000726B0A0D007265205B236E5D205B2B7CFD
:100DA0002D5D205B6D61736B7C6175746F2C6D6163
:100DB000736B5D202D206D6F7465207265706F728E
:100DC00074207365742F6D6F646966790A0D006F06
:100DD00077202020202020202020202020202020BC
:100DE00020202020202020202020202D206F6E6514
:100DF0002D776972652073656E736F72730A0D00CB
:100E00006C6F67205B6175746F7C6F6E7C6F66665C
:100E10005D20202020202020202020202D206D6FEC
:100E20007465732064617461206F6E205553420AAB
:100E30000D006E65205B666C7573685D2020202058
:100E400020202020202020202020202020202D2095
:100E50006E65696768626F72207461626C650A0D05
:100E600000657272202020202020202020202020B9
:100E7000202020202020202020202020202D206520
:100E800072726F722073746174730A0D006D6375F2
:100E90002020202020202020202020202020202052
:100EA0002020202020202020202D206D6375206907
:100EB0006E666F0A0D00693263205B70726F626547
:100EC0007C737065656420236E5D202020202020C7
:100ED00020202D206932632070726F626520627558
:100EE000737C736574206275732073706565640A22
:100EF0000D006964205B72657365745D202020209D
:100F000020202020202020202020202020202D20D4
:100F100069642068616E646C696E670A0D006875AB
:100F20006D20202020202020202020202020202074
:100F3000202020202020202020202D2068756D6971
:100F4000646974792073656E736F720A0D0072653F
:100F50006C6179205B6F6E7C6F66667C7374617404
:100F6000735D20202020202020202D2072656C61C0
:100F700079206E6574776F726B207265706F727412
:100F8000730A0D006465205B6D61736B5D2020202A
:100F90002020202020202020202020202020202051
:100FA0002D2064656275670A0D006368616E205BC1
:100FB00031312D32365D202020202020202020209D
:100FC0002020202020202D206368616E2031312DCB
:100FD00032362028322E3430352D32343830204D00
:100FE000687A290A0D0063616C69205B5B765F6932
:100FF0006E7C61317C61325D20766F6C747C7265D1
:101000007365747C6E6F6E655D202D2063616C6905
:1010100062726174650A0D0062756C6B205B5B73B4
:10102000686F777C666C7573685D205B7365742090
:1010300074687273682064656C61795D5D20202D31
:101040002062756C6B696E67207061636B65747389
:10105000200A0D0061646320202020202020202011
:101060002020202020202020202020202020202080
:101070002D2073686F7720765F696E2C2061312C8C
:1010800020613220766F6C74616765730A0D00759C
:101090002020202020202020202020202020202050
:1010A00020202020202020202020202D207570743A
:1010B000696D650A0D007620202020202020202048
:1010C0002020202020202020202020202020202020
:1010D00020202D2076657273696F6E0A0D006820DE
:1010E0002020202020202020202020202020202000
:1010F000202020202020202020202D2068656C70BA
:101100000A0D00256300756E6B6E6F776E20636D40
:10111000640A00484D433538383300257300257381
:1011200000202573002025362E326620002530321F
:10113000780074656D705F65787465726E3D252DFD
:10114000362E326600202573002025362E3266208A
:101150004F6E2D426F6172640025303278007465E5
:101160006D705F626F6172643D252D362E326600B0
:101170000A0042756C6B2072656D3A20737461725F
:10118000743D25752C20656E643D25752C20696E97
:101190005F7573653D25750A0042756C6B2061644F
:1011A000643A2073746172743D25752C20656E64F9
:1011B0003D25752C20696E5F7573653D25750A00A8
:1011C00042756C6B207468726573683A2074696D3F
:1011D00065723D25750A00503A20256C64205061E7
:1011E0002020252D372E3266206D0A004932433AE1
:1011F00020004A54414720726573657474210A00C7
:101200005761746368646F67207265736574210A3F
:101210000042726F776E6F7574207265736574210A
:101220000A0045787465726E616C2072657365742E
:10123000210A00506F7765722D6F6E20726573659D
:1012400074212E0A004F6E6C696E650A00526F752C
:1012500074696E6720456E61626C65640A00525065
:101260004C20456E61626C65640A0025732025730D
:101270002C206368616E6E656C202575202C2063C0
:101280006865636B207261746520257520487A203B
:10129000747820706F7765722025750A000A2A2AF3
:1012A0002A2A2A2A2A426F6F74696E672025732AB8
:1012B0002A2A2A2A2A2A0A004A5441472072657398
:1012C0006574210A005761746368646F67207265F2
:1012D000736574210A0042726F776E6F75742072A5
:1012E00065736574210A0045787465726E616C20BF
:1012F0007265736574210A00506F7765722D6F6E89
:101300002072657365742E0A00726E6720697373AC
:101310007565732025640A00454550524F4D20697C
:101320007320636F72727570742C207265777269A6
:1013300074696E6720776974682064656661756C8E
:1013400074732E0A006C6F63616C686F7374004174
:10135000544D454741323536726672320002000004
:10136000FFFE000001452025642E256420636C6F7C
:10137000636B20256C752063707520256C75206C5F
:10138000706D20256C752069727120256C75206741
:101390006C656420256C7520796C656420256C75FE
:1013A00020726C656420256C7520747820256C751E
:1013B000206C697374656E20256C752073656E737F
:1013C0006F727320256C752073657269616C2025BE
:1013D0006C750A0000407A10F35A00A0724E18098A
:1013E0000010A5D4E80000E87648170000E40B548C
:1013F000020000CA9A3B000000E1F505000080965B
:101400009800000040420F000000A086010000008C
:10141000102700000000E803000000006400000046
:1014200000000A00000000000100000000002C760F
:10143000D888DC674F0823DFC1DFAE59E1B1B7962A
:10144000E5E3E453C63AE651997696E8E6C2842687
:10145000EB898C9B62ED407C6FFCEFBC9C9F40F263
:10146000BAA56FA5F490055A2AF75C936B6CF967DF
:101470006DC11BFCE0E40D47FEF520E6B500D0EDA4
:10148000902E0300943577050080841E080000200C
:101490004E0A000000C80C333333330F986E1283AA
:1014A0001141EF8D2114893BE65516CFFEE6DB187E
:1014B000D1844B381BF77C1D901DA4BBE424203243
:1014C00084725E228100C9F124ECA1E53D274E41E2
:1014D0004E494E495459494E46CDCCCC3D0AD723AE
:1014E0003C17B7D13877CC2B329595E6241FB14FF6
:1014F0000A000020410000C84200401C4620BCBE3B
:101500004CCA1B0E5AAEC59D740011241FBECFEFEE
:10151000D1E8DEBFCDBF00E00CBF1AE0A0E0B2E032
:10152000E0E6FDE201E00BBF02C007900D92A63499
:10153000B107D9F729E3A6E4BAE001C01D92AD3F97
:10154000B207E1F70E9447640C94AE960C94000039
:101550002F923F924F925F926F927F928F929F92C3
:10156000AF92BF92CF92DF92EF92FF920F931F93B1
:10157000CF93DF93CDB7DEB763970FB6F894DEBF96
:101580000FBECDBF6C014B012A01FC0117821682F0
:10159000838181FF43C3AE014F5F5F4F3A01F60184
:1015A0009381F40193FD859193FF81914F018823ED
:1015B00009F430C3853239F493FD859193FF81910D
:1015C0004F01853239F4B60190E00E947A935201BE
:1015D0002501E5CF10E0F12C20E02032A0F48B3281
:1015E00069F030F4803259F0833269F420612CC004
:1015F0008D3239F0803339F4216026C022602460B6
:1016000023C0286021C027FD27C030ED380F3A30B5
:1016100078F426FF06C0FAE01F9F300D1124132F27
:1016200013C04AE0F49E300D1124F32E20620CC04A
:101630008E3221F426FDEEC2206406C08C3611F4F1
:10164000206802C0883641F4F40193FD859193FF30
:1016500081914F018111C1CF9BEB980F933018F40A
:101660002061805E06C09BE9980F933008F071C13D
:101670002F7E26FF16E02F73322E853619F4206454
:10168000322E08C0863621F4F22FF0683F2E02C0B9
:101690001111115037FE07C01C3350F4EE24E394AF
:1016A000E10E27E00BC0183038F027E017E005C046
:1016B00027E04CE3E42E02C0212FE12C520144E04C
:1016C000A40EB11CF20160817181828193810E2D83
:1016D000A3010E94F1912C01098100FF02C003FFC8
:1016E00007C031FC08C032FE09C030E2232E07C01B
:1016F0002DE2222E04C09BE2292E01C0212C802F36
:101700008C7019F0211068C2A8C237FE0FC0E40C1B
:1017100004FF04C08A81813309F4EA941E1474F52D
:10172000F8E0FE1578F588E0E82E2CC036FC2AC0DB
:10173000812F90E0841595059CF02CEF42162FEF39
:10174000520674F0432D4068342E0AC0E2E0F0E007
:10175000EC0FFD1FE10FF11D8081803319F4115052
:101760001111F4CF37FE0EC0EE24E394E10E812F69
:1017700090E0481659062CF4141904C0EE24E394A2
:1017800001C010E037FE06C01414150434F4C20181
:10179000019605C085E090E002C081E090E0211054
:1017A0000196112331F0212F30E02F5F3F4F820F40
:1017B000931F2F2D30E08217930714F4F81A01C0FD
:1017C000F12C832D897049F4FF2039F0B60180E2B5
:1017D00090E00E947A93FA94F7CF222029F0B60184
:1017E000822D90E00E947A9333FC09C0FF2039F0EB
:1017F000B60180E390E00E947A93FA94F7CF37FE27
:101800005AC0942D852D57FE02C090E080E0292E0D
:10181000382E20E030E0A2014E1951095D874C8737
:10182000A201421953095F874E87612F70E0442758
:101830005527461B570B598B488B5FEF25163506EE
:1018400049F4B6018EE290E02A8B3B8B0E947A939A
:101850003B892A89421453046CF04C855D854215FE
:10186000530544F4EE85FF85E20FF31FE60DF71DE7
:10187000818101C080E351E0251A31082F5F3F4F7D
:1018800048895989241635064CF0B60190E02A8B18
:101890003B8B0E947A932A893B89CFCF241435044D
:1018A00039F49A81963318F4953311F404FF81E3E7
:1018B000B60190E04BC08A81813309F00F7EB601FA
:1018C00090E00E947A93111105C034FC18C085E69F
:1018D00090E017C0B6018EE290E00E947A9382E019
:1018E000EE24E394E80EF301E80FF11D8081B601C8
:1018F00090E00E947A9311508E2D91F7E6CF85E407
:1019000090E0B6010E947A9357FC05C0411451043F
:1019100039F404FF05C05194419451088DE201C08F
:101920008BE2B60190E00E947A9380E39AE0491638
:1019300051042CF08F5F5AE0451A5108F7CFB601D9
:1019400090E00E947A93B601C201C0960E947A93F9
:1019500057C1833631F0833779F0833509F058C0A9
:1019600021C05201E2E0AE0EB11CF20180818983F8
:1019700001E010E0230114C05201F2E0AF0EB11CEF
:10198000F2014080518026FF03C0612F70E002C049
:101990006FEF7FEFC2012A8B0E9426938C012A8968
:1019A0002F7715C05201F2E0AF0EB11CF20140805A
:1019B000518026FF03C0612F70E002C06FEF7FEF00
:1019C000C2012A8B0E94DB928C012A892068322E68
:1019D00023FD1AC08F2D90E008171907A8F4B6014F
:1019E00080E290E00E947A93FA94F4CFF20137FCFF
:1019F000859137FE81912F01B60190E00E947A9384
:101A0000F110FA94015011090115110579F7F8C088
:101A1000843611F0893659F5520127FF09C0F4E0E8
:101A2000AF0EB11CF20160817181828193810AC085
:101A3000F2E0AF0EB11CF20160817181072E000C43
:101A4000880B990B2F76322E97FF09C090958095C1
:101A5000709561957F4F8F4F9F4F2068322E2AE0FF
:101A600030E0A3010E948B94E82EE6183FC0022FBD
:101A7000853721F40F7E2AE030E01DC0097F8F36C4
:101A800091F018F4883559F0C5C0803719F08837BF
:101A900011F0C0C0006104FF09C0046007C024FF4A
:101AA00008C0066006C028E030E005C020E130E054
:101AB00002C020E132E0520107FF09C0F4E0AF0E9E
:101AC000B11CF201608171818281938108C0F2E0D2
:101AD000AF0EB11CF2016081718180E090E0A30142
:101AE0000E948B94E82EE6180F77302E36FE0BC03E
:101AF000332D3E7FE11650F434FE0AC032FC08C09C
:101B0000332D3E7E05C00E2D332D03C00E2D01C09A
:101B1000012F34FF0CC0FE01EE0DF11D80818033DA
:101B200011F4397E08C032FF05C00E5F04C0832F58
:101B3000867809F00F5F33FD13C030FF06C01E2DFD
:101B40000F1518F41F0D101B0F2D0F1568F4B6019B
:101B500080E290E03B8B0E947A930F5F3B89F5CF48
:101B60000F1510F4F01A01C0F12C34FF12C0B601A9
:101B700080E390E03B8B0E947A933B8932FF17C051
:101B800031FD03C088E790E002C088E590E0B6012F
:101B90000CC0832F867859F031FF02C08BE201C060
:101BA00080E237FD8DE2B60190E00E947A93E11663
:101BB00038F4B60180E390E00E947A931150F7CF99
:101BC000EA94F301EE0DF11D8081B60190E00E94D0
:101BD0007A93E110F5CF14C0F4E0FF1558F584E0D6
:101BE000F81A33FE1EC0211026C003FF2AC008EEDB
:101BF00012E0F32DF0713F2EF8018491811124C081
:101C0000FF2009F4E5CCB60180E290E00E947A93CF
:101C1000FA94F6CFF6018681978126C08FEF9FEF69
:101C200023C0B60180E290E00E947A93FA94F1100A
:101C3000F8CFD9CFF12CB601822D90E00E947A9393
:101C4000D4CF0CEE12E0D5CF31108052B60190E027
:101C50000E947A930F5F1F4FCFCF23E02F1510F410
:101C600083E0BECFF12CC1CF63960FB6F894DEBFF0
:101C70000FBECDBFDF91CF911F910F91FF90EF90DD
:101C8000DF90CF90BF90AF909F908F907F906F909C
:101C90005F904F903F902F9008958115910511F01E
:101CA0000197F1F7089580E696E09F938F930E9445
:101CB000C6938091660290916702A0916802B091EC
:101CC00069020F900F9093FF03C08AE596E002C06F
:101CD00084E596E09F938F930E94C6930F900F9098
:101CE0000895E091F81CEF73F0E0E75BF24E80831B
:101CF0008091F81C8F5F8093F81C809199358860E3
:101D0000809399354CE452E061E1CA010E945D7014
:101D100080E090E00895CF93DF93EC0180919F13D2
:101D20009091A013A091A113B091A21386FF1DC0A2
:101D30008E811F928F938D811F928F938C811F9222
:101D40008F938B811F928F938A811F928F9389EE3D
:101D500092E09F938F930E94B2938DB79EB70C969B
:101D60000FB6F8949EBF0FBE8DBFBE0181E99AE009
:101D70000E945671BE0188E092E0DF91CF910C94F1
:101D8000E77152985A981DBAE9E6F0E080818062C6
:101D90008083EA9A53985B98EB9A8081806880836D
:101DA000E8E6F0E08081816080830895EEEAFDE15D
:101DB0001182128210820895CF92DF92EF92FF92E9
:101DC0000F931F93CF93DF93EC019B018091AE1D86
:101DD000843108F0BBC08091B01D64E10E9441884D
:101DE0009093B01DC090CB30D090CC30E090CD30EF
:101DF000F090CE30092F10E08DE8989FD00111248B
:101E0000A255B24E1396CD92DD92ED92FC921697AA
:101E10004115510559F0FA018081FD01EA57FF4F44
:101E20008083FA018181A957BF4F8C932097A9F035
:101E300089819DE8909FF001919FF00D1124E2555A
:101E4000F24EDF01A657BF4F8C93E557FF4F8881B5
:101E50008F70808388818F70808321153105E1F137
:101E6000D90116964C9116975DE8509FC001519F7D
:101E7000900D11248255924EFC01E757FF4F40838D
:101E800015964C9115973197408334961B964D913A
:101E90005D916D917C911E97452F562F672F772767
:101EA000518340837C01BEE8EB0EF11CF9012385D0
:101EB000348545855685A4E6B0E00E94DC88672F0E
:101EC000782F892F992724E630E040E050E00E94E7
:101ED0007588D7016D937C938DE8809FD001819F99
:101EE000B00D1124AB54B24EFE0132968FE7019033
:101EF0000D928A95E1F78091B01D8F5F8093B01DA0
:101F00009091AE1D9F5F9093AE1D40919F13509195
:101F1000A0136091A1137091A21360FF2DC01F92B6
:101F20009F931F928F938091AF1D1F928F9389E98A
:101F300091E19F938F930E94C693EDB7FEB73896B9
:101F40000FB6F894FEBF0FBEEDBF16C08091DB3018
:101F50009091DC30A091DD30B091DE300196A11D72
:101F6000B11D8093DB309093DC30A093DD30B093D3
:101F7000DE3080E090E002C081E090E0DF91CF9120
:101F80001F910F91FF90EF90DF90CF9008952091D7
:101F9000AE1D222361F18091AF1D8F5F21502093F0
:101FA000AE1D64E10E9441889093AF1D40919F1344
:101FB0005091A0136091A1137091A21360FF1AC0F9
:101FC0001F922F938091B01D1F928F931F929F930A
:101FD00082E791E19F938F930E94C6938DB79EB73E
:101FE00008960FB6F8949EBF0FBE8DBF03C080E069
:101FF00090E0089581E090E008951F920F920FB64F
:102000000F9211248F939F93AF93BF938091680099
:1020100080FF24C08091743590917535A0917635FC
:10202000B09177350196A11DB11D809374359093C1
:102030007535A0937635B093773580919F13909145
:10204000A013A091A113B091A21387FF07C07498A9
:1020500082E090E09093920280939102BF91AF91C1
:102060009F918F910F900FBE0F901F9018951F9208
:102070000F920FB60F9211248F939F93AF93BF933C
:102080008091680080FF24C08091783590917935E7
:10209000A0917A35B0917B350196A11DB11D809339
:1020A000783590937935A0937A35B0937B358091CC
:1020B0009F139091A013A091A113B091A21390FF30
:1020C00007C0739882E090E090939202809391020F
:1020D000BF91AF919F918F910F900FBE0F901F9066
:1020E000189580937C0080917B00877F80937B0094
:1020F00080917C00806C80937C0085E080937A00E6
:1021000080917A00806880937A0080917B0087FFBD
:10211000FCCF80917B0085FFFCCF80917A008064AA
:1021200080937A0080917A0086FDFCCF109279002E
:102130001092780084E090E060E070E020917A00F6
:10214000206420937A0020917A0026FDFCCF209114
:10215000780030917900620F731F019779F7109220
:102160007C0080917A008F7780937A0076956795CE
:102170007695679580E090E00E944A8C089580E013
:102180000E9471102091890230918A0240918B0245
:1021900050918C020E94448E21EE3AE744E95EE3BE
:1021A0000E94B58A08950F931F93CF93DF930FE199
:1021B00010E0CBE5DEE00093510182E991E00E945E
:1021C0004D0E8091510185FD0DC00031110521F0AA
:1021D0002CF0CB54D10903C0C4ECD9E0E2970150F4
:1021E0001109E9CFBE0180E090E00E944A8C20E016
:1021F00030E04AE754E40E94988BDF91CF911F9121
:102200000F910895CF93DF93EC0188819981009716
:1022100099F08E3F914121F01982188283E011C01C
:10222000623171F40E94D3106093C7307093C8304C
:102230008093C9309093CA308EEF91E1998388835F
:1022400081E0DF91CF91089580917B008860809339
:102250007B0089EC80937C0085E080937A008091FC
:102260007A00806880937A0080917B0087FFFCCFA2
:1022700080917B0085FFFCCF80917A008064809301
:102280007A0080917A0086FDFCCF80917A0080648C
:1022900080937A0080917A0086FDFCCF609178006F
:1022A0007091790080917A008F7780937A0080E036
:1022B00090E00E944A8C27ED33EA40E95FE30E94F8
:1022C000448E26E636E648E853E40E94B48A089530
:1022D000CF92DF92EF92FF921F93CF93DF93CDB710
:1022E000DEB729970FB6F894DEBF0FBECDBF6C01E5
:1022F000109299138FEF898781E0E82E8DE1F82EF7
:1023000010E089858823E9F11830D9F1BE016F5FAB
:102310007F4FCE0109960E941E5F99859F3F11F065
:102320009E3F19F4909399132CC0CE010196C114CD
:10233000D10481F40E94385F80939635AEE8B5E30E
:10234000FE01319688E08E0F91919D938E13FCCF04
:1023500081E018C00E94385FF7018087FE01319646
:1023600020E030E08191D701A20FB31F8C932F5F43
:102370003F4F28303105B1F71F5FF9E0EF0EF11C38
:10238000C0CF812F29960FB6F894DEBF0FBECDBF08
:10239000DF91CF911F91FF90EF90DF90CF90089544
:1023A00080E791E19F938F930E94C6930F900F90C7
:1023B00008952F923F924F925F926F927F928F92E9
:1023C0009F92AF92BF92CF92DF92EF92FF920F93C4
:1023D0001F93CF93DF93EC015B01009711F427E08B
:1023E00003C0019749F426E04AE250E06BE270E056
:1023F00089E290E00E94F85DCE010E9468119E0182
:1024000026563C4E6901D9018C93CD2B69F0C1E071
:10241000DDE1E12CF12C85E2282E81E1382E91E2DC
:10242000892E91E1992E9EC08EE895E30E94C95FA6
:10243000BC01990F880B990B0E944C8C6B017C019D
:10244000AB2869F020E030E048EC52E40E94988B21
:102450009F938F937F936F938EE591E1A4C0CEE815
:10246000D5E309E511E189911F928F931F930F9393
:102470000E94C6930F900F900F900F90B5E3C6394E
:10248000DB0789F720E030E048EC52E4C701B601F1
:102490000E94988B9F938F937F936F9389E491E130
:1024A0009F938F930E94C6930F900F900F900F9061
:1024B0000F900F9080919635811103C08CE893E0C6
:1024C00002C088E193E09F938F9385E491E19F930D
:1024D0008F930E94C6930F900F900F900F906DC036
:1024E00000E010E0FE01E00FF11F80811F928F934A
:1024F000ADE2B1E1BF93AF930E94C6930F5F1F4F50
:102500000F900F900F900F900830110559F720E0B1
:1025100030E048EC52E4C301B2010E94988B9F93D3
:102520008F937F936F933F922F920E94C6930F9049
:102530000F900F900F900F900F908885811151C0D0
:102540008CE893E09F938F939F928F920E94C69303
:102550000E94D011FFEFEF1AFF0A29960F900F90FB
:102560000F900F90D6018C9190E0E816F906E4F5F3
:10257000CE010E94C95FBC01990F880B990B0E9484
:102580004C8C2B013C01A114B10409F4A9CF20E02B
:1025900030E048EC52E40E94988B9F938F937F9396
:1025A0006F9382E391E19F938F930E94C6930F9064
:1025B0000F900F900F900F900F90DF91CF911F9180
:1025C0000F91FF90EF90DF90CF90BF90AF909F90D2
:1025D0008F907F906F905F904F903F902F900C94D2
:1025E000D01188E193E0AECFDF91CF911F910F9191
:1025F000FF90EF90DF90CF90BF90AF909F908F9023
:102600007F906F905F904F903F902F900895CF9361
:10261000DF931F921F92CDB7DEB7EEE8F5E381811D
:10262000898387818A83CE0101960E948B740F90E3
:102630000F90DF91CF910895CF93DF93EC0120911C
:102640008E3530918F354091903550919135609114
:102650009235709193358091943590919535AFEF87
:102660000E94A88AE1F427E04AE250E06BE270E0C1
:1026700089E290E00E94F85D80E090E00E9468119D
:10268000C656DC4E888349E050E06EE070E08EE88C
:1026900095E30E949196DF91CF910C940713DF91FF
:1026A000CF9108951F920F920FB60F9211240BB67F
:1026B0000F92FF920F931F932F933F934F935F932C
:1026C0006F937F938F939F93AF93BF93CF93DF933A
:1026D000EF93FF9380919935826080939935809133
:1026E000660286FD2B9A8091660287FD2B9A809167
:1026F0009102909192021816190614F4749A739A22
:1027000080919F139091A013A091A113B091A21357
:1027100085FF02C074987398809106029091070219
:1027200001979093070280930602892B09F04CC110
:102730008091540A9091550A01969093550A80937E
:10274000540A8091CB309091CC30A091CD30B09193
:10275000CE300196A11DB11D8093CB309093CC302B
:10276000A093CD30B093CE3080E190E090930702FB
:10277000809306028091660280FD02C01D9B05C009
:1027800010929E1310929D1306C081E090E09093EA
:102790009E1380939D1380919F139091A013A091FD
:1027A000A113B091A21397FF08C080919D1390913F
:1027B0009E13892B49F0749A739808EA1CE1C0EEC5
:1027C000D0E3FF24F39421C0739A7498F6CF8091DC
:1027D000540A9091550A01960E944D88892BE1F088
:1027E000F8016085718561157105A1F5F8016085B5
:1027F00071856115710509F03FC0065F1F4F259671
:10280000F0E3C43FDF0709F44CC0F801608571852F
:102810006115710529F3DBCF4281417020E030E082
:1028200050E060E070E080E090E0A0E00E94A88AC4
:10283000B9F2779880919F139091A013A091A11362
:10284000B091A21392FFCCCF749810929202109282
:102850009102C6CF8091540A9091550A01960E9428
:102860004D88892B19F61C821B82AE0162E184E23D
:1028700092E00E945D70BACF8091540A9091550AFF
:102880000E944D88892B09F0B8CFF8821A830983FA
:102890001C821B82AE0162E182E492E00E945D70C4
:1028A000ACCF60916C0270916D0261157105A1F160
:1028B0008091540A9091550A0E944D88892B61F5A8
:1028C0008091743590917535A0917635B0917735BA
:1028D0004091BD285091BE286091BF287091C028BA
:1028E000841B950BA60BB70B8093D01C9093D11C27
:1028F000A093D21CB093D31C809174359091753500
:10290000A0917635B09177358093BD289093BE28FD
:10291000A093BF28B093C02860916A0270916B02A7
:1029200061157105A1F18091540A9091550A0E9498
:102930004D88892B61F58091783590917935A091FA
:102940007A35B0917B354091C1285091C228609171
:10295000C3287091C428841B950BA60BB70B8093DA
:10296000D41C9093D51CA093D61CB093D71C8091F7
:10297000783590917935A0917A35B0917B358093F7
:10298000C1289093C228A093C328B093C4288091F3
:10299000660286FD2B988091660290916702A09155
:1029A0006802B091690291FF0FC00E9483698A3169
:1029B00019F0C1E0C80F01C0CBE00E94C0678C2FA6
:1029C0000E949B690E948A6840E050E060E085EBCD
:1029D00092E00E945D70FF91EF91DF91CF91BF91E6
:1029E000AF919F918F917F916F915F914F913F91A7
:1029F0002F911F910F91FF900F900BBE0F900FBE64
:102A00000F901F9018958091F81C9091DF30891BD2
:102A100008950E940315882371F0E091DF30EF7371
:102A2000F0E0E75BF24E808190E02091DF302F5F95
:102A30002093DF3008958FEF9FEF0895CF93DF93BA
:102A4000EC011092850A1092840A8881998100977E
:102A5000C1F0863E934021F01982188283E0BDC008
:102A6000613109F0B9C00E94091599279093800A35
:102A700080937F0A8D30910509F444C08F3F910502
:102A800049F40E9403158111EECF86EE93E09983FD
:102A90008883A2C08231910509F45AC08F3791050D
:102AA00009F052C080917D0A90917E0A181619068D
:102AB0000CF56091F7397091F83988E090E00E9448
:102AC0007A936091F7397091F83980E290E00E9432
:102AD0007A936091F7397091F83988E090E00E941C
:102AE0007A9380917D0A90917E0A019790937E0A55
:102AF00080937D0A80917D0A90917E0A8F3791059F
:102B000009F0BFCF1092DF301092F81C80917D0A3F
:102B100090917E0AFC01EC50FF4C10829093850A44
:102B20008093840A10927E0A10927D0A80919735D4
:102B300090919835009709F4A4CF40E050E060915F
:102B400097130E945D709DCF8830910571F5AACFD3
:102B50006091F7397091F8398DE090E00E947A9396
:102B600010927C0A10927B0A20917B0A30917C0A99
:102B700080917D0A90917E0A281739070CF0BACF10
:102B8000F901EC50FF4C80816091F7397091F83970
:102B900090E00E947A9380917B0A90917C0A019642
:102BA00090937C0A80937B0ADFCF6091F739709114
:102BB000F8390E947A9320917D0A30917E0A8091A3
:102BC0007F0AF901EC50FF4C80832F5F3F4F309319
:102BD0007E0A20937D0A8ECF81E0DF91CF91089508
:102BE00080919D1390919E13892BD1F08091660264
:102BF00090916702A0916802B091690293FD10C0A4
:102C00000E94C06783B7817F866083BFF89483B7D3
:102C1000816083BF7894889583B78E7F83BF7894D3
:102C20000895CF93DF93FC01208131812115310577
:102C300051F02133324129F0FC011182108283E0EE
:102C400015C0653891F4EC010E94BE660E94F01533
:102C500040E050E065E88091E1149091E2140E9418
:102C60005D7081E392E19983888381E0DF91CF9168
:102C70000895CF93DF931F921F92CDB7DEB7892BB4
:102C800081F05F934F938EE191E19F938F936983DE
:102C90007A830E94C6930F900F900F900F907A81C5
:102CA00069817F936F938BE191E19F938F930E9452
:102CB000C6930F900F900F900F900F900F90DF9191
:102CC000CF910895EF92FF920F931F93CF93DF93CD
:102CD0000E94BE6680EB0E94536081111CC00E945E
:102CE000B0608091C52C9091C62C81609093C62CC9
:102CF0008093C52C81E293E09F938F938BE191E1C8
:102D00009F938F930E94C6930F900F900F900F90F8
:102D1000C1E0D0E002C0C0E0D0E01EB11470729AF1
:102D20000E94BE668EE40E945360811117C00E940B
:102D3000B0608091C52C9091C62C82609093C62C77
:102D40008093C52C7E018FEFE81AF80A48E259E01B
:102D500069E273E0CE010E943916E701111101C04A
:102D600072980E94BE668EEE0E945360811116C05A
:102D70000E94B0608091C52C9091C62C8460909385
:102D8000C62C8093C52C8E010F5F1F4F48E259E07F
:102D900061E373E0CE010E943916E8010E94BE662D
:102DA00086EA0E945360811116C00E94B060809133
:102DB000C52C9091C62C88609093C62C8093C52C0E
:102DC0008E010F5F1F4F48E259E068E373E0CE01C8
:102DD0000E943916E8010E94BE668CE30E9453608F
:102DE00081111EC00E94B0608091C52C9091C62CAC
:102DF00080619093C62C8093C52C8E010F5F1F4F6E
:102E000048E259E060E473E0CE010E94391683E1A4
:102E100091E19F938F930E94C6930F900F90E801CA
:102E20000E94BE6682ED0E945360811116C00E940E
:102E3000B0608091C52C9091C62C80629093C62C76
:102E40008093C52C8E010F5F1F4F48E259E068E464
:102E500073E0CE010E943916E8010E94BE6680E848
:102E60000E945360811116C00E94B0608091C52CF1
:102E70009091C62C91609093C62C8093C52C8E01A6
:102E80000F5F1F4F48E259E061E573E0CE010E94F9
:102E90003916E8010E94BE6680ED0E9453608111E0
:102EA00016C00E94B0608091C52C9091C62C80689D
:102EB0009093C62C8093C52C8E010F5F1F4F48E264
:102EC00059E067E573E0CE010E943916E8010E94DF
:102ED000BE668CEE0E945360811116C00E94B060E5
:102EE0008091C52C9091C62C92609093C62C8093B3
:102EF000C52C8E010F5F1F4F48E259E06FE573E06C
:102F0000CE010E943916E80107E010E00E94BE667B
:102F10008CE70E945360811113C00E94B0608091C1
:102F2000C52C9091C62C80649093C62C8093C52CA0
:102F300048E259E066E673E0CE010E94391603C00C
:102F40000150110919F70E94B060DF91CF911F91D4
:102F50000F91FF90EF900C94D011CF93DF931F92BD
:102F60001F92CDB7DEB74A8369830E94876069816B
:102F7000862F0E94B8604A81842F0E94B8600F900B
:102F80000F90DF91CF910C94B060AF92BF92CF922F
:102F9000DF92EF92FF920F931F93CF93DF9300D0B6
:102FA000CDB7DEB7182F022F4A835B8369830E9457
:102FB00087606981862F0E94B860812F81600E949E
:102FC000AE604A81A42E5B81B52E10E0E12CF12C7D
:102FD000680181E0C81AD108E016F10689F0EC1406
:102FE000FD0419F40E94D36002C00E94C960F5017B
:102FF0008083FFEFEF1AFF0A8FEFA81AB80AECCF11
:103000000F900F900F90DF91CF911F910F91FF9034
:10301000EF90DF90CF90BF90AF900C94B060BF92D4
:10302000CF92DF92EF92FF920F931F93CF93DF9394
:10303000CDB7DEB760970FB6F894DEBF0FBECDBF39
:10304000F82EE42E6623D9F18E010F5F1F4F80E129
:10305000F80111928A95E9F728E0A80168E980EB68
:103060000E94C517FF2041F08FE693E09F938F9356
:103070000E94B2930F900F9026E7C22E23E0D22E2B
:1030800037E0B32EB00EF80181918F011F928F931C
:10309000DF92CF920E94B2930F900F900F900F90FB
:1030A000B012F1CF88851F928F938BEC93E09F93A2
:1030B0008F930E94B2930F900F900F900F90EE207D
:1030C000D9F18E010F5F1F4F80E1F80111928A95AF
:1030D000E9F720E1A80160E880EB0E94C517FF2016
:1030E00041F08BE793E09F938F930E94B2930F90F0
:1030F0000F9086E7E82E83E0F82E9FE0D92ED00EC1
:10310000F80181918F011F928F93FF92EF920E949D
:10311000B2930F900F900F900F90D012F1CF88893B
:103120001F928F938BEC93E09F938F930E94B293A7
:103130000F900F900F900F9060960FB6F894DEBF2F
:103140000FBECDBFDF91CF911F910F91FF90EF90F8
:10315000DF90CF90BF9008950F931F93CF93DF938D
:103160001F921F92CDB7DEB71A82198222E0AE01FC
:103170004F5F5F4F6AEA8EEE0E94C51709E81DE1B6
:10318000898190E0982F88272A81822BF8019183EA
:10319000808322E0AE014F5F5F4F6CEA8EEE0E94AB
:1031A000C517898190E0982F88272A81822BF80102
:1031B0009383828322E0AE014F5F5F4F6EEA8EEE13
:1031C0000E94C517898190E0982F88272A81822B39
:1031D000F8019583848322E0AE014F5F5F4F60EB7F
:1031E0008EEE0E94C517898190E0982F88272A814A
:1031F000822BF801938B828B22E0AE014F5F5F4FF1
:1032000062EB8EEE0E94C517898190E0982F882787
:103210002A81822BF801958B848B22E0AE014F5FCF
:103220005F4F64EB8EEE0E94C517898190E0982F66
:1032300088272A81822BF801978B868B22E0AE01AA
:103240004F5F5F4F66EB8EEE0E94C517898190E05D
:10325000982F88272A81822BF8019783868322E082
:10326000AE014F5F5F4F68EB8EEE0E94C5178981FC
:1032700090E0982F88272A81822BF80191878087F8
:1032800022E0AE014F5F5F4F6AEB8EEE0E94C517E2
:10329000898190E0982F88272A81822BF8019587D1
:1032A000848722E0AE014F5F5F4F6CEB8EEE0E9491
:1032B000C517898190E0982F88272A81822BF801F1
:1032C0009787868722E0AE014F5F5F4F6EEB8EEEF1
:1032D0000E94C517898190E0982F88272A81822B28
:1032E000F801918B808B0F900F90DF91CF911F9100
:1032F0000F9108952F923F924F925F926F927F921B
:103300008F929F92AF92BF92CF92DF92EF92FF92F5
:103310000F931F93CF93DF93CDB7DEB76C970FB6A4
:10332000F894DEBF0FBECDBF182F042F2D8B19824E
:103330001A821B828091AD1D811107C06C8F0E9483
:10334000AC1881E08093AD1D6C8D662309F472C0CA
:103350004EE264EF8EEE0E94AD1762E174E380E00E
:1033600090E00E94306022E0AE014F5F5F4F66EF59
:103370008EEE0E94C5172981822F90E0A0E0B0E078
:103380004427582F692F7A2F8A81482B80919F1DBF
:103390009091A01D9A01AB01281B390B41095109DD
:1033A000A0919D1DB0919E1D0E94DC886B017C0147
:1033B0003FE0F594E794D794C7943A95D1F760919C
:1033C000971D7091981DCB01770FAA0BBB0BBC0109
:1033D000CD014BE0660F771F881F991F4A95D1F7E3
:1033E0002091991D30919A1D4901330FAA08BB08FD
:1033F000A7019601280D391D4A1D5B1D0E94978863
:10340000C20ED31ED092941DC092931D28E0C20E0E
:10341000D11C54E0D594C7945A95E1F70D2C000CBB
:10342000EE08FF08C092A11DD092A21DE092A31D3C
:10343000F092A41D812F8295880F880F807C8C5C70
:103440008887212E312CA3E0B0E0012E02C0AA0F04
:10345000BB1F0A94E2F72AE63AE00E94D5889B0156
:10346000AC012E5F3F4F4F4F5F4F29873A874B8705
:103470005C8780E593ECA0E0B0E09C01AD0104C066
:1034800055954795379527951A95D2F7298B3A8BFD
:103490004B8B5C8B10E0412C512C320188E090E08A
:1034A000AC01421953095B8F4A8F101709F43EC1D2
:1034B000488564EF8EEE0E94AD1769857A858B850D
:1034C0009C850E94306023E0AE014F5F5F4F66EF46
:1034D0008EEE0E94C517E091931DF091941DE05A65
:1034E000FF409F01DF010E94BE886C837D838E8335
:1034F0009F8380918B1D90918C1D9E878D8720913D
:10350000891D30918A1D388B2F8720918D1D309118
:103510008E1D0E94BE886B017C01ADE0F594E7949E
:10352000D794C794AA95D1F7A0918F1DB091901D03
:103530002C813D814E815F818CE055954795379573
:1035400027958A95D1F70E94E788BB2797FDB0950C
:10355000AB2F8C0D9D1DAE1DBF1D0296A11DB11D73
:1035600032E0B595A795979587953A95D1F79C0147
:10357000AD0130584F4F5F4FA0919B1DB0919C1DE6
:103580000E94DC884B015C014FE0B694A7949794AD
:1035900087944A95D1F739818A8190E0A0E0B0E024
:1035A000BA2FA92F982F8827A32B2B81822B9C0120
:1035B000AD010A8C04C055954795379527950A9417
:1035C000D2F72E8B3F8B488F598F4F8558896A01D0
:1035D000550FEE08FF0862E0CC0CDD1CEE1CFF1C52
:1035E0006A95D1F7A091911DB091921D2C813D81DA
:1035F0004E815F810E94E7889B01AC0177E1559580
:103600004795379527957A95D1F72C833D834E833F
:103610005F832D853E85DF010E94BE88DC01CB01E2
:10362000EBE0B595A79597958795EA95D1F72C810D
:103630003D814E815F81820F931FA41FB51FC80E6D
:10364000D91EEA1EFB1E022C04C0CC0CDD1CEE1C95
:10365000FF1C0A94D2F732E0C30ED11CE11CF11C0E
:10366000F2E0F594E794D794C794FA95D1F72E89B0
:103670003F89488D598D2C193D094E095F0969898B
:103680007A898B899C890E94318897FD0BC0660FCF
:10369000771F881F991FA50194010E9475886901F1
:1036A0007A010AC0A50194010E94758869017A0116
:1036B000CC0CDD1CEE1CFF1C9927F7FC9A958F2D76
:1036C0007E2D6D2D9B01AC010E9431889B01AC01C8
:1036D000AEEDBBE00E94DC884C01BB2497FCB094AB
:1036E000AB2CA3E4B3EEA70196010E94EA88BB27A6
:1036F00097FDB095AB2F880E991EAA1EBB1E4FECEE
:10370000840E4EE0941EA11CB11C44E0B594A79415
:10371000979487944A95D1F7C80CD91CEA1CFB1CD6
:103720004C0C5D1C6E1C7F1C1F5FBFCE112381F0F3
:10373000212F30E040E050E0C301B2010E947588C3
:103740002093A51D3093A61D4093A71D5093A81D3F
:103750005D89552389F16091A51D7091A61D809109
:10376000A71D9091A81D611571058105910521F195
:103770000E944C8C20E836EE45EC57E40E94988B72
:1037800021E03EED42E45EE30E94B18E9B01AC017C
:1037900060E070E080E89FE30E94B48A2BE43AE3A3
:1037A0004DEB57E30E94988B6093A91D7093AA1D5F
:1037B0008093AB1D9093AC1D6C960FB6F894DEBF52
:1037C0000FBECDBFDF91CF911F910F91FF90EF9072
:1037D000DF90CF90BF90AF909F908F907F906F9031
:1037E0005F904F903F902F9008950F931F93CF932A
:1037F000DF9300D000D0CDB7DEB78E010F5F1F4F33
:1038000086E0F80111928A95E9F780919F1C811159
:1038100013C040E061E386EA0E94AD174AE06CE223
:1038200086EA0E94AD1781E080939F1C68EF7CE7D9
:1038300080E090E00E94306048E06DE286EA0E94FD
:10384000AD1768EF7CE780E090E00E94306026E0F2
:10385000A80162E386EA0E94C51747E06DE286EAA6
:103860000E94AD178A8190E0982F88272981822BAA
:1038700090939A1C8093991C2C8130E0322F222740
:103880004B81242B30939C1C20939B1C4E8150E039
:10389000542F44276D81462B50939E1C40939D1CB2
:1038A0005F934F933F932F939F938F938FE793E073
:1038B0009F938F930E94B2930FB6F894DEBF0FBE12
:1038C000CDBF26960FB6F894DEBF0FBECDBFDF91F9
:1038D000CF911F910F910895CF92DF92EF92FF92B7
:1038E0000F931F93CF93DF93CDB7DEB72A970FB611
:1038F000F894DEBF0FBECDBF8E010F5F1F4F86E075
:10390000F80111928A95E9F741E062E08CE30E94A8
:10391000AD1748E560E08CE30E94AD1764E278E6FD
:1039200080E090E00E94306026E0A80163E08CE334
:103930000E94C51743E062E08CE30E94AD17098145
:1039400010E0102F00278A81082BE9E7FCE11183A2
:103950000083EB80F12CFE2CEE248C81E82AF3828C
:10396000E282CD80D12CDC2CCC248E81C82AD58259
:10397000C482B801012E000C880B990B0E944C8C5C
:103980009B01AC01B7010F2C000C880B990B2F8306
:10399000388749875A870E944C8C2F813885498502
:1039A0005A850E94348B20EE3EE245E652E40E94A6
:1039B000448E20E030E044E353E40E94B58A9F93B4
:1039C0008F937F936F93DF92CF92FF92EF921F932B
:1039D0000F938DE893E09F938F930E94B2930FB65D
:1039E000F894DEBF0FBECDBF2A960FB6F894DEBFA7
:1039F0000FBECDBFDF91CF911F910F91FF90EF9040
:103A0000DF90CF900895CF93DF93EC018881998167
:103A1000009759F18A31924121F01982188283E08E
:103A200071C082E69AE00E94EB6E892B51F1809181
:103A30009F139091A013A091A113B091A21393FD95
:103A400022C080919F139091A013A091A113B091D7
:103A5000A21394FD49C080919F139091A013A0914F
:103A6000A113B091A21395FD46C040E850E060E07C
:103A700070E082E69AE00E94CD6E8AE192E199833D
:103A8000888381E03FC08091C52C82FFDACF21E09E
:103A900048E061E083E00E947A198091AC1D8F9329
:103AA0008091AB1D8F938091AA1D8F938091A91D4A
:103AB0008F938091A81D8F938091A71D8F938091E4
:103AC000A61D8F938091A51D8F9387ED91E19F9304
:103AD0008F930E94C6938DB79EB70A960FB6F8943F
:103AE0009EBF0FBE8DBFADCF8091C52C83FFB3CFDE
:103AF0000E94F51BB0CF8091C52C84FFB6CF0E94E9
:103B00006C1CB3CFDF91CF910895CF93C82F8CEE6B
:103B10000E94AE608C2F0E94B8606AE67AE080E076
:103B200090E00E9430608DEE0E94AE600E94C960FD
:103B3000C82F0E94D3602C2F30E0322F2227A901FA
:103B4000482BCA01CF9108950F931F93CF93DF9312
:103B5000C82F8CEE0E94AE608C2F0E94B86064E289
:103B600078E680E090E00E9430608CEE0E94AE60CB
:103B700080E00E94B8606AE67AE080E090E00E940F
:103B800030608DEE0E94AE600E94C960C82F0E9416
:103B9000C960D82F0E94D3604D2F50E060E070E0E4
:103BA000762F652F542F44276C2B8A019B01082BFD
:103BB000C901B801DF91CF911F910F9108952F9204
:103BC0003F924F925F926F927F928F929F92AF92AD
:103BD000BF92CF92DF92EF92FF920F931F93CF93FA
:103BE000DF93CDB7DEB7CB54D1090FB6F894DEBF63
:103BF0000FBECDBF8091040290910502892BD1F1B7
:103C000010920502109204028CEE0E94AE608EE1CA
:103C10000E94B86066E37CE980E090E00E9430603A
:103C200082EA0E94851D9093530A8093520A84EA87
:103C30000E94851D9093510A8093500A86EA0E9443
:103C4000851D90934F0A80934E0A88EA0E94851D35
:103C500090934D0A80934C0A8AEA0E94851D9093A6
:103C60004B0A80934A0A8CEA0E94851D9093490A68
:103C70008093480A88E40E94A41D6DAB7EAB8FAB95
:103C800098AF88E50E94A41D4B015C0180914A0A0F
:103C900090914B0A8C0120E030E040E050E0BA0106
:103CA00022968FAF229723961FAF239724962FAF8C
:103CB000249725963FAF259726964FAF26972796B0
:103CC0005FAF279728966FAF289729967FAF2997E0
:103CD0009C0140E050E060E070E080E090E008E0AF
:103CE0000E944A8A0E94038A3901B42FA52FF62F19
:103CF000E72F8C019401A50160E070E080E090E086
:103D00005301CB2EDA2EEF2EFE2E0E94818A2CA399
:103D10003BA34B83252E362E472E582E792E632D0E
:103D2000742D852D972D315041095F4F6F4F7F4F77
:103D30008F4F9F4F88248394912C21153F4F4F4FD5
:103D40005140610571058105910509F010F4812C40
:103D5000912C9A8289820091480A1091490A58014F
:103D6000C12CD12CE12CF12C00E010E02CA13BA1C6
:103D70004B81522D632D742D852D972D0E94EF8838
:103D8000F22E032F142FB52FF62FE72FD82EE92E62
:103D9000A0E00E94A88A84F42150310940485F4F76
:103DA0006F4F7F4F8F4F9F4FF22E032F142FB52F42
:103DB000F62FE72FD82EE92E2F2D302F412F5B2FF6
:103DC0006F2F7E2F8D2D9E2D07E10E94638A2B8FF2
:103DD0003C8F4D8F5E8F6F8F78A389A39AA320535A
:103DE000384F4F4F5F4F6F4F7F4F8F4F9F4F2B8BF2
:103DF0003C8B4D8B5E8B6F8B788F898F9A8F205683
:103E0000304F4F4F5F4F6F4F7F4F8F4F9F4F243D2E
:103E1000304341055105610571058105910529F082
:103E200020F0F4013196FA83E9838090500A909053
:103E3000510A940140E050E060E070E080E090E0E2
:103E400000E10E944A8A2C833D834E835F83662E65
:103E500078874C0140914C0A50914D0AACA0BBA010
:103E6000CB80D22CE32CF42C052D172D9A0140E0A9
:103E700050E060E070E080E090E00E94EF88F22E79
:103E8000032F142FB52FF62FE72FD82EE92EA0E001
:103E90000E94A88A5CF4AFE70E948A8AF22E032F60
:103EA000142FB52FF62FE72FD82EE92E2F2D302FD8
:103EB000412F5B2F6F2F7E2F8D2D9E2D07E00E94AF
:103EC000638A59016A017B018C012C813D814E81FD
:103ED0005F81662D7885C4010E94818A2C833D8391
:103EE0004E835F8368877E878F87988B2E5F3F4FD7
:103EF000434051096E4F7F4F8F4F9F4F2230310506
:103F0000494F5F4F644071058105910539F030F0EC
:103F100009811A810F5F1F4F1A8309836091520A2A
:103F20007091530A80E090E020E030E840E050E0FB
:103F30000E94488929873A874B875C87662E7D8750
:103F40004C0140914E0A50914F0AACA0BBA0CB80CF
:103F5000D22CE32CF42C052D172D9A0140E050E0D3
:103F600060E070E080E090E00E94EF88F22E032F86
:103F7000142FB52FF62FE72FD82EE92EA0E00E94A0
:103F8000A88A84F421503F4F4F4F5F4F6F4F7F4FB0
:103F90008F4F9F4FF22E032F142FB52FF62FE72FA1
:103FA000D82EE92E2F2D302F412F5B2F6F2F7E2FF4
:103FB0008D2D9E2D08E00E94638A59016A017B01C4
:103FC0008C0129853A854B855C85662D7D85C401EC
:103FD0000E94818A29873A874B875C876D87798B16
:103FE0008A8B692E2F5F3F4F41405109610971094A
:103FF00081099109213030484C4F5F47614071057C
:104000008105910539F030F029813A812F5F3F4FCA
:104010003A8329832B893C894D895E896F89788D04
:10402000898D9A8D2F3C37404105510561057105F9
:104030008105910511F00CF0A4C1ACA0BBA0CB8010
:10404000D22CE32CF42C052D172D95014C2D522D3F
:10405000632D742D852D972D0E94EF88A12CB12CF6
:10406000C12CE0E8DE2EE12CF12C00E010E00E94F3
:10407000758929AF3AAF4BAF5CAF6DAF7EAF8FAFF5
:1040800021969FAF2197AB8CBC8CCD8CDE8CEF8CB6
:10409000F8A009A11AA19501A601B701C8010E94C3
:1040A000EF8859016A017B01E82F192F02E00E9475
:1040B0004A8A0E2F0E94818A7901142F552EF62FDD
:1040C000E72F6C01922EAF2CB42E052F462EB72F62
:1040D000782E8D2CA0E00E94A88A5CF4A1E00E94BA
:1040E0008A8A922EA32EB42E052F462EB72F782E15
:1040F000892E292D3A2D4B2D502F642D7B2F872D66
:10410000982D01E00E94638A2AA7732E4A012C96FB
:104110006FAF2C972B967FAF2B978BA79CA72B83EA
:104120003BA34CA39DA26EA37FA388A799A7B52DFF
:104130009701412F552D6F2F7E2FC601A0E00E94C1
:10414000A88A4CF4A3E00E948A8A7901142FB52F23
:10415000F62FE72F6C019701412F5B2F6F2F7E2FDA
:10416000C60102E00E94638A2DA73EA74FA758AB65
:1041700069AB7AAB8BAB9CAB2901B42FA52F2296F0
:104180006FAF2297F72F1C012B893C894D895E89DF
:104190006F89788D898D9A8D24323A4F4F4F5F4FBA
:1041A0006F4F7F4F8F4F9F4F0CF08BC02B8D3C8DEF
:1041B0004D8D5E8D6F8D78A189A19AA12455324FC6
:1041C0004F4F5F4F6F4F7F4F8F4F9F4F59016A0186
:1041D0007B018C010E94EF8819012A01B62FA72FBD
:1041E000FC0103E00E944A8A51016201EB2EFA2E83
:1041F0008F010E94968A59016A017B018C012AA5D0
:10420000372DA4012C966FAD2C972B967FAD2B9755
:104210008BA59CA50E94818A2B833BA34CA35DA305
:104220006EA37FA388A799A79101A2016B2F7A2F74
:10423000CF0102E00E944A8A51016201EB2EFA2E60
:104240008F010E94968A02E00E944A8A0E2F0E94E5
:10425000968A122FD32EE42EB52FF62FE72FF82EA5
:10426000092FA0E00E94A88A5CF4A1E00E948A8A3B
:10427000122FD32EE42EB52FF62FE72FF82E092F6D
:10428000212F3D2D4E2D5B2F6F2F7E2F8F2D902FA9
:1042900001E00E94638A59016A017B018C012DA50E
:1042A0003EA54FA558A969A97AA98BA99CA90E94E6
:1042B000818A2901B42FA52F22966FAF2297F72F5D
:1042C0001C012C813D814E815F8168857E858F85B3
:1042D0009889AB80BBA0CCA0DDA0EEA0FFA008A574
:1042E00019A50E94968A2C833D834E835F8368873D
:1042F0007E878F87988B29853A854B855C856D8570
:1043000079898A89962D5201CB2EDA2E2296EFAC2E
:104310002297FF2E81010E94968A29873A874B8730
:104320005C876D87798B8A8B692E2B893C894D89B7
:104330005E896F89788D898D9A8DA9ACBAACCBAC2A
:10434000DCACEDACFEAC0FAD21961FAD21970E9409
:10435000968A2056304F4F4F5F4F6F4F7F4F8F4F92
:104360009F4F243D3043410551056105710581058D
:10437000910539F030F009811A810F5F1F4F1A83C0
:1043800009834DA95EA96FA978AD9A01AB0160E0E0
:1043900070E0CB0122962FAF229723963FAF239751
:1043A00024964FAF249725965FAF259726966FAF3B
:1043B000269727967FAF279728968FAF289729961D
:1043C0009FAF2997A984BA84CB84DC84ED84F988D3
:1043D0000A89162D60E070E080E090E00E94EF888E
:1043E000122FD32EE42EB52FF62FE72FF82E092FFC
:1043F000A0E00E94A88A84F421503109404E5F4F0A
:104400006F4F7F4F8F4F9F4F122FD32EE42EB52F1C
:10441000F62FE72FF82E092F212F3D2D4E2D5B2F44
:104420006F2F7E2F8F2D902F05E10E94638AAC8025
:10443000BD80CE80DF80E884FE840F8518890E94CD
:10444000968A122FD32EE42EB52FF62FE72FF82EB3
:10445000092FA0E00E94A88A84F4215030484F4FD1
:104460005F4F6F4F7F4F8F4F9F4F122FD32EE42EF2
:10447000B52FF62FE72FF82E092F212F3D2D4E2D8A
:104480005B2F6F2F7E2F8F2D902F0FE00E94638A5E
:1044900039014A015B016C0179018A011B012C0180
:1044A000285E334041095109610971098109910967
:1044B000283D304D4140510561057105810591054B
:1044C00031F028F0E981FA813196FA83E9830E947C
:1044D000B06029813A81232B51F09301A401B501E9
:1044E000C6010E94038A79018A011B012C019701F0
:1044F000A801B101C2010E94448C20E030E048ECE8
:1045000052E40E94988BC55BDF4F0FB6F894DEBF74
:104510000FBECDBFDF91CF911F910F91FF90EF9014
:10452000DF90CF90BF90AF909F908F907F906F90D3
:104530005F904F903F902F9008954F925F926F92AF
:104540007F928F929F92AF92BF92CF92DF92EF9223
:10455000FF922B013C0169017A0123EC35EF4CE815
:1045600051E4C701B6010E94448E4B015C0128EB67
:104570003EE143E753E4C701B6010E94B58A9B01BF
:10458000AC01C501B4010E94988B0E94128C4B01B2
:104590005C0120E030E048EC52E4C301B2010E942B
:1045A000988B21E835E943EC50E40E94448EA50144
:1045B00094010E94448E4B015C0123E333E948E8F7
:1045C00053E4C701B6010E94B58A9B01AC01C50145
:1045D000B4010E94988B23E333EB48E553E40E9437
:1045E000448EFF90EF90DF90CF90BF90AF909F9060
:1045F0008F907F906F905F904F9008954F925F9251
:104600006F927F928F929F92AF92BF92CF92DF92E2
:10461000EF92FF9269017A010E94B88D20E030E0AC
:1046200040E050E40E94B48A22E93CE54EED5EE3AE
:104630000E94988B4B015C0123EC35EF4CE851E470
:10464000C701B6010E94448E2B013C0128EB3EE1DC
:1046500043E753E4C701B6010E94B58A9B01AC0150
:10466000C301B2010E94988B9B01AC01C501B4014A
:104670000E94B58A6B017C0128EB3EE143E753E4DD
:104680000E94448E4B015C01A701960163EC75EF1B
:104690008CE891E40E94B48A9B01AC01C501B4018D
:1046A0000E94988BFF90EF90DF90CF90BF90AF90DB
:1046B0009F908F907F906F905F904F9008954F9252
:1046C0005F926F927F928F929F92AF92BF92CF92A2
:1046D000DF92EF92FF922B013C0169017A0123ECFA
:1046E00035EF4CE851E4C701B6010E94448E4B01FE
:1046F0005C0128EB3EE143E753E4C701B6010E94A9
:10470000B58A9B01AC01C501B4010E94988B0E943F
:10471000128C4B015C0120E030E048EC52E4C30114
:10472000B2010E94988BA50194010E94448E20E062
:1047300030E040E251E40E94B48A24EE38E34EE0D7
:104740005FE30E94448E9B01AC01C701B6010E9449
:10475000B58AFF90EF90DF90CF90BF90AF909F9081
:104760008F907F906F905F904F90089580E80E94A7
:10477000AE6081110DC08EEF0E94B860811108C03B
:1047800066E37CE980E090E00E9430600C94B060C9
:104790000E94B0608091D7309091D830A091D930EC
:1047A000B091DA300196A11DB11D8093D73090935E
:1047B000D830A093D930B093DA300895FC01DC01F1
:1047C000AC014E5F5F4F90E031E38D91982788E018
:1047D000292F220F97FF03C0922F932701C0922FFA
:1047E0008150B1F7A417B50781F721E030E082814D
:1047F000981711F020E030E0C9010895DF92EF92A0
:10480000FF920F931F93CF93DF930E94B62380E80C
:104810000E94AE6081116DC08AEF0E94B860811164
:1048200068C08FE00E94B860811163C06AE67AE0D8
:1048300080E090E00E94306081E80E94AE608111CB
:1048400058C00E94C960D82F0E94C9600E94C960E8
:10485000182F0E94C9600E94C960082F0E94C96079
:104860000E94D360F82E80E80E94AE60811141C0A2
:104870008CEF0E94B86081113CC089EC0E94B86046
:10488000811137C06AE67AE080E090E00E943060F3
:1048900081E80E94AE600E94C960E82E0E94C96053
:1048A000D82E0E94C9600E94C960C82F0E94D360A0
:1048B0001F92DF921F92EF921F92FF921F920F930F
:1048C0001F921F931F92DF931F928F931F92CF937C
:1048D00082EA93E09F938F930E94B2930E94B0600C
:1048E0008DB79EB742960FB6F8949EBF0FBE8DBF90
:1048F00017C00E94B0608091D7309091D830A091BD
:10490000D930B091DA300196A11DB11D8093D73016
:104910009093D830A093D930B093DA300E94B62368
:1049200020E030E040E050E060E070E080E090E0C7
:10493000DF91CF911F910F91FF90EF90DF9008953D
:10494000EF92FF920F931F93CF93DF9300D0CDB7D9
:10495000DEB78C0180E80E94AE60811154C0011561
:10496000110551F085EE0E94B86081114CC062E0E3
:104970007EE281E090E009C083EE0E94B860811180
:1049800042C062E375E783E090E00E94306081E816
:104990000E94AE60811137C00E94C960E82E8983F1
:1049A0000E94C960F82E8A830E94D3608B830E9484
:1049B000B060CE0101960E94DE23892B21F16F2D7C
:1049C00070E07E296C7F80E090E0012B69F00E940E
:1049D0004A8C20E030E04AEF5AE30E94448E20E007
:1049E00030E040EC50E40CC00E944A8C22E538EBE9
:1049F0004FE25BE30E94448E26E636E64BE352E448
:104A00000E94B48A1BC00E94B0608091D730909100
:104A1000D830A091D930B091DA300196A11DB11DE6
:104A20008093D7309093D830A093D930B093DA30B8
:104A30000E94B62360EF7FEF89E794E40F900F9018
:104A40000F90DF91CF911F910F91FF90EF900895FC
:104A50000F931F93CF93DF93729A8091660283FF27
:104A600008C08EE40E945360811165C0C0E5D0E0AB
:104A700009C0C0E5D0E08FED97E00E944D0E219770
:104A8000D1F7EFCF8FED97E00E944D0E2197D1F730
:104A90008FE40E9453600E94C960D82FDF730E9488
:104AA000C960082F0E94C960C82F0E94D360182FC8
:104AB0000E94B0608091660283FF72986D2F70E053
:104AC000762F6627600F711D80E090E00E944A8C6F
:104AD00020E134E048EC5BE30E94448E6093B92807
:104AE0007093BA288093BB289093BC286C2F70E0F9
:104AF000762F6627610F711D769567957695679578
:104B000080E090E00E944A8C24EA3CEF44E25CE3BF
:104B10000E94448E20E030E040E252E40E94B48AD9
:104B200060939A3570939B3580939C3590939D3517
:104B300080E090E002C081E090E0DF91CF911F9192
:104B40000F9108957298729A8EE40E94536080EAE1
:104B50000E94B86080E00E94B86080E00E94B86067
:104B60008FE40E9453600E94C9608EE40E945360EB
:104B700080E80E94B86080E00E94B86080E00E94F7
:104B8000B8600E94B06080E090E0089586E091E116
:104B90009F938F930E94C693809180020F900F90F5
:104BA000882361F01F928F9383E091E19F938F930D
:104BB0000E94C6930F900F900F900F9008958EED66
:104BC00090E19F938F930E94C69386EB90E19F9311
:104BD0008F930E94C6938FE890E19F938F930E94DA
:104BE000C69384E590E19F938F930E94C69388E1DA
:104BF00090E19F938F930E94C69386EE9FE09F93D0
:104C00008F930E94C6938AEA9FE09F938F930E949E
:104C1000C69384E89FE09F938F930E94C6938EE48F
:104C20009FE09F938F930E94C6938091C52C909193
:104C3000C62C827091702DB73EB72E5E3F4F0FB6D7
:104C4000F8943EBF0FBE2DBF892B41F08EE19FE04F
:104C50009F938F930E94C6930F900F9082EF9EE0D8
:104C60009F938F930E94C69386EB9EE09F938F93B2
:104C70000E94C6938DE89EE09F938F930E94C693F7
:104C800081E69EE09F938F930E94C69382E39EE00D
:104C90009F938F930E94C69380E09EE09F938F9393
:104CA0000E94C6938FEC9DE09F938F930E94C693C2
:104CB00085E99DE09F938F930E94C6938FE59DE0C9
:104CC0009F938F930E94C6938FE29DE09F938F9353
:104CD0000E94C69383E09DE09F938F930E94C693AA
:104CE00084ED9CE09F938F930E94C6938BE99CE098
:104CF0009F938F930E94C69382E69CE09F938F932D
:104D00000E94C6938BE29CE09F938F930E94C69370
:104D10008DEF9BE09F938F930E94C6938DB79EB7B4
:104D200080960FB6F8949EBF0FBE8DBF89EC9BE0B6
:104D30009F938F930E94C69388E99BE09F938F93E4
:104D40000E94C69389E69BE09F938F930E94C6932F
:104D50008AE39BE09F938F930E94C69383E19BE03D
:104D60009F938F930E94C6938DED9AE09F938F93AC
:104D70000E94C69387EA9AE09F938F930E94C693FE
:104D800081E79AE09F938F930E94C69388E49AE00C
:104D90009F938F930E94C69380E19AE09F938F9395
:104DA0000E94C69385EE99E09F938F930E94C693CD
:104DB0002DB73EB72A5E3F4F0FB6F8943EBF0FBEE9
:104DC0002DBF089581ED93E00C94EE934F925F9286
:104DD0006F927F928F929F92AF92BF92CF92DF920B
:104DE000EF92FF92CF93DF93CDB7DEB728970FB640
:104DF000F894DEBF0FBECDBF8091CB309091CC3008
:104E0000A091CD30B091CE3089839A83AB83BC839F
:104E10004090CB305090CC306090CD307090CE3000
:104E20008091CB309091CC30A091CD30B091CE30EC
:104E30008D839E83AF83B8876091CB307091CC30E7
:104E40008091CD309091CE302CE3822E912CA12CEC
:104E5000B12CA50194010E9475887F936F9330E176
:104E6000C32E3EE0D32EE12CF12C6D817E818F810B
:104E70009885A70196010E947588A50194010E945A
:104E800075883F932F9340E8842E41E5942EAA2401
:104E9000A394B12CC301B201A50194010E947588AD
:104EA000A70196010E9475883F932F9369817A81AB
:104EB0008B819C81A50194010E9475883F932F935B
:104EC0008FEB99E09F938F930E94C6930FB6F8944F
:104ED000DEBF0FBECDBF28960FB6F894DEBF0FBE63
:104EE000CDBFDF91CF91FF90EF90DF90CF90BF903B
:104EF000AF909F908F907F906F905F904F900895AC
:104F0000EDEFF9E3808191818234924479F0ED5F95
:104F1000F943FF93EF9381EA99E09F938F930E9467
:104F2000C6930F900F900F900F9008953A96E53F1B
:104F300081E8F80738F30895CF93DF93EC018C9A5A
:104F40000E94BF109F938F937F936F9385E999E0A1
:104F50009F938F930E94C6930F900F900F900F9086
:104F60000F900F90209719F00E94D01108C083E98C
:104F700099E09F938F930E94C6930F900F9081E0CA
:104F80000E94711020918502309186024091870223
:104F9000509188020E94448E9F938F937F936F93CA
:104FA00087E899E09F938F930E94C6930F900F908C
:104FB0000F900F900F900F90209719F00E94D01132
:104FC00008C085E899E09F938F930E94C6930F9045
:104FD0000F9082E00E947110209181023091820234
:104FE00040918302509184020E94448E9F938F933C
:104FF0007F936F9389E799E09F938F930E94C69365
:105000000F900F900F900F900F900F90209719F026
:105010000E94D01108C087E799E09F938F930E9468
:10502000C6930F900F9083E00E9471109F938F930F
:105030007F936F9388E699E09F938F930E94C69326
:105040008C980F900F900F900F900F900F902097CB
:1050500019F00E94D01108C086E699E09F938F93C3
:105060000E94C6930F900F908091C52C87FF83C03C
:1050700021E042E161E080ED0E941A629F938F93EC
:105080007F936F9389E599E09F938F930E94C693D6
:105090000F900F900F900F900F900F90209719F096
:1050A0000E94D01108C087E599E09F938F930E94DA
:1050B000C6930F900F9021E042E162E080ED0E94E4
:1050C0001A629F938F937F936F938AE499E09F93E3
:1050D0008F930E94C6930F900F900F900F900F9098
:1050E0000F90209719F00E94D01108C088E499E031
:1050F0009F938F930E94C6930F900F9021E042E1FF
:1051000063E080ED0E941A629F938F937F936F9369
:105110008BE399E09F938F930E94C6930F900F901B
:105120000F900F900F900F90CD2B19F00E94D0117F
:1051300008C089E399E09F938F930E94C6930F90D4
:105140000F9021E042E164E080ED0E941A629F939B
:105150008F937F936F938CE299E09F938F930E943C
:10516000C6930F900F900F900F900F900F90DF91BC
:10517000CF910C94D011CD2BD1F3DF91CF91089525
:105180000F931F93CF93DF93882389F049E050E07A
:105190006FEF70E08EE895E30E94009349E050E0E5
:1051A0006EE070E08EE895E30E94919613C0CEE821
:1051B000D5E307E219E089911F928F931F930F9314
:1051C0000E94C6930F900F900F900F9085E3C63901
:1051D000D80789F7DF91CF911F910F910C94D011CF
:1051E000882311F0299A089529980895882311F0A9
:1051F0002A9A08952A980895CF92DF92EF92FF920B
:10520000CF93DF936B017C0160FF11C08EE094E0CF
:105210009F938F938BE191E19F938F930E94C6930D
:105220000F900F900F900F9081E090E002C080E00F
:1052300090E0C1FE09C0EC01219648E259E063E12B
:1052400074E00E943916CE01C2FE09C0EC0121961D
:1052500048E259E06BE174E00E943916CE01C3FECA
:1052600009C0EC01219648E259E063E274E00E9433
:105270003916CE01C4FE09C0EC01219648E259E07E
:1052800063E975E00E943916CE01C5FE09C0EC0144
:10529000219648E259E067E274E00E943916CE0197
:1052A000C6FE09C0EC01219648E259E06BE274E0C9
:1052B0000E943916CE01C7FE09C0EC01219648E2D2
:1052C00059E061E374E00E943916CE01D0FE09C0B6
:1052D000EC01219648E259E069E374E00E94391636
:1052E000CE01D1FE09C0EC01219648E259E061E40B
:1052F00074E00E943916CE01D2FE09C0EC0121965D
:1053000048E259E065E474E00E943916CE0120912C
:10531000C52C3091C62C24703270232B59F0D3FE4B
:1053200009C0EC01219648E259E06BE474E00E9468
:105330003916CE012091C52C23FF0BC0D4FE09C025
:10534000EC01219648E259E060E574E00E943916CC
:10535000CE012091C52C24FF0BC0D5FE09C0EC0165
:10536000219648E259E066E574E00E943916CE01C4
:10537000D6FE09C0EC01219648E259E06EE574E0E2
:105380000E943916CE01D7FE09C0EC01219648E2F1
:1053900059E069E674E00E943916CE01E0FE0CC0C7
:1053A00048E259E06AE774E0DF91CF91FF90EF9017
:1053B000DF90CF900C943916CD28CE28CF2841F419
:1053C00082E299E09F938F930E94C6930F900F9073
:1053D000DF91CF91FF90EF90DF90CF900895CF9223
:1053E000DF92EF92FF92CF93DF93EC01C12CD12C8F
:1053F0007601209709F4A3C06DE179E0CE010E9407
:10540000D292892B11F46894C0F865E179E0CE015D
:105410000E94D292892B11F46894C1F86DE079E072
:10542000CE010E94D292892B11F46894C2F869E0EF
:1054300079E0CE010E94D292892B11F46894C3F8CE
:1054400066E079E0CE010E94D292892B11F4689433
:10545000C4F862E079E0CE010E94D292892B11F467
:105460006894C5F86CEF78E0CE010E94D292892B47
:1054700011F46894C6F864EF78E0CE010E94D292ED
:10548000892B11F46894C7F86CEE78E0CE010E9485
:10549000D292892B11F46894D0F868EE78E0CE01AE
:1054A0000E94D292892B11F46894D1F862EE78E0D0
:1054B000CE010E94D292892B11F46894D2F86DED3E
:1054C00078E0CE010E94D292892B11F46894D3F82F
:1054D00067ED78E0CE010E94D292892B11F4689496
:1054E000D4F86FEC78E0CE010E94D292892B11F4AF
:1054F0006894D5F864EC78E0CE010E94D292892BB2
:1055000011F46894D6F863EB78E0CE010E94D29251
:10551000892B11F46894D7F86EEA78E0CE010E94E6
:10552000D292892B11F46894E0F860917E02709118
:105530007F0280E090E00E94E692EC015ACFC70122
:10554000B601DF91CF91FF90EF90DF90CF9008955B
:10555000AF92BF92CF92DF92EF92FF920F931F9381
:10556000CF93DF93D22FC32F8A01F62EC72ED82ECA
:10557000E92E217030E040E050E060E070E080E033
:1055800090E0A0E00E94A88A89F08FE794E09F93C2
:105590008F938BE191E19F938F930E94C6930F901D
:1055A0000F900F900F90E1E0F0E002C0E0E0F0E03B
:1055B0008091C52C80FF19C02D2F247030E040E071
:1055C00050E060E070E080E090E0A0E00E94A88AF7
:1055D00061F05F018FEFA81AB80A48E259E063E86A
:1055E00074E0CF010E943916F5012D2F227030E0B2
:1055F00040E050E060E070E080E090E0A0E00E94D9
:10560000A88A61F05F018FEFA81AB80A48E259E052
:1056100067E874E0CF010E943916F5012D2F28703C
:1056200030E040E050E060E070E080E090E0A0E03A
:105630000E94A88A61F05F018FEFA81AB80A48E2B9
:1056400059E06FE974E0CF010E943916F5012D2F62
:10565000207130E040E050E060E070E080E090E0F9
:10566000A0E00E94A88A61F05F018FEFA81AB80A33
:1056700048E259E06AE874E0CF010E943916F5016A
:105680002D2F207230E040E050E060E070E080E0DC
:1056900090E0A0E00E94A88A61F05F018FEFA81A55
:1056A000B80A48E259E06DE874E0CF010E9439166B
:1056B000F5012D2F207430E040E050E060E070E014
:1056C00080E090E0A0E00E94A88A61F05F018FEF87
:1056D000A81AB80A48E259E063E974E0CF010E94D1
:1056E0003916F5012D2F207830E040E050E060E0E1
:1056F00070E080E090E0A0E00E94A88A61F05F0185
:105700008FEFA81AB80A48E259E069E974E0CF01BE
:105710000E943916F50120E03C2F317040E050E046
:1057200060E070E080E090E0A0E00E94A88A61F074
:105730005F018FEFA81AB80A48E259E06CE974E0FB
:10574000CF010E943916F50120E03C2F327040E075
:1057500050E060E070E080E090E0A0E00E94A88A65
:1057600061F05F018FEFA81AB80A48E259E061EAD8
:1057700074E0CF010E943916F50120E03C2F34700F
:1057800040E050E060E070E080E090E0A0E00E9447
:10579000A88A61F05F018FEFA81AB80A48E259E0C1
:1057A00068EA74E0CF010E943916F50120E03C2F31
:1057B000387040E050E060E070E080E090E0A0E011
:1057C0000E94A88A61F05F018FEFA81AB80A48E228
:1057D00059E06BEA74E0CF010E943916F50120E030
:1057E0003C2F307140E050E060E070E080E090E0FD
:1057F000A0E00E94A88A61F05F018FEFA81AB80AA2
:1058000048E259E060EB74E0CF010E943916F501DF
:1058100020E03C2F307240E050E060E070E080E03B
:1058200090E0A0E00E94A88A61F05F018FEFA81AC3
:10583000B80A48E259E067EB74E0CF010E943916DC
:10584000F50120E030E040E050E06F2D647070E042
:1058500080E090E0A0E00E94A88A61F05F018FEFF5
:10586000A81AB80A48E259E06EEB74E0CF010E9432
:105870003916F5018091C52C81FF19C020E03C2F1D
:10588000307440E050E060E070E080E090E0A0E044
:105890000E94A88A61F05F018FEFA81AB80A48E257
:1058A00059E062EC74E0CF010E943916F501809155
:1058B000C52C9091C62C90FF19C020E030E040E04C
:1058C000512F507160E070E080E090E0A0E00E9415
:1058D000A88A61F05F018FEFA81AB80A48E259E080
:1058E00065EC74E0CF010E943916F5018091C52C5A
:1058F0009091C62C90FF19C020E030E040E0512F7D
:10590000507260E070E080E090E0A0E00E94A88A21
:1059100061F05F018FEFA81AB80A48E259E068EC1D
:1059200074E0CF010E943916F5018091C52C909149
:10593000C62C90FF19C020E030E040E0512F507499
:1059400060E070E080E090E0A0E00E94A88A61F052
:105950005F018FEFA81AB80A48E259E06EEC74E0D4
:10596000CF010E943916F50120E03C2F307840E04D
:1059700050E060E070E080E090E0A0E00E94A88A43
:1059800061F05F018FEFA81AB80A48E259E069EDAB
:1059900074E0CF010E943916F50120E030E0402F7D
:1059A000417050E060E070E080E090E0A0E00E9494
:1059B000A88A61F05F018FEFA81AB80A48E259E09F
:1059C0006EED74E0CF010E943916F50120E030E061
:1059D000402F427050E060E070E080E090E0A0E096
:1059E0000E94A88A61F05F018FEFA81AB80A48E206
:1059F00059E061EE74E0CF010E943916F50120E014
:105A000030E040E050E06F2D687070E080E090E0A2
:105A1000A0E00E94A88A61F05F018FEFA81AB80A7F
:105A200048E259E064EE74E0CF010E943916F501B6
:105A300020E030E040E050E06F2D607170E080E0E9
:105A400090E0A0E00E94A88A61F05F018FEFA81AA1
:105A5000B80A48E259E068EE74E0CF010E943916B6
:105A6000F5018091C52C87FF19C020E030E0402F60
:105A7000487050E060E070E080E090E0A0E00E94BC
:105A8000A88A61F05F018FEFA81AB80A48E259E0CE
:105A90006CEE74E0CF010E943916F5018091C52C9F
:105AA00087FF19C020E030E0402F407150E060E0F7
:105AB00070E080E090E0A0E00E94A88A61F05F01C1
:105AC0008FEFA81AB80A48E259E060EF74E0CF01FE
:105AD0000E943916F5018091C52C87FF19C020E07E
:105AE00030E0402F407250E060E070E080E090E0F5
:105AF000A0E00E94A88A61F05F018FEFA81AB80A9F
:105B000048E259E064EF74E0CF010E943916F501D4
:105B10008091C52C87FF19C020E030E0402F4074F1
:105B200050E060E070E080E090E0A0E00E94A88A91
:105B300061F05F018FEFA81AB80A48E259E068EFF8
:105B400074E0CF010E943916F5018091C52C82FFC7
:105B500019C020E030E0402F407850E060E070E075
:105B600080E090E0A0E00E94A88A61F05F018FEFE2
:105B7000A81AB80A48E259E066E276E0CF010E942E
:105B80003916F5018091C52C82FF19C020E030E064
:105B900040E0512F517060E070E080E090E0A0E0C4
:105BA0000E94A88A61F05F018FEFA81AB80A48E244
:105BB00059E06CEF74E0CF010E943916F501809135
:105BC000C52C9091C62C90FF19C020E030E040E039
:105BD000512F527060E070E080E090E0A0E00E9401
:105BE000A88A61F05F018FEFA81AB80A48E259E06D
:105BF0006FEF74E0CF010E943916F5018091C52C3A
:105C00009091C62C90FF19C020E030E040E0512F69
:105C1000547060E070E080E090E0A0E00E94A88A0C
:105C200061F05F018FEFA81AB80A48E259E067E017
:105C300075E0CF010E943916F5018091C52C909135
:105C4000C62C91FF1EC020E030E040E0512F58707C
:105C500060E070E080E090E0A0E00E94A88A89F017
:105C600048E259E060E175E0CF01DF91CF911F91EB
:105C70000F91FF90EF90DF90CF90BF90AF900C947A
:105C800039162D2F3C2FA8016F2D7C2D8D2D9E2D8B
:105C9000A0E00E94A88A41F489EA98E09F938F933C
:105CA0000E94C6930F900F90DF91CF911F910F919B
:105CB000FF90EF90DF90CF90BF90AF900895AF929C
:105CC000BF92DF92EF92FF920F931F93CF93DF93D8
:105CD000EC015B01FB01108264EA78E00E94D29241
:105CE000892B59F58091C52C3DE4F32E00E882FF05
:105CF00003C024E8E22E02C094E0E92E10E0D12C8B
:105D000081FD00EC26E04AE250E06BE270E089E2BF
:105D100090E00E94F85D81E090E00E946811882385
:105D200011F08DE5F82E8091C52C9091C62C90FD38
:105D300016E091FF07C0186005C0F12C00E0E12CCF
:105D400010E0D12C62EA78E0CE010E94D292892B39
:105D500061F481E0F501808360917E0270917F02A1
:105D600080E090E00E94E692EC0160EA78E0CE01EB
:105D70000E94D292892B61F48FEFF50180836091AC
:105D80007E0270917F0280E090E00E94E692EC013A
:105D9000209709F438C16CE978E0CE010E94D292D4
:105DA000892B19F4FF2DF160FF2E68E978E0CE0110
:105DB0000E94D292892B19F48F2D8460F82E65E908
:105DC00078E0CE010E94D292892B19F4EF2DE26087
:105DD000FE2E63E978E0CE010E94D292892B19F45D
:105DE000FF2DF860FF2E60E978E0CE010E94D2928C
:105DF000892B19F48F2D8061F82E6AE878E0CE01A6
:105E00000E94D292892B19F4EF2DE062FE2E64E8F5
:105E100078E0CE010E94D292892B19F4FF2DF06414
:105E2000FF2E61E878E0CE010E94D292892B19F40E
:105E30008F2D8068F82E6CE778E0CE010E94D29218
:105E4000892B09F4016065E778E0CE010E94D292C7
:105E5000892B09F4026062E778E0CE010E94D292B9
:105E6000892B09F404606DE678E0CE010E94D2929D
:105E7000892B09F4086066E678E0CE010E94D29290
:105E8000892B09F400616FE578E0CE010E94D2927F
:105E9000892B09F400626BE578E0CE010E94D29272
:105EA000892B19F4ED2DE460DE2E68E578E0CE0153
:105EB0000E94D292892B09F4006463E578E0CE0158
:105EC0000E94D292892B09F4006860E578E0CE0147
:105ED0000E94D292892B19F4FE2DF160EF2E6DE411
:105EE00078E0CE010E94D292892B19F48E2D826027
:105EF000E82E6AE478E0CE010E94D292892B19F450
:105F0000EE2DE460EE2E66E478E0CE010E94D2929F
:105F1000892B19F4FE2DF860EF2E62E478E0CE01B3
:105F20000E94D292892B19F48E2D8061E82E6EE3A7
:105F300078E0CE010E94D292892B19F4EE2DE06216
:105F4000EE2E6AE378E0CE010E94D292892B19F4FA
:105F5000FE2DF064EF2E68E378E0CE010E94D2922D
:105F6000892B19F48E2D8068E82E65E378E0CE0148
:105F70000E94D292892B09F411606DE278E0CE0183
:105F80000E94D292892B09F4126064E278E0CE017B
:105F90000E94D292892B09F414606BE178E0CE0163
:105FA0000E94D292892B09F4186068E178E0CE0152
:105FB0000E94D292892B09F4106162E178E0CE014F
:105FC0000E94D292892B09F4106267E078E0CE013A
:105FD0000E94D292892B09F4106463E078E0CE012C
:105FE0000E94D292892B19F4ED2DE860DE2E6FEF1E
:105FF00077E0CE010E94D292892B09F0C0CEFD2D10
:10600000F061DF2EBCCE2F2D302F4E2D512F6D2D58
:1060100070E080E090E0DF91CF911F910F91FF90B1
:10602000EF90DF90BF90AF9008955F926F927F9254
:106030008F929F92AF92BF92CF92DF92EF92FF9298
:106040000F931F93CF93DF93782EC8EADCE100E033
:1060500010E089EFE82E87E0F82E872D8170582E0A
:10606000872D8270682E94EEC92E97E0D92E2CEEE3
:10607000A22E27E0B22E3AEE832E37E0932E772021
:1060800051F01F930F93FF92EF920E94C6930F90CF
:106090000F900F900F905520A1F089858F938885E0
:1060A0008F93BF92AF920E94C6930F900F900F9064
:1060B0000F906620C1F09F928F920E94C6930F901E
:1060C0000F90662081F0DF92CF920E94C6932881C4
:1060D00039814A815B816C817D818E819F810E94A3
:1060E000A82A0F900F900E94D0110F5F1F4F2A9681
:1060F0000430110521F6DF91CF911F910F91FF9090
:10610000EF90DF90CF90BF90AF909F908F907F9057
:106110006F905F9008958FED97E09F938F930E940B
:10612000C6938091B5289091B628A091B728B091D8
:10613000B8280F900F90813027EA92072EE1A2072E
:10614000B10519F481ED97E01DC0823026EA92076F
:106150002EE1A207B10519F484EC97E013C0823058
:1061600027EA92072EE1A207B10519F486EB97E022
:1061700009C0823028EA92072EE1A207B10549F44E
:1061800088EA97E09F938F930E94C6930F900F9099
:106190000895BF93AF939F938F9382EA97E09F9365
:1061A0008F930E94C6930F900F900F900F900F90B7
:1061B0000F90089582E997E09F938F930E94C69372
:1061C0000E94E2260E948B300E94D0118FE89CE151
:1061D0009F938F938AE897E09F938F930E94C69333
:1061E00060916002709161028091620290916302FD
:1061F00028EE33E040E050E00E9475885F934F93B3
:106200003F932F938AE797E09F938F930E94C693C3
:1062100081E797E09F938F930E94C6930E94621636
:106220008091C52C2DB73EB7225F3F4F0FB6F89433
:106230003EBF0FBE2DBF80FF05C041E061E081E0A1
:106240000E940F188DE697E09F938F930E94C6934C
:1062500080E00E94C0280E94E626809165021F927D
:106260008F9384E697E09F938F930E94C6938091CB
:106270009C131F928F938BE597E09F938F930E94BF
:10628000C693809190028F9380918F028F9380911B
:106290008E028F9380918D028F938DE497E09F9370
:1062A0008F930E94C6931F9280E48F9385E397E0BB
:1062B0009F938F930E94C6938091A4371F928F93D0
:1062C0008091A3371F928F9382E297E09F938F93E1
:1062D0000E94C693809164021F928F9389E197E098
:1062E0009F938F930E94C69380916602909167025C
:1062F000A0916802B09169022DB73EB7225E3F4F70
:106300000FB6F8943EBF0FBE2DBF96FD03C08CE1C3
:1063100095E002C089E195E09F938F938FE097E02D
:106320009F938F930E94C69383E00E9415300F9035
:106330000F900F900F901D9903C08CE195E002C063
:1063400089E195E09F938F9383E097E09F938F93EC
:106350000E94C69389EF96E09F938F930E94C69305
:10636000809166020F900F900F900F900F900F90FA
:1063700081FF09C083EF96E09F938F930E94C6939D
:106380000F900F9013C080FD03C08CE195E002C018
:1063900089E195E09F938F938FEE96E09F938F9383
:1063A0000E94C6930F900F900F900F9080916602FD
:1063B00090916702A0916802B091690297FD03C0B5
:1063C0008CE195E002C089E195E09F938F9386EE82
:1063D00096E09F938F930E94C6938FED96E09F93D4
:1063E0008F930E94C69360919F137091A013809128
:1063F000A1139091A2130E94FC280E94D0110F902B
:106400000F900F900F900F900F90779B03C08CE12F
:1064100095E002C089E195E09F938F9386ED96E029
:106420009F938F930E94C6930E94530E0E94241143
:106430009F938F937F936F9388EC96E09F938F93B6
:106440000E94C6930E94D3109F938F937F936F9364
:106450008AEB96E09F938F930E94C69381E090E031
:106460000E949C278091743590917535A091763566
:10647000B0917735BF93AF939F938F938CEA96E05B
:106480009F938F930E94C693809189358F938091BB
:1064900088358F93809187358F93809186358F9340
:1064A00088E996E09F938F930E94C69380917835F8
:1064B00090917935A0917A35B0917B35BF93AF93A8
:1064C0009F938F938AE896E09F938F930E94C69341
:1064D0008DB79EB782960FB6F8949EBF0FBE8DBF44
:1064E00080918D358F9380918C358F9380918B35F2
:1064F0008F9380918A358F9386E796E09F938F9351
:106500000E94C69361E070E080E090E00E94D911A3
:1065100061E070E081E090E00E94D9110F900F904F
:106520000F900F900F900F90299903C08CE195E088
:1065300002C089E195E09F938F938EE696E09F934A
:106540008F930E94C6930F900F900F900F902A99EF
:1065500003C08CE195E002C089E195E09F938F93A1
:1065600086E696E09F938F930E94C6930F900F90BC
:106570000F900F900895F89491E2E0E0F0E090938E
:1065800057008491E2E0F0E0909357002491E4E01A
:10659000F0E090935700E49190E0A0E0B0E0BC01FF
:1065A00055274427822F90E0A0E0B0E0BA2FA92F12
:1065B000982F8827840F951FA61FB71F8E0F911D38
:1065C000A11DB11D8093B5289093B628A093B7283C
:1065D000B093B82878940895CF93DF93CDB7DEB702
:1065E00061970FB6F894DEBF0FBECDBF48E250E012
:1065F00062E270E088EA9CE10E9473962091A81CF8
:106600003091A91C4091AA1C5091AB1C6091AC1C0C
:106610007091AD1C8091AE1C9091AF1CAFEF0E94A9
:10662000A88A09F05DC08DE48093A81C80E880935F
:10663000A91C84E08093AA1C1092AB1C1092AC1C85
:106640001092AD1C1092AE1C1092AF1C8CE390E027
:106650009093B11C8093B01C1092B21C1092B31C8A
:106660001092B41C1092B51C1092B61C1092B71C5C
:106670001092B81C1092B91C1092BB1C1092BA1C3C
:106680001092BC1C1092BD1C1092BE1C1092BF1C1C
:106690001092C01C1092C11C1092C21C1092C31CFC
:1066A0001092C51C1092C41C1092C61C1092C71CDC
:1066B0001092C81C1092C91C1092CA1C1092CB1CBC
:1066C0001092CC1C1092CD1C1092CF1C1092CE1C9C
:1066D00048E250E062E270E088EA9CE10E94919614
:1066E00044E050E06EE170E0CE010B960E9473969C
:1066F0008B859C85AD85BE858F3F2FEF9207A207C6
:10670000B207A9F48AE090E4A0E0B0E080936602CA
:1067100090936702A0936802B093690244E050E04E
:106720006EE170E086E692E00E94919608C0809348
:10673000660290936702A0936802B0936902809109
:10674000660290916702A0916802B0916902A2FF6F
:1067500002C02A9A03C080E00E94F62844E050E07C
:106760006AE570E0CE010B960E9473968B859C853E
:10677000AD85BE858F3F2FEF9207A207B20789F440
:1067800010929F131092A0131092A1131092A213B3
:1067900044E050E06AE570E08FE993E10E94919651
:1067A00008C080939F139093A013A093A113B0935C
:1067B000A21349E050E06EE070E08EE895E30E949D
:1067C00073960E94071344E050E06EE470E0CE013F
:1067D0000B960E9473968B859C85AD85BE8544E0A3
:1067E00050E06EE470E08F3F9F4FAF4FBF4F29F4F2
:1067F00085E892E00E94919604C085E892E00E94AC
:10680000739644E050E06AE470E0CE010B960E947B
:1068100073968B859C85AD85BE8544E050E06AE427
:1068200070E08F3F9F4FAF4FBF4F29F481E892E058
:106830000E94919604C081E892E00E94739644E021
:1068400050E062E570E0CE010B960E9473968B8556
:106850009C85AD85BE8544E050E062E570E08F3FE9
:106860009F4FAF4FBF4F29F489E892E00E94919665
:1068700004C089E892E00E94739641E050E06DE127
:1068800070E0CE0141960E947396898941E050E004
:106890006DE170E08F3F29F48CE993E10E949196BD
:1068A00004C08CE993E10E94739641E050E06CE1F2
:1068B00070E0CE0141960E947396898941E050E0D4
:1068C0006CE170E08F3F29F485E692E00E9491969A
:1068D00004C085E692E00E94739641E050E06BE1CF
:1068E00070E0CE0141960E947396898941E050E0A4
:1068F0006BE170E08F3F29F484E692E00E9491966C
:1069000004C084E692E00E9473964AE050E064E09E
:1069100070E0CE0101960E94739689814AE050E0B2
:1069200064E070E08F3F29F48FE89CE10E9491962B
:1069300004C08FE89CE10E94739644E050E066E555
:1069400070E0CE010B960E9473968B859C85AD8579
:10695000BE8544E050E066E570E08F3F9F4FAF4F4B
:10696000BF4F29F48DE892E00E94919604C08DE813
:1069700092E00E94739644E050E067E170E0CE013F
:106980000B960E9473968B859C85AD85BE8544E0F1
:1069900050E067E170E08F3F9F4FAF4FBF4F29F44A
:1069A00080E692E00E94919604C080E692E00E9408
:1069B00073968091600290916102A0916202B09101
:1069C000630281389A41A640B105A0F083EF92E0BE
:1069D0009F938F930E94C69380E197E2A0E0B0E07E
:1069E0008093600290936102A0936202B09363026D
:1069F0000F900F9042E050E062E070E0CE010F9601
:106A00000E9473968F85988942E050E062E070E0C2
:106A10008F3F910529F485E993E10E94919604C086
:106A200085E993E10E94739642E050E060E070E0F7
:106A3000CE010F960E9473968F85988942E050E0B0
:106A400060E070E08F3F910529F483E993E10E94B3
:106A5000919604C083E993E10E94739661960FB604
:106A6000F894DEBF0FBECDBFDF91CF910895CF92D6
:106A7000DF92EF92FF9260917E0270917F0280E040
:106A800090E00E94E69260E275E00E940793892BF5
:106A900009F03BC18DE48093A81C80E88093A91C79
:106AA00084E08093AA1C1092AB1C1092AC1C109234
:106AB000AD1C1092AE1C1092AF1C8CE390E0909332
:106AC000B11C8093B01C1092B21C1092B31C109297
:106AD000B41C1092B51C1092B61C1092B71C1092E8
:106AE000B81C1092B91C1092BB1C1092BA1C1092C8
:106AF000BC1C1092BD1C1092BE1C1092BF1C1092A8
:106B0000C01C1092C11C1092C21C1092C31C109287
:106B1000C51C1092C41C1092C61C1092C71C109267
:106B2000C81C1092C91C1092CA1C1092CB1C109247
:106B3000CC1C1092CD1C1092CF1C1092CE1C48E29F
:106B400050E062E270E088EA9CE10E9491968AE05F
:106B500090E4A0E0B0E08093660290936702A09377
:106B60006802B093690244E050E06EE170E086E6AE
:106B700092E00E94919610929F131092A01310928F
:106B8000A1131092A21344E050E06AE570E08FE98F
:106B900093E10E94919682E2C82EDD24DA948CEC77
:106BA000E82E8BE3F82EC0928502D0928602E09206
:106BB0008702F092880244E050E06EE470E085E8DD
:106BC00092E00E949196C0928102D0928202E0925D
:106BD0008302F092840244E050E06AE470E081E8CD
:106BE00092E00E94919687ED94E3AFEEBCE3809330
:106BF000890290938A02A0938B02B0938C0244E0A6
:106C000050E062E570E089E892E00E9491968AE99E
:106C100099E9A9E1B0E480938D0290938E02A0934C
:106C20008F02B093900244E050E066E570E08DE89A
:106C300092E00E94919610929C1380E00E94AD6AAF
:106C400041E050E06DE170E08CE993E10E949196A3
:106C50008AE1809365020E94866941E050E06CE120
:106C600070E085E692E00E9491968FE08093640246
:106C700041E050E06BE170E084E692E00E94919682
:106C80008AE0EFE8FCE1DF011D928A95E9F74AE02E
:106C900050E064E070E0CF010E94919680E197E2BD
:106CA000A0E0B0E08093600290936102A093620242
:106CB000B093630244E050E067E170E080E692E068
:106CC0000E949196109296131092951342E050E014
:106CD00062E070E085E993E10E949196109294132E
:106CE0001092931342E050E060E070E083E993E19A
:106CF0000E94919681E00E94C02880E090E0FF9081
:106D0000EF90DF90CF900C941C13FF90EF90DF90EA
:106D1000CF9008950E94A4666C9A6B9A6A9A6F9AB3
:106D2000729A749A739A779A809880B3897F80BB9D
:106D30008398849887E080937E00549A0E94BB32A7
:106D40000E94EC320E94C10E80E090E00E941C1371
:106D50006091600270916102809162029091630281
:106D60000E943D600E94D3106093C7307093C8307A
:106D70008093C9309093CA308091660286FD239A31
:106D8000219A229A239A0E94D60E1D9B05C010922A
:106D90009E1310929D13089581E090E090939E13AE
:106DA00080939D130895CF93DF9390E040919F13BC
:106DB0005091A0136091A1137091A21341FD08C0DE
:106DC0002091660220FD04C021FF8CC01D9B8AC05B
:106DD0002DE8289FE001299FD00D1124CE018B546E
:106DE000924E9F938F9387E295E09F938F930E949B
:106DF000B293FE01E255F24EDF01AA57BF4F2C912C
:106E00000F900F900F900F90438154816581768190
:106E10008091CB309091CC30A091CD30B091CE30DC
:106E2000841B950BA60BB70B2223D1F1BF93AF9315
:106E30009F938F93DF01A257BF4F11968C911197AB
:106E40008F938C918F93129711968C9111978F93AA
:106E50008C918F9313978C911F928F9311978C9194
:106E60001F928F9313968C911F928F9311978C91F1
:106E70001F928F93E957FF4F80811F928F931F922C
:106E80002F938DE295E09F938F930E94B2938DB7DD
:106E90009EB746960FB6F8949EBF0FBE8DBF10C02A
:106EA000BF93AF939F938F9384E795E09F938F93C6
:106EB0000E94B2930F900F900F900F900F900F9031
:106EC0000E94D01180918002882361F01F928F93DD
:106ED00080EF92E09F938F930E94C6930F900F9044
:106EE0000F900F90DF91CF9108958091AE1D882370
:106EF00041F08091AF1D90E00E94D3360E94C70FF1
:106F0000F4CF0895CF93DF93EC0188819981873E78
:106F10002EE09207F1F018F4892BC1F04BC08F3EA0
:106F20002EE0920709F44CC0833F9E4009F042C016
:106F300086E59AE00E94EB6E892B09F43FC086E556
:106F40009AE00E94D76E80E00E94F02887EE9EE0D3
:106F50002EC0623199F5299A409193135091941360
:106F60005695542F44275795479560E070E086E585
:106F70009AE00E94CD6E80919F139091A013A091F2
:106F8000A113B091A213A0FF10C0809194138F930E
:106F9000809193138F9380EC91E19F938F930E9444
:106FA000C6930F900F900F900F908FEE9EE09983F5
:106FB000888304C01982188283E019C081E017C059
:106FC00086E59AE00E94EB6E892BC1F386E59AE094
:106FD0000E94D76E0E94753740E250E060E070E09A
:106FE00086E59AE00E94CD6E83EF9EE0E0CFDF91D0
:106FF000CF9108952F923F924F925F926F927F921E
:107000008F929F92AF92BF92CF92DF92EF92FF92B8
:107010000F931F93CF93DF93CDB7DEB72B970FB6A8
:10702000F894DEBF0FBECDBF9B878A873A01FC0173
:1070300080819181892B11F00C94274C60917E0204
:1070400070917F02CA010E94E69260E870E0C3017D
:107050000E942693009759F46091F7397091F8399E
:107060008AE090E00E947A9381E00C942C4C81306D
:10707000910561F4F3011081912E990C9908892CE6
:10708000092D292C392C492C592CB9C08230910555
:10709000B9F4F3018081082E000C990B982F8827F2
:1070A0002181820F911D27FD9A95182F992E892EE7
:1070B000880C8808082D282C382C482C582C9FC068
:1070C00083309105B1F5F3012081922F990F990B2F
:1070D000392F492F592F692F792F892F00E10E94CD
:1070E0004A8A19012A014B01B82FA92F2181922F19
:1070F000990F990B392F492F592F692F792F892FE4
:1071000008E00E944A8A59016A017B018C019101C1
:10711000A201B4018B2F9A2F0E94818AA2801A2D7E
:10712000110F110BB12EC12ED12EE12EF12E012FF8
:1071300055C004970CF45BC0F3012081922F990F86
:10714000990B392F492F592F692F792F892F08E152
:107150000E944A8A19012A014B01B82FA92F2181C7
:10716000922F990F990B392F492F592F692F792F6A
:10717000892F00E10E944A8A59016A017B018C0132
:107180009101A201B4018B2F9A2F0E94818AA380C2
:107190001A2D110F110BB12EC12ED12EE12EF12E71
:1071A000012F0E94818A19012A014B01B82FA92FB2
:1071B0002281922F990F990B392F492F592F692F1F
:1071C000792F892F08E00E944A8A59016A017B01C0
:1071D0008C019101A201B4018B2F9A2F0E94818A08
:1071E000122F932E842E052F1B012C0108C01AE0AC
:1071F000912C812C00E0212C312C412C512C0E940F
:10720000D011212F392D482D502FB101C201253722
:10721000F3E63F07FDE64F0751056105710581055E
:10722000910511F40C940F472537E3E63E07EDE690
:107230004E075105610571058105910511F008F0B2
:10724000B2C12337F2E73F074105510561057105DA
:107250008105910511F40C94A8492337E2E73E0714
:1072600041055105610571058105910511F008F091
:10727000B9C02536F4E63F074105510561057105A2
:107280008105910509F4D1C72536E4E63E0741059D
:107290005105610571058105910511F008F041C0A6
:1072A000A6E70E94A88A11F40C9497430E94A88A2A
:1072B00009F070F4A8E60E94A88A11F40C946641C3
:1072C000A5E70E94A88A11F40C9481430C94254CE4
:1072D000212F392D482D502FB101C2012436F1E65E
:1072E0003F0741055105610571058105910511F4BF
:1072F0000C94D0492537E2E63E074105510561056A
:1073000071058105910509F431C52A3336424105DD
:107310005105610571058105910509F430C30C948F
:10732000254C212F392D482D502FB101C20127376F
:10733000EFE63E074105510561057105810591059F
:1073400011F40C9475472737FFE63F0741055105B7
:10735000610571058105910509F0C8F42436E9E657
:107360003E0741055105610571058105910511F43F
:107370000C945A4325363E46410551056105710579
:107380008105910511F40C94A9470C94254C212FEB
:10739000392D482D502FB101C2012536E2E73E07B5
:1073A00041055105610571058105910511F40C94A4
:1073B00075482936F2E73F0741055105610571051A
:1073C0008105910511F40C94574923333147410548
:1073D0005105610571058105910511F00C94254C4D
:1073E0000C94D049212F392D482D502FB101C201C5
:1073F0002236F5E63F07F4E64F07510561057105B2
:107400008105910509F411C72236E5E63E07E4E659
:107410004E075105610571058105910511F008F0D0
:107420005BC02133F4E63F07F1E64F0751056105E4
:1074300071058105910509F4B6C22133E4E63E07E2
:10744000E1E64E075105610571058105910509F0D9
:10745000C0F42337F3E73F07410551056105710586
:107460008105910511F40C94BC4928373447410536
:107470005105610571058105910509F480C20C94DF
:10748000254C212F392D482D502FB101C20128370D
:10749000F4E63F07F1E64F075105610571058105E7
:1074A000910509F47CC22C36E5E73E07E2E64E077B
:1074B0005105610571058105910509F457C423360D
:1074C000344641465105610571058105910511F06C
:1074D0000C94254C0C94D049212F392D482D502F38
:1074E000B101C2012D36E5E73E07E8E64E0751053A
:1074F000610571058105910511F40C94E6492D365D
:10750000F5E73F07F8E64F0751056105710581056D
:10751000910509F0E0F42237E2E73E07E5E64E0781
:107520005105610571058105910511F40C94C04662
:1075300023363D4648465105610571058105910593
:1075400011F00C94254C0E946C1C0C94274C212F9C
:10755000392D482D502FB101C2012436E3E63E07F4
:10756000ECE64E075105610571058105910511F4A1
:107570000C9423462736FFE63F07FCE64F075105EC
:10758000610571058105910511F40C942646233699
:10759000324349465105610571058105910511F098
:1075A0000C94254C20C2212F392D482D502FB1018C
:1075B000C2012037FCE63F07F5E64F07F8E65F0714
:1075C000610571058105910509F480C62037ECE657
:1075D0003E07E5E64E07E8E65E07610571058105B1
:1075E000910511F008F0E0C02437F8E73F07F4E711
:1075F0004F075105610571058105910511F40C9442
:1076000003442437E8E73E07E4E74E0751056105E8
:1076100071058105910511F008F05DC02033F1E39B
:107620003F07F1E74F075105610571058105910598
:1076300011F40C94C0462033E1E33E07E1E74E0726
:107640005105610571058105910509F0C0F42133EB
:10765000F2E63F07F0E74F07510561057105810527
:10766000910509F498C2223332464047510561051D
:1076700071058105910509F4E3C20C94254C212F75
:10768000392D482D502FB101C2012037F5E63F07B3
:10769000F2E74F075105610571058105910511F468
:1076A0000C9475482C36E4E73E074E0751056105FA
:1076B00071058105910511F40C944B4B2133314335
:1076C00041475105610571058105910511F00C9443
:1076D000254C0C940F47212F392D482D502FB101E7
:1076E000C2012B36ECE63E07E5E74E07E2E65E0711
:1076F000610571058105910509F438C32B36FCE657
:107700003F07F5E74F07F2E65F0761057105810561
:10771000910509F0E0F42437E4E63E07E7E74E0779
:107720005105610571058105910511F40C94994B82
:1077300024373F464F465246610571058105910544
:1077400011F00C94254C0C9400000C94274C212F24
:10775000392D482D502FB101C2012E36E1E63E07EA
:10776000E8E64E07E3E65E076105710581059105D0
:1077700011F40C94D7432633F9E63F07F5E74F079A
:10778000F5E65F07610571058105910509F4A2C55C
:1077900029363C46414653466105710581059105F0
:1077A00011F00C94254C7FC3212F392D482D502FDB
:1077B000B101C2012437F3E73F07F5E64F07F2E7CF
:1077C0005F07610571058105910511F40C94254849
:1077D0002437E3E73E07E5E64E07E2E75E0761058B
:1077E00071058105910511F008F062C02337F5E6B7
:1077F0003F07F2E74F07F0E75F0761057105810575
:10780000910511F40C94964A2337E5E63E07E2E72A
:107810004E07E0E75E07610571058105910509F0F6
:10782000D0F42136FDE63F07F5E74F07F8E65F079E
:10783000610571058105910511F40C949347223778
:10784000374740475047610571058105910509F4A7
:107850005CC20C94254C212F392D482D502FB1019D
:10786000C2012436FDE63F07F3E64F07F2E75F0764
:10787000610571058105910509F437C62136ECE6ED
:107880003E07E5E64E07E2E75E0761057105810503
:10789000910509F43CC523373247474750476105F6
:1078A00071058105910511F00C94254C0C94284824
:1078B000212F392D482D502FB101C2012437E2E785
:1078C0003E07E1E64E07E5E75E07610571058105C4
:1078D000910509F465C62437F2E73F07F1E64F0743
:1078E000F5E75F07610571058105910509F0C8F4A9
:1078F0002437E3E73E07E5E64E07E4E75E07610568
:1079000071058105910509F4A9C727373047484714
:107910005447610571058105910509F41EC70C9452
:10792000254C212F392D482D502FB101C2012F3662
:10793000ECE63E07EFE54E07E6E75E0761057105F9
:107940008105910509F47CC52C36F1E63F07F4E783
:107950004F07F8E75F07610571058105910511F48F
:107960000C94184B2237374640475547610571053F
:107970008105910511F00C94254C0C94FF4583E092
:1079800080937C3510927E3510927D354CE755E31F
:1079900062E182E492E00E945D700C94274C0E94A8
:1079A000F51B0C94274C21E042E161E080ED0E9440
:1079B0001A6221E042E161E080ED0E941A6221E05A
:1079C00042E161E080ED0E941A6221E042E161E063
:1079D00080ED0E941A6221E042E161E080ED0E94A8
:1079E0001A620C94274C60917E0270917F0280E0B5
:1079F00090E00E94E69260E875E00E940793892B70
:107A000009F0C5C060917E0270917F0280E090E035
:107A10000E94E6928C01009709F497C064E673E037
:107A20000E940793892BE1F488EE93E0A0E0B0E098
:107A30008093600290936102A0936202B09363020C
:107A400068EE73E080E090E00E943D6044E050E02A
:107A500067E170E080E692E00E9491960C94274CDA
:107A600066E875E0C8010E940793892BE1F480E184
:107A700097E2A0E0B0E08093600290936102A0934F
:107A80006202B093630260E177E280E090E00E94DE
:107A90003D6044E050E067E170E080E692E00E94E3
:107AA00091960C94274C69E875E0C8010E940793F1
:107AB000892BE1F480EA96E8A1E0B0E080936002CF
:107AC00090936102A0936202B093630260EA76E849
:107AD00081E090E00E943D6044E050E067E170E0AA
:107AE00080E692E00E9491960C94274C6DE875E038
:107AF000C8010E940793892BE1F480E89AE1A6E08F
:107B0000B0E08093600290936102A0936202B09310
:107B1000630260E87AE186E090E00E943D6044E024
:107B200050E067E170E080E692E00E9491960C944C
:107B3000274C8EE994E09F938F930E94C6930E94F6
:107B4000D0110F900F900C94274C609160027091AF
:107B50006102809162029091630228EE33E040E07E
:107B600050E00E9475885F934F933F932F938AE96B
:107B700094E09F938F930E94C6930E94D0110F9020
:107B80000F900F900F900F900F900C94274C0E9425
:107B900062160C94274C60917E0270917F0280E007
:107BA00090E00E94E6928C0169E175E00E940793E3
:107BB000892BA1F48091660290916702A0916802DE
:107BC000B0916902A2608093660290936702A093CD
:107BD0006802B0936902299A0C94274C6CE175E015
:107BE000C8010E940793892BB1F48091660290919D
:107BF0006702A0916802B0916902AD7F809366022E
:107C000090936702A0936802B093690280E00E949B
:107C1000F0280C94274C299903C08CE195E002C010
:107C200089E195E09F938F9382E994E09F938F93EE
:107C30000E94C6930F900F900F900F900C94274CBA
:107C400060917E0270917F0280E090E00E94E69257
:107C50008C0169E175E00E940793892BE1F4809122
:107C6000660290916702A0916802B0916902A460D7
:107C70008093660290936702A0936802B0936902B2
:107C80002A9A44E050E06EE170E086E692E00E94BD
:107C900091960C94274C6CE175E0C8010E94079303
:107CA000892BF1F48091660290916702A09168029D
:107CB000B0916902AB7F8093660290936702A093B4
:107CC0006802B093690280E00E94F62844E050E028
:107CD0006EE170E086E692E00E9491960C94274C4B
:107CE0002A9903C08CE195E002C089E195E09F9359
:107CF0008F938AE894E09F938F930E94C6930F908E
:107D00000F900F900F900C94274C60917E02709111
:107D10007F0280E090E00E94E6928C0169E175E0CC
:107D20000E940793892B19F477980C94274C6CE1E7
:107D300075E0C8010E940793892B19F4779A0C9477
:107D4000274C779B03C08CE195E002C089E195E068
:107D50009F938F9380E596E09F938F930E94C693A5
:107D60000F900F900F900F900C94274C60917E0213
:107D700070917F0280E090E00E94E6928C0161E9C0
:107D800075E00E940793892BD1F48091AE1D1F925C
:107D90008F938091B01D1F928F938091AF1D1F9282
:107DA0008F931F9284E18F9380E694E09F938F934B
:107DB0000E94C6930FB6F894DEBF0FBECDBF66E932
:107DC00075E0C8010E940793892B19F40E9475374A
:107DD00066C06EE975E0C8010E940793892BF1F532
:107DE00060917E0270917F0280E090E00E94E692B6
:107DF000009709F454C00E94D3918531910528F56C
:107E0000909396138093951342E050E062E070E007
:107E100085E993E10E94919660917E0270917F02C4
:107E200080E090E00E94E6920097C9F10E94D39111
:107E3000909394138093931342E050E060E070E0DD
:107E400083E993E10E9491962AC08EE494E09F9387
:107E50008F930E94C6930F900F9021C0809196132C
:107E60008F93809195138F9385E494E09F938F93E4
:107E70000E94C6930E94D011809194138F93809199
:107E800093138F9386E394E09F938F930E94C693FE
:107E90000E94D0110FB6F894DEBF0FBECDBF0E9476
:107EA000D0110C94274C60917E0270917F0280E08B
:107EB00090E00E94E6928C016EED74E00E940793C0
:107EC000892B09F077C060917E0270917F0280E07B
:107ED00090E00E94E6928C01009711F40C94274CDC
:107EE0006CE975E00E940793892BB1F482E29FEF61
:107EF000ACECBBE38093850290938602A09387024B
:107F0000B093880244E050E06EE470E085E892E0CF
:107F10000E9491960C94274C62EA75E0C8010E9479
:107F20000793892BB1F482E29FEFACECBAE3809324
:107F3000850290938602A0938702B093880244E062
:107F400050E06EE470E085E892E00E9491960C9417
:107F5000274CC8010E94CF912B013C0120E030E06A
:107F6000A9010E94938B8823D9F081E00E947110AF
:107F70009B01AC01C301B2010E94988B6093850202
:107F800070938602809387029093880244E050E0C9
:107F90006EE470E085E892E00E9491960C94274C84
:107FA00089E294E09F938F930E94C6930F900F9065
:107FB0000C94274C61EE74E0C8010E940793892B52
:107FC00009F077C060917E0270917F0280E090E0BE
:107FD0000E94E6928C01009711F40C94274C6CE9F6
:107FE00075E00E940793892BB1F482E29FEFACEC1D
:107FF000BBE38093810290938202A0938302B093AB
:10800000840244E050E06AE470E081E892E00E947B
:1080100091960C94274C62EA75E0C8010E94079380
:10802000892BB1F482E29FEFACECBAE3809381023A
:1080300090938202A0938302B093840244E050E0C4
:108040006AE470E081E892E00E9491960C94274CDB
:10805000C8010E94CF912B013C0120E030E0A90132
:108060000E94938B8823D9F082E00E9471109B01BB
:10807000AC01C301B2010E94988B6093810270939E
:108080008202809383029093840244E050E06AE489
:1080900070E081E892E00E9491960C94274C8CE16C
:1080A00094E09F938F930E94C6930F900F900C942F
:1080B000274C69ED74E0C8010E940793892B09F0F1
:1080C00073C060917E0270917F0280E090E00E9418
:1080D000E6928C01009711F40C94274C6CE975E042
:1080E0000E940793892BB1F487ED94E3AFEEBCE3D4
:1080F0008093890290938A02A0938B02B0938C02A2
:1081000044E050E062E570E089E892E00E949196D8
:108110000C94274C62EA75E0C8010E940793892BF2
:1081200051F48DE094E09F938F930E94C6930F903B
:108130000F900C94274CC8010E94CF912B013C0159
:1081400020E030E0A9010E94938B882319F180E0A0
:108150000E9471104B015C0121EE3AE744E95EE3B5
:10816000C301B2010E94B48AA50194010E94988BB8
:108170006093890270938A0280938B0290938C02A1
:1081800044E050E062E570E089E892E00E94919658
:108190000C94274C80E094E09F938F930E94C693A9
:1081A0000F900F900C94274C0E94BF109F938F93B9
:1081B0007F936F9389EF93E09F938F930E94C69371
:1081C00082E00E94711020918102309182024091E0
:1081D0008302509184020E94448E162F072FF82E9E
:1081E000E92E81E00E947110EF92FF920F931F938E
:1081F0002091850230918602409187025091880239
:108200000E94448E9F938F937F936F938DEE93E0A4
:108210009F938F930E94C6930E94D0110FB6F8943B
:10822000DEBF0FBECDBF0C94274C60917E027091D3
:108230007F0280E090E00E94E692009711F10E9498
:10824000EF2900919F131091A0132091A113309159
:10825000A213601771078207930739F160939F1388
:108260007093A0138093A1139093A21344E050E065
:108270006AE570E08FE993E10E94919689E496E0C7
:1082800002C082E496E09F938F930E94C693609110
:108290009F137091A0138091A1139091A2130E943B
:1082A000FC280E94D0110F900F9087E396E09F93D7
:1082B0008F930E94C6936FEF7FEFCB010E94FC2843
:1082C0000E94D0110F900F900C94274C0E94DF2534
:1082D0000C94274CF3018481843329F440E061E05D
:1082E00080E00E940F1880918002882311F40C9482
:1082F000274C1F928F9384E396E09F938F930E9465
:10830000C6930F900F900F900F900C94274CF30191
:108310008481893709F080C060917E0270917F026C
:1083200080E090E00E94E6928C0169E175E00E9495
:108330000793892B51F48091660290916702A09176
:108340006802B0916902906410C06CE175E0C801E8
:108350000E940793892BD1F4809166029091670265
:10836000A0916802B09169029F7B8093660290930E
:108370006702A0936802B093690244E050E06EE1A6
:1083800070E086E692E00E94919646C067EA75E04A
:10839000C8010E940793892B21F58091A71C8F9318
:1083A0008091A61C8F938091A51C8F938091A41C13
:1083B0008F938091A31C8F938091A21C8F938091A7
:1083C000A11C8F938091A01C8F9382EC93E09F93CC
:1083D0008F930E94C6930FB6F894DEBF0FBECDBF39
:1083E0001BC08091660290916702A0916802B091D3
:1083F000690296FD03C08CE195E002C089E195E039
:108400009F938F938EEB93E09F938F930E94C693DD
:108410000F900F900F900F9080918002882311F49D
:108420000C94274C1F928F9381E396E09F938F9338
:108430000E94C6930F900F900F900F900C94274CB2
:10844000F30184818737E9F560917E0270917F02A4
:1084500080E090E00E94E6920097D9F00E94CF91D0
:108460002B013C0120E030E0A9010E94938B88237E
:1084700081F040928D0250928E0260928F02709233
:10848000900244E050E066E570E08DE892E00E94E2
:108490009196809190028F9380918F028F9380911B
:1084A0008E028F9380918D028F9380EB93E09F9348
:1084B0008F930E94C6930F900F900F900F900F9084
:1084C0000F9080918002882311F40C94274C1F9206
:1084D0008F938EE296E09F938F930E94C6930F90A6
:1084E0000F900F900F900C94274C60917E0270912A
:1084F0007F0280E090E00E94E6928C0169E175E0E5
:108500000E94079340906602509067026090680254
:1085100070906902892B19F4689457F809C06CE1CE
:1085200075E0C8010E940793892B99F4E89457F8E5
:1085300040926602509267026092680270926902ED
:1085400044E050E06EE170E086E692E00E94919691
:1085500013C057FC03C08CE195E002C089E195E0AF
:108560009F938F938CEA93E09F938F930E94C6937F
:108570000F900F900F900F9080918002882311F43C
:108580000C94274C1F928F938BE296E09F938F93CE
:108590000E94C6930F900F900F900F900C94274C51
:1085A00060917E0270917F0280E090E00E94E692EE
:1085B0008C016DEA75E00E940793892B11F489E123
:1085C00008C061EB75E0C8010E940793892B49F44C
:1085D00080E18093C4001092C50082E08093C000C7
:1085E00055C065EB75E0C8010E940793892B11F413
:1085F00088E0EFCF6AEB75E0C8010E940793892BF2
:1086000039F06FEB75E0C8010E940793892B11F4D4
:1086100083E0DFCF8091C400893141F487EA93E0A1
:108620009F938F930E94C6930F900F908091C400E8
:10863000803141F482EA93E09F938F930E94C69326
:108640000F900F908091C400883041F48CE993E042
:108650009F938F930E94C6930F900F908091C400B8
:10866000833041F486E993E09F938F930E94C693F1
:108670000F900F908091C400883041F480E993E01E
:108680009F938F930E94C6930F900F9080918002CA
:10869000882311F40C94274C1F928F9388E296E064
:1086A0009F938F930E94C6930F900F900F900F90FF
:1086B0000C94274C60917E0270917F0280E090E0E4
:1086C0000E94E6926CE975E00E940793892B11F4F1
:1086D00081E001C080E00E94C02880918002882350
:1086E00011F40C94274C1F928F9385E296E09F9390
:1086F0008F930E94C6930F900F900F900F900C9441
:10870000274C0E94E62680918002882311F40C9465
:10871000274C1F928F9382E296E09F938F930E9443
:10872000C6930F900F900F900F900C94274C0E94BF
:10873000E22680918002882311F40C94274C1F922A
:108740008F938FE196E09F938F930E94C6930F9033
:108750000F900F900F900C94274C60917E027091B7
:108760007F0280E090E00E94E6920E94D3918031E7
:1087700070F480939C130E94AD6A41E050E06DE17B
:1087800070E08CE993E10E9491960C94274C8091C3
:108790009C131F928F9386E893E09F938F930E9480
:1087A000C6930F900F900F900F900C94274C6091F0
:1087B0007E0270917F0280E090E00E94E6920E942B
:1087C000D39195EF980F903170F4809365020E94D9
:1087D000866941E050E06CE170E085E692E00E943D
:1087E00091960C94274C809165021F928F938DE790
:1087F00093E09F938F930E94C6930F900F900F90DA
:108800000F900C94274C60917E0270917F0280E063
:1088100090E00E94E692009789F04AE050E0BC01A7
:108820008FE89CE10E9417934AE050E064E070E01A
:108830008FE89CE10E9491960C94274C8FE89CE174
:108840009F938F9384EC95E09F938F930E94B293B4
:108850000F900F900F900F900C94274C60917E0218
:1088600070917F0280E090E00E94E6928C0164E6C5
:1088700073E00E940793892BD9F4219A80916602B4
:1088800090916702A0916802B09169028061809323
:10889000660290936702A0936802B093690244E075
:1088A00050E06EE170E086E692E00E949196CFC7BC
:1088B00062EE74E0C8010E940793892BD9F4229AD2
:1088C0008091660290916702A0916802B09169025E
:1088D00080628093660290936702A0936802B093CF
:1088E000690244E050E06EE170E086E692E00E94AA
:1088F0009196ADC766E473E0C8010E940793892B87
:10890000D9F4239A8091660290916702A09168023F
:10891000B091690280648093660290936702A0938D
:108920006802B093690244E050E06EE170E086E6D0
:1089300092E00E9491968BC765E874E0C8010E949E
:108940000793892BD9F4239A80916602909167024C
:10895000A0916802B091690280688093660290934A
:108960006702A0936802B093690244E050E06EE1B0
:1089700070E086E692E00E94919669C76AE779E026
:10898000C8010E940793892B71F581E08093E03044
:1089900088EA9CE19093E2308093E1301092E430D9
:1089A0001092E3308091660290916702A091680274
:1089B000B091690291608093660290936702A093E0
:1089C0006802B093690244E050E06EE170E086E630
:1089D00092E00E94919640EE50E362E182E492E0E0
:1089E0000E945D7034C76DE673E0C8010E94079372
:1089F000892B11F5E8EDFCE1119211922CE1E83F91
:108A0000F207D1F78091660290916702A091680207
:108A1000B091690292608093660290936702A0937E
:108A20006802B093690244E050E06EE170E086E6CF
:108A300092E00E9491960BC76CE175E0C8010E941C
:108A400007934091660250916702609168027091AD
:108A50006902892BC1F44F705C7F4093660250938A
:108A6000670260936802709369022B9A44E050E0B9
:108A70006EE170E086E692E00E94919680918535E5
:108A80000E949B69E4C644FD03C08CE195E002C0EE
:108A900089E195E09F938F9382E793E09F938F9373
:108AA0000E94C693809166020F900F900F900F90D6
:108AB00085FD03C08CE195E002C089E195E09F93BC
:108AC0008F9387E693E09F938F930E94C693809144
:108AD00066020F900F900F900F9086FD03C08CE1FF
:108AE00095E002C089E195E09F938F938CE593E038
:108AF0009F938F930E94C693809166020F900F9070
:108B00000F900F9087FD03C08CE195E002C089E1D2
:108B100095E09F938F9381E593E09F938F930E94BD
:108B2000C6938091660290916702A0916802B0910D
:108B300069020F900F900F900F9090FD03C08CE191
:108B400095E002C089E195E09F938F9386E493E0DE
:108B50009F938F930E94C6938091660290916702C3
:108B6000A0916802B09169020F900F900F900F9042
:108B700091FD03C08CE195E002C089E195E09F93EF
:108B80008F938BE393E09F938F930E94C693809182
:108B9000660290916702A0916802B09169020F90FD
:108BA0000F900F900F9091FF52C68CEC95E00E94B1
:108BB000EE9398EDE92E9CE1F92E00E010E024ED13
:108BC000822E25E0922EF70180819181F2E0EF0E56
:108BD000F11C9F938F93C8010B969F938F939F9245
:108BE0008F920E94B2930F5F1F4F0F900F900F90C4
:108BF0000F900F900F900031110529F728C68BE1D7
:108C000096E09F938F930E94C693809180020F906D
:108C10000F90882361F01F928F9388E196E09F93D5
:108C20008F930E94C6930F900F900F900F90F8941F
:108C300098E088E10FB6F894A895809360000FBE85
:108C400090936000FFCF0E94CB6101C660917E02CD
:108C500070917F0280E090E00E94E6928C0169E1D1
:108C600075E00E940793892BE9F40E948A6880913D
:108C7000660290916702A0916802B09169028D7FAF
:108C800081608093660290936702A0936802B0931C
:108C9000690244E050E06EE170E086E692E00E94F6
:108CA0009196D5C56CE175E0C8010E940793892BA8
:108CB000E1F40E94C0678091660290916702A091E2
:108CC0006802B09169028C7F80936602909367027C
:108CD000A0936802B093690244E050E06EE170E056
:108CE00086E692E00E949196B2C56FED75E0C801EC
:108CF0000E940793892BE9F40E94C0678091660265
:108D000090916702A0916802B09169028E7F8260A3
:108D10008093660290936702A0936802B093690201
:108D200044E050E06EE170E086E692E00E949196A9
:108D30008EC58091660281FF0FC08FED95E09F93F5
:108D40008F9387E393E09F938F930E94C6930F9036
:108D50000F900F900F907BC580FD03C08CE195E0D4
:108D600002C089E195E09F938F9383E393E09F9303
:108D70008F930E94C6930F900F900F900F9067C52E
:108D80008091DE308F938091DD308F938091DC3045
:108D90008F938091DB308F938091DA308F93809125
:108DA000D9308F938091D8308F938091D7308F9323
:108DB0008091D6308F938091D5308F938091D4302D
:108DC0008F938091D3308F938091D2308F93809105
:108DD000D1308F938091D0308F938091CF308F930B
:108DE0008CEE95E09F938F930E94C6930E94D011C2
:108DF000809180020FB6F894DEBF0FBECDBF8823EE
:108E000009F425C51F928F9389EE95E09F938F9368
:108E10000E94C6930F900F900F900F9018C5F89472
:108E200089E021E030E0F90180935700C895E02CFB
:108E300020E030E0F90180935700C895F02C789439
:108E4000F89423E030E0F90180935700C895002D95
:108E500022E030E0F90180935700C895102D7894F6
:108E60008091B8288F938091B7288F938091B628EE
:108E70008F938091B5288F938FED95E09F938F937B
:108E80000E94C6931F92EF921F92FF921F920F9320
:108E90001F921F9388EB95E09F938F930E94C69338
:108EA0000E948027809166001F928F938CEA95E044
:108EB0009F938F930E94C6930E94D011809180024D
:108EC0000FB6F894DEBF0FBECDBF882309F4BFC430
:108ED0001F928F9389EA95E09F938F930E94C69388
:108EE0000F900F900F900F90B2C460E070E080E0A0
:108EF00090E00E94D91160E070E081E090E00E9473
:108F0000D91180918002882309F4A1C41F928F9304
:108F100086EA95E09F938F930E94C6930F900F90DF
:108F20000F900F9094C40E94A2250E94D0118091AE
:108F30008002882309F48BC41F928F9383EA95E003
:108F40009F938F930E94C6930F900F900F900F9056
:108F50007EC460917E0270917F0280E090E00E946A
:108F6000E69266E975E00E940793892B31F5F89443
:108F700081E99AE00E9436718C01892B69F0C80161
:108F80000F960E94A36DB80188E092E00E94E771FD
:108F9000C8010E949B71F0CF81E99AE00E948E7116
:108FA000892B29F081E99AE00E944A71F5CF81E985
:108FB0009AE00E943271789436C081E99AE00E946A
:108FC00036718C0184EEE82E85E0F82E011511052E
:108FD00051F1F80186811F928F9380851F928F93A4
:108FE00085811F928F9381851F928F9387811F9216
:108FF0008F9384811F928F9383811F928F9382819D
:109000001F928F9382851F928F93FF92EF920E94FF
:10901000B293C8010E949B718C010FB6F894DEBF19
:109020000FBECDBFD3CF80918002882309F40FC437
:109030001F928F9380EA95E09F938F930E94C6932F
:109040000F900F900F900F9002C40E943735FFC30E
:1090500060917E0270917F0280E090E00E94E69233
:109060008C0163E276E00E940793892BD1F4809112
:10907000660290916702A0916802B0916902977FA1
:109080008093660290936702A0936802B09369028E
:1090900044E050E06EE170E086E692E00E94919636
:1090A000D6C362EA75E0C8010E940793892BD1F408
:1090B0008091660290916702A0916802B091690266
:1090C00098608093660290936702A0936802B093C1
:1090D000690244E050E06EE170E086E692E00E94B2
:1090E0009196B5C30E94530EB2C360917E027091F7
:1090F0007F0280E090E00E94E692FC012081233212
:10910000C1F44AE050E060E070E001960E946D8F8B
:109110007B836A8360917E0270917F0280E090E0A1
:109120000E94E6922A813B81243031050CF096C0E2
:1091300002C01B821A82009709F490C01982BE01F6
:109140006F5F7F4F0E945F2E19013A014B01B82FCC
:10915000A92F8AE02A813B81829FF001839FF00D35
:109160001124E855F34E4080518032813C83838145
:109170008D8394819E8325812F83368138878781D3
:1091800089879101A301B4018B2F9A2F5201CC80C2
:10919000DD80EE80FF80088519850E949F8A09F492
:1091A00060C08981811103C0208231822AC01816D3
:1091B00084F4422853289C81692A2D81722A3E8199
:1091C000832A8F81982A9885B92B2985A22B4082E2
:1091D00017C0209430946094709480949094B095CB
:1091E000A095242053203C8163228D8178229E818A
:1091F00089222F8192223885B3238985A823208252
:1092000051826282738284829582B683A78348E208
:1092100050E062E270E088EA9CE10E94919688E961
:1092200095E09F938F930E94C6938AE02A813B81A9
:10923000829FF001839FF00D1124E855F34E2081A9
:1092400031814281538164817581868197810E9439
:10925000A82A0E94D0110F900F9003C082E00E94B4
:1092600015308CE895E09F938F930E94C6932FEF63
:109270003FEF4FEF5FEF6FEF7FEF8FEF9FEF0E94BA
:10928000A82A0E94D011809180020F900F9088230D
:1092900009F4DDC21F928F9389E895E09F938F9325
:1092A0000E94C6930F900F900F900F90D0C26091C4
:1092B0007E0270917F0280E090E00E94E692FC01C5
:1092C00020812332A1F44AE050E060E070E0019692
:1092D0000E946D8F8B0160917E0270917F0280E011
:1092E00090E00E94E69204301105ECF402C000E028
:1092F00010E00097C1F04AE050E060E070E00E94AA
:1093000098902AE0209FF001219FF00D1124E8554C
:10931000F34E7187608748E250E062E270E088EACD
:109320009CE10E94919681E00E941530809180021C
:10933000882309F48CC21F928F9386E895E09F934F
:109340008F930E94C6930F900F900F900F907FC243
:109350000E942A7280918002882309F478C21F92A9
:109360008F9383E895E09F938F930E94C6930F900D
:109370000F900F900F906BC20E94DA3080918002A4
:10938000882309F464C21F928F9380E895E09F932D
:109390008F930E94C6930F900F900F900F9057C21B
:1093A00080E090E00E949C2780918002882309F44D
:1093B0004EC21F928F938DE795E09F938F930E94EB
:1093C000C6930F900F900F900F9041C28091C52CC3
:1093D00081FF2DC00E942825892B49F58091BC284A
:1093E0008F938091BB288F938091BA288F9380911F
:1093F000B9288F9382E795E09F938F930E94C6933D
:1094000080919D358F9380919C358F9380919B3572
:109410008F9380919A358F9385E695E09F938F93F4
:109420000E94C6930FB6F894DEBF0FBECDBF0E9458
:10943000D0118091C52C9091C62C90FF63C081E023
:1094400090E00E94A0247B011C0180E090E00E943B
:10945000A0244B018C010E94FE233F922F92FF9289
:10946000EF9284E595E09F938F930E94C6931F939C
:109470000F939F928F9284E495E09F938F930E9425
:10948000C693240138019401A80147018101B70165
:10949000C1010E949D229F938F937F936F9389E3D5
:1094A00095E09F938F930E94C693242D352D462DD2
:1094B000572D6E2D792D822D912F0E94FE229F9384
:1094C0008F937F936F938BE295E09F938F930E948E
:1094D000C693242D352D462D572D6E2D792D822D99
:1094E000912F0E945F239F938F937F936F9388E1C7
:1094F00095E09F938F930E94C6930FB6F894DEBFBA
:109500000FBECDBF0E94D01180918002882309F444
:109510009EC11F928F9385E195E09F938F930E9448
:10952000C6930F900F900F900F9091C18091C52C12
:1095300082FF2BC021E048E061E083E00E947A19BD
:109540008091AC1D8F938091AB1D8F938091AA1D4C
:109550008F938091A91D8F938091A81D8F938091E7
:10956000A71D8F938091A61D8F938091A51D8F932A
:109570008EEF94E09F938F930E94C6930E94D01128
:109580000FB6F894DEBF0FBECDBF8091C52C909171
:10959000C62C91FF3BC00E94DF1D20E030E048EC6C
:1095A00052E4162F072FF82EE92E0E94448E20E851
:1095B00036EE45EC57E40E94988B21E03EED42E404
:1095C0005EE30E94B18E9B01AC0160E070E080E838
:1095D0009FE30E94B48A2BE43AE34DEB57E30E94E9
:1095E000988B9F938F937F936F93EF92FF920F933C
:1095F0001F9385EE94E09F938F930E94C6930E94E1
:10960000D0110FB6F894DEBF0FBECDBF809180029F
:10961000882309F41CC11F928F9382EE94E09F93DC
:109620008F930E94C6930F900F900F900F900FC1D1
:1096300060917E0270917F0280E090E00E94E6924D
:1096400068E276E00E940793892B99F460917E028C
:1096500070917F0280E090E00E94E692009709F40A
:10966000F6C00E94D39190915201892B80935201B0
:10967000EEC0809152018F701F928F9386E293E02B
:109680009F938F930E94C6930E94D0110F900F90CA
:109690000F900F90DCC060917E0270917F0280E09D
:1096A00090E00E94E692009711F14AE050E060E0FD
:1096B00070E00E946D8F603198F4609364021F9295
:1096C0006F9385ED94E09F938F930E94C69341E042
:1096D00050E06BE170E084E692E00E94919611C048
:1096E000809164021F928F938CEC94E006C080916D
:1096F00064021F928F9383EC94E09F938F930E9458
:10970000C6930F900F900F900F900E94D0118091F0
:109710008002882309F49BC01F928F9380EC94E011
:109720009F938F930E94C6930F900F900F900F906E
:109730008EC060917E0270917F0280E090E00E9476
:10974000E6928C0169E175E00E940793892BE1F4B0
:109750000E94B3668091660290916702A0916802B0
:10976000B091690290618093660290936702A09322
:109770006802B093690244E050E06EE170E086E672
:1097800092E00E94919663C06CE175E0C8010E946E
:109790000793892B99F5F8940E94C0660FB6F89448
:1097A000A8958091600088618093600010926000AD
:1097B0000FBE84B7877F84BF8091600088618093EB
:1097C0006000109260007894809166029091670228
:1097D000A0916802B09169029F7E80936602909387
:1097E0006702A0936802B093690244E050E06EE122
:1097F00070E086E692E00E94919629C06DE276E0E4
:10980000C8010E94079340916602509167026091DF
:10981000680270916902892B21F454FF18C0F894F2
:10982000FFCF54FD03C08CE195E002C089E195E0D3
:109830009F938F9382E293E09F938F930E94C693AE
:109840000F900F900F900F9002C00E94C625EA85DE
:10985000FB851182108283E02B960FB6F894DEBF51
:109860000FBECDBFDF91CF911F910F91FF90EF9071
:10987000DF90CF90BF90AF909F908F907F906F9030
:109880005F904F903F902F900895CF93DF93EC011E
:1098900088819981009741F0833F914109F48CC000
:1098A0001982188283E093C00E948A3680916602F2
:1098B00080FD05C081FF01C01D9B0E94C067809193
:1098C00070008C7F809370008091B60080628093DE
:1098D000B6001092B20082E08093B1008091B60091
:1098E0008770E1F78091700081608093700061E77C
:1098F0007EE080E090E00E948D660E94E22680E09B
:109900000E94C0288CEE91E19F938F930E94C69392
:109910000E9462168091C52C0F900F9086FD0E94C8
:1099200077618091C52C9091C62C90FD0E94B62342
:109930008091C52C87FF06C021E04CE061E080EDFE
:109940000E941A6280919C130E94AD6A8091650208
:109950000E9486690E9483698093810A80916502D2
:109960000E94866980919C131F928F938091810A37
:109970001F928F9382E396E09F938F930E94B293FE
:109980001092830A1092820A0F900F900F900F90FE
:109990000F900F9086E592E09093983580939735DD
:1099A00083E290E0909398138093971383EF91E173
:1099B0009983888381E00BC06332E1F744EF50E381
:1099C00060E070E082E89AE00E94FA37E3CFDF912E
:1099D000CF9108950F931F93CF93DF93EC018A01EA
:1099E00088819981009711F18830924121F0198284
:1099F000188283E020C06231E9F4A80162E170E0DE
:109A000082E89AE00E94FA3784E080937C351092D5
:109A10007E3510927D351093803500937F354CE76D
:109A200055E362E182E492E00E945D7088E092E199
:109A30009983888381E0DF91CF911F910F910895E1
:109A40008436910514F19F938F9388E896E09F9355
:109A50008F930E94B2938091CF309091D030A0919B
:109A6000D130B091D2300196A11DB11D8093CF307D
:109A70009093D030A093D130B093D2300F900F900C
:109A80000F900F9081E090E0089580E090E00895BD
:109A90002F923F924F925F926F927F928F929F92FE
:109AA000AF92BF92CF92DF92EF92FF920F931F93EC
:109AB000CF93DF93CDB7DEB7CC59D1090FB6F89469
:109AC000DEBF0FBECDBFCB56DF4F99838883C5590C
:109AD000D0408A01633871F486E89AE0C456DF4FBB
:109AE0006883CC59D0400E947B73C456DF4F688195
:109AF000CC59D040CB56DF4FA881B981C559D04051
:109B00002D913C91203AB1E13B0711F40C94155B87
:109B100040F42115310581F0263C3F4009F43BC457
:109B20002FC4223B41E1340709F409C4293B3141E8
:109B300011F40C941D5B24C44AE259E061E870E022
:109B400086E89AE00E94607386EC9FE0EFC35A01BA
:109B5000E3E0F0E0EC0FFD1FE40FF51F1082CA01F7
:109B60000E94204D892B81F720E030E040E050E05A
:109B7000CC56DF4F6881C459D040627070E080E0FD
:109B800090E0A0E00E94A88A09F0A0C6212F2870CA
:109B900030E040E050E060E070E080E090E0A0E085
:109BA0000E94A88A99F127E04AE250E06BE270E057
:109BB00089E290E00E94F85D8EE895E30E94C95F1B
:109BC000BC01990F880B990B0E944C8C20E030E06F
:109BD00048EC52E40E94988B9F938F937F936F93EE
:109BE0008CEB96E09F938F931F9287E78F93CE0124
:109BF0008A0D9B1D03969F938F930E941E94A80E1F
:109C0000B91E0FB6F894DEBF0FBECDBF212F207155
:109C100030E040E050E060E070E080E090E0A0E004
:109C20000E94A88AE9F126E04AE250E06BE270E087
:109C300089E290E00E94F85D81E090E00E94681166
:109C400080939B1381E09DE10E94C95FBC01990F45
:109C5000880B990B0E944C8C20E030E048EC52E4D9
:109C60000E94988B9F938F937F936F9386EC96E0DF
:109C70009F938F931F9287E78F93C501029621E0F0
:109C800030E02C0F3D1F820F931F9F938F930E94F4
:109C90001E94A80EB91E0FB6F894DEBF0FBECDBF3E
:109CA000C257DF4F2881CE58D04030E040E050E02E
:109CB00060E070E080E090E0A0E00E94A88A01F1FE
:109CC0000E9424119F938F937F936F9381ED96E071
:109CD0009F938F931F9287E78F93C5010296A1E010
:109CE000B0E0AC0FBD1F8A0F9B1F9F938F930E9404
:109CF0001E94A80EB91E0FB6F894DEBF0FBECDBFDE
:109D0000212F207430E040E050E060E070E080E01F
:109D100090E0A0E00E94A88A31F18091CA308F9330
:109D20008091C9308F938091C8308F938091C730D4
:109D30008F938FED96E09F938F931F9287E78F937A
:109D4000C501029621E030E02C0F3D1F820F931FCA
:109D50009F938F930E941E94A80EB91E0FB6F8947D
:109D6000DEBF0FBECDBF212F207830E040E050E0B5
:109D700060E070E080E090E0A0E00E94A88A41F1FD
:109D8000F8948091743590917535A0917635B091A5
:109D900077357894BF93AF939F938F938DEE96E032
:109DA0009F938F931F9287E78F93C5010296A1E03F
:109DB000B0E0AC0FBD1F8A0F9B1F9F938F930E9433
:109DC0001E94A80EB91E0FB6F894DEBF0FBECDBF0D
:109DD00020E0302F317040E050E060E070E080E043
:109DE00090E0A0E00E94A88A09F082C520E0302F10
:109DF000327040E050E060E070E080E090E0A0E091
:109E00000E94A88A09F0F2C520E0302F347040E0AB
:109E100050E060E070E080E090E0A0E00E94A88A5E
:109E200009F015C620E0302F387040E050E060E0C7
:109E300070E080E090E0A0E00E94A88A09F036C6B9
:109E400020E0302F307140E050E060E070E080E0D2
:109E500090E0A0E00E94A88A09F0A6C620E0302F7A
:109E6000307240E050E060E070E080E090E0A0E020
:109E70000E94A88A09F0C8C620E030E040E050E027
:109E8000CC56DF4F6881C459D040647070E080E0E8
:109E900090E0A0E00E94A88A09F0E4C620E0C8563D
:109EA000DF4F3881C859D04040E050E060E070E0BA
:109EB00080E090E0A0E00E94A88A09F040C720E07E
:109EC000C756DF4F3881C959D04040E050E060E0CC
:109ED00070E080E090E0A0E00E94A88A09F05DC7F1
:109EE000CE56DF4F5881C259D0405170952E20E098
:109EF00030E0452F50E060E070E080E090E0A0E0CE
:109F00000E94A88A09F077C720E030E0CE56DF4FE4
:109F10004881C259D040427050E060E070E080E07B
:109F200090E0A0E00E94A88A09F098C720E030E005
:109F3000C657DF4F4881CA58D04050E060E070E01B
:109F400080E090E0A0E00E94A88A09F0BAC720E073
:109F500030E040E050E0CC56DF4F6881C459D0403B
:109F6000687070E080E090E0A0E00E94A88A09F0AC
:109F7000D2C720E030E040E050E0CC56DF4F6881AF
:109F8000C459D040607170E080E090E0A0E00E9491
:109F9000A88A09F0ECC720E030E0CE56DF4F4881B8
:109FA000C259D040487050E060E070E080E090E03E
:109FB000A0E00E94A88A11F00C94E35720E030E062
:109FC000CE56DF4F4881C259D040407150E060E02A
:109FD00070E080E090E0A0E00E94A88A11F00C946C
:109FE000165820E030E0CE56DF4F4881C259D040AD
:109FF000407250E060E070E080E090E0A0E00E94FD
:10A00000A88A11F00C94495820E030E0CE56DF4F7A
:10A010004881C259D040407450E060E070E080E078
:10A0200090E0A0E00E94A88A11F00C947C58CE56D3
:10A03000DF4FF881C259D040F0787F2E20E030E029
:10A040004F2F50E060E070E080E090E0A0E00E94E0
:10A05000A88A11F00C94AF58CD56DF4F2881C35910
:10A06000D0402170622E20E030E040E0562D60E0CC
:10A0700070E080E090E0A0E00E94A88A11F40C94C7
:10A08000305B8091C52C82FD02C00C94F75821E012
:10A0900046E061E083E00E947A1920E030E0472D3D
:10A0A00050E060E070E080E090E0A0E00E94A88ACC
:10A0B00011F40C94F7588091C52C82FF02C00C94C7
:10A0C000BC5820E030E040E0CD56DF4F5881C35906
:10A0D000D040527060E070E080E090E0A0E00E942C
:10A0E000A88A11F00C942C5920E030E040E0CD56C5
:10A0F000DF4F5881C359D040547060E070E080E079
:10A1000090E0A0E00E94A88A11F00C945F5920E032
:10A1100030E040E0CD56DF4F5881C359D0405071F8
:10A1200060E070E080E090E0A0E00E94A88A11F07A
:10A130000C94925920E030E040E0CD56DF4F58813A
:10A14000C359D040507260E070E080E090E0A0E041
:10A150000E94A88A11F00C94D15920E030E040E030
:10A16000CD56DF4F5881C359D040507460E070E045
:10A1700080E090E0A0E00E94A88A11F00C94105AB0
:10A1800020E030E040E0CD56DF4F5881C359D04049
:10A19000587060E070E080E090E0A0E00E94A88A43
:10A1A00011F00C944F5A20E030E040E0C656DF4FEB
:10A1B0005881CA59D04060E070E080E090E0A0E0B3
:10A1C0000E94A88A11F00C94805A20E030E0492DBA
:10A1D00050E060E070E080E090E0A0E00E94A88A9B
:10A1E00011F00C94B75A212F302FCE56DF4F4881F3
:10A1F000C259D040CD56DF4F5881C359D040CC56BC
:10A20000DF4F6881C459D0407D2DC956DF4F88810A
:10A21000C759D0409C2DA0E00E94A88A11F00C9450
:10A22000C25A809164028061898380917A0A8A830C
:10A23000FE01EA0DFB1D138280919F139091A013E4
:10A24000A091A113B091A21385010D5F1F4F80FF54
:10A250000CC01F930F938DE898E09F938F930E94FB
:10A26000B2930F900F900F900F90B801CE0101960E
:10A270000E946A758091660282FF0AC024E731E37A
:10A28000A801BE016F5F7F4F8EE692E00E94DD6005
:10A2900080919F139091A013A091A113B091A2134C
:10A2A00082FD73980E948A6886E89AE00E947D7316
:10A2B0008091660290916702A0916802B091690254
:10A2C00090FD02C00C94F95A3FEFA31AB30A0E9402
:10A2D0008369F82E89E10E949B69809166029091C2
:10A2E0006702A0916802B091690290FD02C00C94CF
:10A2F000F55A739880917A0A8F5F80937A0A8A83DD
:10A30000B5016F5F7F4FCE0101960E946A7586E8A6
:10A310009AE00E947D7340E050E065E88091E1148E
:10A320009091E2140E945D7080EA91E1CB56DF4F7C
:10A33000A881B981C559D0408D939C931EC08EE6EB
:10A340009AE00E94EB6E892BC1F00E948A6880918E
:10A35000660287FD2B9840E450E060E070E08EE6F6
:10A360009AE00E94CD6E89EB91E1CB56DF4FE881F8
:10A37000F981C559D0409183808381E00C94405B82
:10A38000CB56DF4FA881B981C559D0401D921C9290
:10A3900083E00C94405B623181F78090660290907C
:10A3A0006702A0906802B090690291FCCDCBF801E1
:10A3B0008081813021F50180F281E02D10810181C1
:10A3C0002281CE56DF4F2883C259D0403381CD56EB
:10A3D000DF4F3883C359D0404481CC56DF4F488388
:10A3E000C459D040D5805681C956DF4F5883C759CC
:10A3F000D040C780E084F184212C312C52C08230BF
:10A40000B9F423803480E12CF12C11E000E0CE5629
:10A41000DF4F1882C259D040B0E8CD56DF4FB88325
:10A42000C359D040CC56DF4F1882C459D04032C0F7
:10A430008330D1F0843009F087CBE12CF12C212C32
:10A44000312C15E000E0CE56DF4F1882C259D040C3
:10A45000CD56DF4F1882C359D040E2E0CC56DF4FD3
:10A46000E883C459D04016C0E12CF12C212C312CAA
:10A4700015E000E0CE56DF4F1882C259D040CD56CD
:10A48000DF4F1882C359D040F1E0CC56DF4FF8833C
:10A49000C459D040D12CC956DF4F1882C759D0407B
:10A4A000C12C4090C7305090C8306090C930709037
:10A4B000CA3020918D0230918E0240918F025091CE
:10A4C0009002C657DF4F288339834A835B83CA587B
:10A4D000D0402DEC3CEC4CE45EE3C657DF4F688186
:10A4E00079818A819B81CA58D0400E94B58A9B019C
:10A4F000AC01C301B2010E94718D87FD0BC0E894CD
:10A50000A0F88092660290926702A0926802B092D0
:10A51000690246C0C657DF4F288139814A815B8175
:10A52000CA58D040C301B2010E94938B87FF38C044
:10A530008091D3309091D430A091D530B091D63065
:10A540000196A11DB11D8093D3309093D430A09378
:10A55000D530B093D630A0FCF7CA6894A0F88092AA
:10A56000660290926702A0926802B092690215E4B6
:10A5700000E2CE56DF4F1882C259D040CD56DF4F91
:10A580001882C359D04034E0CC56DF4F3883C459C9
:10A59000D040D12CC956DF4F1882C759D040C12CAA
:10A5A000CE56DF4F4881C259D0404470C657DF4F66
:10A5B0004883CA58D04020E030E050E060E070E0CE
:10A5C00080E090E0A0E00E94A88A09F08C9A512FC8
:10A5D0005072C257DF4F5883CE58D040252F30E0FD
:10A5E00040E050E060E070E080E090E0A0E00E9499
:10A5F000A88A11F00E942411802F8074C856DF4F62
:10A600008883C859D04020E0382F40E050E060E017
:10A6100070E080E090E0A0E00E94A88A11F00E9423
:10A620002825902F9078C756DF4F9883C959D0407E
:10A6300020E0392F40E050E060E070E080E090E002
:10A64000A0E00E94A88A51F00E94BF10609381355B
:10A65000709382358093833590938435212F2170B8
:10A6600030E040E050E060E070E080E090E0A0E0AA
:10A670000E94A88AF1F08FE89CE19F938F938CE968
:10A6800096E09F938F931F9287E78F93CE01039657
:10A690009F938F930E941E944C010E94204D0FB6F1
:10A6A000F894DEBF0FBECDBF892B09F04DCA54010F
:10A6B00002C0A12CB12C212F227030E040E050E0EC
:10A6C00060E070E080E090E0A0E00E94A88AD1F114
:10A6D000C501029664EA76E0E1E0F0E0EC0FFD1FD0
:10A6E0008E0F9F1F0E941093F3E0AF0EB11C2EE857
:10A6F000622E25E3722E36E7832E33E0932E47E752
:10A70000542ED3018D913D011F928F939F928F9272
:10A710001F925F92C5010296E1E0F0E0EC0FFD1F91
:10A720008E0F9F1F9F938F930E941E94A80EB91E99
:10A730000FB6F894DEBF0FBECDBF36E9631635E322
:10A740007306F9F6212F247030E040E050E060E01D
:10A7500070E080E090E0A0E00E94A88A09F450C078
:10A76000C501029668EA76E041E050E04C0F5D1FBB
:10A77000840F951F0E94109354E0A50EB11C2E016A
:10A780008AE7480E511C80E1D2011D928A95E9F7B3
:10A7900028E0A20168E980EB0E94C5173201B8E009
:10A7A0006B0E711C96E7892E93E0992E27E7F20134
:10A7B00081912F011F928F939F928F921F922F93BF
:10A7C000C501029641E050E04C0F5D1F840F951FBC
:10A7D0009F938F93C556DF4F2883CB59D0400E945B
:10A7E0001E94A80EB91E0FB6F894DEBF0FBECDBFE3
:10A7F000C556DF4F2881CB59D04046145704B9F6CF
:10A80000CD56DF4F9881C359D0409078C656DF4F60
:10A810009883CA59D04020E030E040E0592F60E0F2
:10A8200070E080E090E0A0E00E94A88AE1F48091CE
:10A830009D1390919E139F938F938DEA96E09F9323
:10A840008F931F9287E78F93CE018A0D9B1D0396EE
:10A850009F938F930E941E94A80EB91E0FB6F89472
:10A86000DEBF0FBECDBF20E030E040E050E0CC5670
:10A87000DF4F6881C459D040617070E080E090E0A3
:10A88000A0E00E94A88A09F46FC9E3E0F0E0EC0FB1
:10A89000FD1FEA0DFB1D80E28083A50183E090E0AF
:10A8A0008A199B09FC01E40FF51FEC50FF4C208135
:10A8B0004F5F5F4F222309F44AC92081E1E0F0E0B5
:10A8C000EC0FFD1FE40FF51F2283ECCFCE018A0DA4
:10A8D0009B1D64EB76E003960E941093B7E0AB0EED
:10A8E000B11CC5010E94204D892B09F02DC94EC90C
:10A8F000E114F10409F47ACAF89440907435509048
:10A900007535609076357090773578948091F91C24
:10A910009091FA1CA091FB1CB091FC1CA301920128
:10A92000281B390B4A0B5B0BCA01B9010E944A8CE8
:10A93000C257DF4F688379838A839B83CE58D04088
:10A94000B70180E090E00E944A8C9B01AC01C257A5
:10A95000DF4F688179818A819B81CE58D0400E94E7
:10A96000988B4C019F928F937F936F9388EF96E023
:10A970009F938F931F9287E78F939E012A0D3B1D14
:10A980002D5F3F4F3F932F93C456DF4F6883CC59C1
:10A99000D040C556DF4F7883CB59D0400E941E94DB
:10A9A000A80EB91EC456DF4F6881CC59D040C55699
:10A9B000DF4F7881CB59D040862F972FA82DB92D06
:10A9C0008093863590938735A0938835B0938935E9
:10A9D0004092F91C5092FA1C6092FB1C7092FC1C75
:10A9E0000FB6F894DEBF0FBECDBF00CAE114F1046C
:10A9F00009F40ACAF8948091D01C9091D11CA091BE
:10AA0000D21CB091D31C78949F938F9380916D0248
:10AA10008F9380916C028F9385E097E09F938F9343
:10AA20001F9287E78F93C5010296A1E0B0E0AC0FBB
:10AA3000BD1F8A0F9B1F9F938F930E941E94A80E89
:10AA4000B91E0FB6F894DEBF0FBECDBFDDC9F894B6
:10AA50008091783590917935A0917A35B0917B3598
:10AA60007894BF93AF939F938F9385E197E09F93E3
:10AA70008F931F9287E78F93C501029621E030E004
:10AA80002C0F3D1F820F931F9F938F930E941E9444
:10AA9000A80EB91EC5010E94204D0FB6F894DEBF66
:10AAA0000FBECDBF892B09F04FC8BCC9E114F1041A
:10AAB00009F4C6C9F8944090783550907935609083
:10AAC0007A3570907B3578948091FD1C9091FE1CB6
:10AAD000A091FF1CB091001DA3019201281B390B0E
:10AAE0004A0B5B0BCA01B9010E944A8CC257DF4F67
:10AAF000688379838A839B83CE58D040B70180E0F6
:10AB000090E00E944A8C9B01AC01C257DF4F6881E4
:10AB100079818A819B81CE58D0400E94988B4C01CC
:10AB20009F928F937F936F9380E297E09F938F9391
:10AB30001F9287E78F939E012A0D3B1D2D5F3F4F8C
:10AB40003F932F93C456DF4F6883CC59D040C556EE
:10AB5000DF4F7883CB59D0400E941E94A80EB91EB7
:10AB6000C456DF4F6881CC59D040C556DF4F78813D
:10AB7000CB59D040862F972FA82DB92D80938A3599
:10AB800090938B35A0938C35B0938D354092FD1CFE
:10AB90005092FE1C6092FF1C7092001D0FB6F8943C
:10ABA000DEBF0FBECDBF4CC9EF2809F457C9F894DA
:10ABB0008091D41C9091D51CA091D61CB091D71C2B
:10ABC00078949F938F9380916B028F9380916A0208
:10ABD0008F938DE297E09F938F931F9287E78F93D8
:10ABE000C5010296A1E0B0E0AC0FBD1F8A0F9B1F0C
:10ABF0009F938F930E941E94A80EB91E0FB6F894CF
:10AC0000DEBF0FBECDBF2AC98091CB309091CC3032
:10AC1000A091CD30B091CE30BF93AF939F938F93DF
:10AC20008DE397E09F938F931F9287E78F93C501E2
:10AC3000029621E030E02C0F3D1F820F931F9F935F
:10AC40008F930E941E94A80EB91EC5010E94204D2C
:10AC50000FB6F894DEBF0FBECDBF892B11F00C9458
:10AC6000A44D0AC98091D6308F938091D5308F93AF
:10AC70008091D4308F938091D3308F938091D23054
:10AC80008F938091D1308F938091D0308F9380912A
:10AC9000CF308F9388E497E09F938F931F9287E73D
:10ACA000982E9F92C5010296A1E0B0E0AC0FBD1FA7
:10ACB0008A0F9B1F9F938F930E941E94A80EB91E0C
:10ACC000C5010E94204D0FB6F894DEBF0FBECDBF68
:10ACD000892B11F00C94A44D8091C52C9091C62C19
:10ACE00090FFDCC88091DA308F938091D9308F93B8
:10ACF0008091D8308F938091D7308F938CE697E0F6
:10AD00009F938F931F929F92C501029621E030E09E
:10AD10002C0F3D1F820F931F9F938F930E941E94B1
:10AD2000A80EB91EC5010E94204D0FB6F894DEBFD3
:10AD30000FBECDBF892B11F00C94A44DAFC88091EC
:10AD4000BC288F938091BB288F938091BA288F93D2
:10AD50008091B9288F938EE797E09F938F931F92EE
:10AD600087E78F93C5010296A1E0B0E0AC0FBD1F4D
:10AD70008A0F9B1F9F938F930E941E94A80EB91E4B
:10AD8000C5010E94204D0FB6F894DEBF0FBECDBFA7
:10AD9000892B11F00C94A44D92C8809184358F9327
:10ADA000809183358F93809182358F938091813507
:10ADB0008F9389E897E09F938F931F9287E78F93F4
:10ADC000C501029621E030E02C0F3D1F820F931F3A
:10ADD0009F938F930E941E94A80EB91EC5010E94D6
:10ADE000204D0FB6F894DEBF0FBECDBF892B11F0FA
:10ADF0000C94A44D75C881E00E94711020918502C9
:10AE00003091860240918702509188020E94448EC0
:10AE10009F938F937F936F9386E997E09F938F9390
:10AE20001F9287E78F93C5010296A1E0B0E0AC0FB7
:10AE3000BD1F8A0F9B1F9F938F930E941E94A80E85
:10AE4000B91EC5010E94204D0FB6F894DEBF0FBE9B
:10AE5000CDBF892B11F00C94A44D56C882E00E94FE
:10AE600071102091810230918202409183025091B1
:10AE700084020E94448E9F938F937F936F9383EA03
:10AE800097E09F938F931F9287E78F93C501029658
:10AE900021E030E02C0F3D1F820F931F9F938F9373
:10AEA0000E941E94A80EB91EC5010E94204D0FB627
:10AEB000F894DEBF0FBECDBF892B11F00C94A44DCA
:10AEC00035C883E00E9471109F938F937F936F9397
:10AED00080EB97E09F938F931F9287E78F93C50135
:10AEE0000296A1E0B0E0AC0FBD1F8A0F9B1F9F939D
:10AEF0008F930E941E94A80EB91E8C98C5010E94C3
:10AF0000204D0FB6F894DEBF0FBECDBF892B11F0D8
:10AF10000C94A44D1CC8299903C08CE195E002C093
:10AF200089E195E09F938F938DEB97E09F938F93AB
:10AF30001F9287E78F93C501029621E030E02C0F26
:10AF40003D1F820F931F9F938F930E941E94A80E04
:10AF5000B91EC5010E94204D0FB6F894DEBF0FBE8A
:10AF6000CDBF892B11F00C94A44D0C94B94F2A99A4
:10AF700003C08CE195E002C089E195E09F938F9337
:10AF800085EC97E09F938F931F9287E78F93C5017E
:10AF90000296A1E0B0E0AC0FBD1F8A0F9B1F9F93EC
:10AFA0008F930E941E94A80EB91EC5010E94204DC9
:10AFB0000FB6F894DEBF0FBECDBF892B11F00C94F5
:10AFC000A44D0C94CB4F8091C52C87FD02C00C94EE
:10AFD000DE4F21E042E161E080ED0E941A629F9322
:10AFE0008F937F936F938DEC97E09F938F931F9236
:10AFF00087E78F93C501029621E030E02C0F3D1FBB
:10B00000820F931F9F938F930E941E94A80EB91EC8
:10B01000C5010E94204D0FB6F894DEBF0FBECDBF14
:10B02000892B11F00C94A44D0C94DE4F8091C52C0B
:10B0300087FD02C00C94F14F21E042E162E080ED17
:10B040000E941A629F938F937F936F938BED97E08B
:10B050009F938F931F9287E78F93C5010296A1E07C
:10B06000B0E0AC0FBD1F8A0F9B1F9F938F930E9470
:10B070001E94A80EB91EC5010E94204D0FB6F8946B
:10B08000DEBF0FBECDBF892B11F00C94A44D0C94E4
:10B09000F14F8091C52C87FD02C00C94045021E033
:10B0A00042E163E080ED0E941A629F938F937F9349
:10B0B0006F9389EE97E09F938F931F9287E78F930B
:10B0C000C501029621E030E02C0F3D1F820F931F37
:10B0D0009F938F930E941E94A80EB91EC5010E94D3
:10B0E000204D0FB6F894DEBF0FBECDBF892B11F0F7
:10B0F0000C94A44D0C9404508091C52C87FD02C083
:10B100000C94175021E042E164E080ED0E941A6245
:10B110009F938F937F936F9387EF97E09F938F9386
:10B120001F9287E78F93C5010296A1E0B0E0AC0FB4
:10B13000BD1F8A0F9B1F9F938F930E941E94A80E82
:10B14000B91EC5010E94204D0FB6F894DEBF0FBE98
:10B15000CDBF892B11F00C94A44D0C941750809105
:10B16000C52C82FD02C00C942C5046E061E083E0C7
:10B170000E947A190C942C508091A81D8F93809175
:10B18000A71D8F938091A61D8F938091A51D8F93EE
:10B1900085E098E09F938F931F9287E78F93C50177
:10B1A000029641E050E04C0F5D1F840F951F9F9366
:10B1B0008F930E941E94A80EB91EC5010E94204DB7
:10B1C0000FB6F894DEBF0FBECDBF892B11F00C94E3
:10B1D000A44D20E030E040E0562D60E070E080E0DB
:10B1E00090E0A0E00E94A88A11F40C946150809134
:10B1F000C52C82FD02C00C9461508091AC1D8F93D0
:10B200008091AB1D8F938091AA1D8F938091A91D72
:10B210008F938DE098E09F938F931F9287E78F9392
:10B22000C5010296E1E0F0E0EC0FFD1F8E0F9F1FBD
:10B230009F938F930E941E94A80EB91EC5010E9471
:10B24000204D0FB6F894DEBF0FBECDBF892B11F095
:10B250000C94A44D0C9461508091C52C9091C62CF7
:10B2600090FD02C00C94745080E090E00E94A024F5
:10B270009F938F937F936F9388E198E09F938F9331
:10B280001F9287E78F93C501029641E050E04C0F73
:10B290005D1F840F951F9F938F930E941E94A80E8D
:10B2A000B91EC5010E94204D0FB6F894DEBF0FBE37
:10B2B000CDBF892B11F00C94A44D0C947450809147
:10B2C000C52C9091C62C90FD02C00C94875081E053
:10B2D00090E00E94A0249F938F937F936F9388E2C6
:10B2E00098E09F938F931F9287E78F93C5010296F3
:10B2F000E1E0F0E0EC0FFD1F8E0F9F1F9F938F93F7
:10B300000E941E94A80EB91EC5010E94204D0FB6C2
:10B31000F894DEBF0FBECDBF892B11F00C94A44D65
:10B320000C9487508091C52C9091C62C90FD02C042
:10B330000C949A5081E090E00E94A0242B013C01E3
:10B3400080E090E00E94A0249B01AC01C301B20107
:10B350000E949D229F938F937F936F9389E398E040
:10B360009F938F931F9287E78F93C501029641E0C9
:10B3700050E04C0F5D1F840F951F9F938F930E9489
:10B380001E94A80EB91EC5010E94204D0FB6F89458
:10B39000DEBF0FBECDBF892B11F00C94A44D0C94D1
:10B3A0009A508091C52C9091C62C90FD02C00C94AF
:10B3B000AD5081E090E00E94A0242B013C0180E090
:10B3C00090E00E94A0249B01AC01C301B2010E9445
:10B3D000FE229F938F937F936F9384E498E09F93D3
:10B3E0008F931F9287E78F93C5010296E1E0F0E00B
:10B3F000EC0FFD1F8E0F9F1F9F938F930E941E9433
:10B40000A80EB91EC5010E94204D0FB6F894DEBFEC
:10B410000FBECDBF892B11F00C94A44D0C94AD50F0
:10B420008091C52C9091C62C90FD02C00C94C05008
:10B4300081E090E00E94A0242B013C0180E090E09C
:10B440000E94A0249B01AC01C301B2010E945F23B2
:10B450009F938F937F936F9382E598E09F938F9351
:10B460001F9287E78F93C501029641E050E04C0F91
:10B470005D1F840F951F9F938F930E941E94A80EAB
:10B48000B91EC5010E94204D0FB6F894DEBF0FBE55
:10B49000CDBF892B11F00C94A44D0C94C050809119
:10B4A000C52C9091C62C91FD02C00C94D3500E94E3
:10B4B000DF1D9F938F937F936F9385E698E09F9313
:10B4C0008F931F9287E78F93C5010296E1E0F0E02A
:10B4D000EC0FFD1F8E0F9F1F9F938F930E941E9452
:10B4E000A80EB91EC5010E94204D0FB6F894DEBF0C
:10B4F0000FBECDBF892B11F00C94A44D0C94D350EA
:10B50000D10116968C9116971F928F9315968C9158
:10B5100015971F928F9313968C9113971F928F9369
:10B5200012968C911F928F9386E798E09F938F934A
:10B530001F9287E78F93C5010296E1E0F0E0EC0FE0
:10B54000FD1F8E0F9F1F9F938F930E941E94A80E26
:10B55000B91EC5010E94204D0FB6F894DEBF0FBE84
:10B56000CDBF892B11F00C94A44D0C94E550779A23
:10B5700080919F139091A013A091A113B091A21359
:10B5800092FD749A80919F139091A013A091A113A2
:10B59000B091A21382FD0CC08091660280FD08C0AC
:10B5A00081FD02C00C9411511D9902C00C941151DF
:10B5B00040E050E060E070E0CE0101960E94DC0EB9
:10B5C0008091AE1D90E020919513309196138217D3
:10B5D000930710F40C94115140E050E062E180E1D7
:10B5E00092E00E945D700C9411518F2D0E949B6916
:10B5F000739A80919D1390919E13892B11F00E9454
:10B60000C06780917A0A8F5F80937A0A80919F1336
:10B610009091A013A091A113B091A21382FD02C03A
:10B620000C94A44D739A0C94A44D653811F00C94AD
:10B63000BD51A12CB12C0C946D518EE69AE00E9464
:10B64000EB6E892B11F40C94BD510E94C067809160
:10B65000660287FD02C00C94A44D2B9A0C94A44D55
:10B6600020E030E0472D50E060E070E080E090E0C6
:10B67000A0E00E94A88A11F00C945B500C946150D9
:10B68000C456DF4F0FB6F894DEBF0FBECDBFDF91BB
:10B69000CF911F910F91FF90EF90DF90CF90BF90CF
:10B6A000AF909F908F907F906F905F904F903F9062
:10B6B0002F9008950C9413734F925F926F927F9224
:10B6C0009F92AF92BF92CF92DF92EF92FF920F9331
:10B6D0001F93CF93DF93CDB7DEB760970FB6F89483
:10B6E000DEBF0FBECDBF5B010E948369E82FF0E093
:10B6F000EE0FFF1FEE53F34E8081918101969183EF
:10B70000808380919F139091A013A091A113B09179
:10B71000A21381FD74984090660250906702609079
:10B720006802709069020E94C6746C01FC018081FD
:10B73000982F92959F70913099F48F7051F4809169
:10B74000A61C9091A71C01969093A71C8093A61C01
:10B750003CC1B50183EA97E30E947F74892B51F0C5
:10B760008091A41C9091A51C01969093A51C809398
:10B77000A41C2BC1D301C2013EE0B695A7959795B5
:10B7800087953A95D1F7F82FF1709F2E81E99AE0CD
:10B790000E9436717C01892B09F44BC0B501C701A9
:10B7A00002960E947F74892B09F43FC087012BE821
:10B7B0003EE040E054E660E070E0C7010F960E9472
:10B7C0006B6DF6019181F7018481981321C0828508
:10B7D0008F5F82878091A21C9091A31C0196909309
:10B7E000A31C8093A21C84E00E94B675F7012085FB
:10B7F00030E02817390708F078C184E00E94B67558
:10B80000F7018087F60180818F70F7018187DDC0A5
:10B81000F701128684E00E94B675F7018087F60171
:10B8200080818F70F701818761C1C7010E949B7180
:10B83000B1CF88E092E00E94C2717C01892B09F4AB
:10B84000C4C0B501C70102960E947874F6018181D7
:10B850008150F701848380E091E0A0E0B0E083872D
:10B860009487A587B687128684E00E94B675F70193
:10B870008087F60180818F70F7018187B70181E9A8
:10B880009AE00E94757187012BE83EE040E054E6A3
:10B8900060E070E0C7010F960E946B6D11E0F60149
:10B8A0008181F7018483F60180818F70F70187839E
:10B8B00084E00E94B675F701858383E00E94B67527
:10B8C000F701868387818F3009F010E0F60141800F
:10B8D000F7018481481A512C612C712C86E0440CAC
:10B8E000551C661C771C8A95D1F7238534854585C0
:10B8F0005685A0ECB0E00E94DC88BB27A92F982FCA
:10B90000872F480E591E6A1E7B1E43865486658605
:10B910007686A501B701C6010E94DC0E8091AE1D9E
:10B9200090E020919513309196138217930738F089
:10B9300040E050E062E180E192E00E945D70809121
:10B94000951390919613029708F44BC08091C52CE3
:10B9500086FF2AC00E946961C60105960E94356172
:10B96000F60181811F928F93F70186811F928F9339
:10B9700085811F928F938EE998E09F938F931F92FA
:10B9800080E18F93CE0101965C019F938F930E947B
:10B990001E9482E00E944F61C5010E9435610FB67E
:10B9A000F894DEBF0FBECDBF809166029091670212
:10B9B000A0916802B091690297FD4DC080919513E6
:10B9C00090919613029708F47AC080919F139091FA
:10B9D000A013A091A113B091A21381FF89C0749A02
:10B9E00087C08091660290916702A0916802B09131
:10B9F000690296FFABCF992009F4A8CFF6018081A8
:10BA0000982F9F709230E8F09150807F892B80832F
:10BA100086E89AE00E945A5B8091A01C9091A11C3C
:10BA200001969093A11C8093A01C80919F139091EC
:10BA3000A013A091A113B091A21396FF87CF739882
:10BA400085CF8091A61C9091A71C01969093A71C6E
:10BA50008093A61C7BCF8FE89CE120918F1C222332
:10BA600009F4ACCF9F938F9381EB98E09F938F93D2
:10BA7000CE0101963C019F938F930E945B945C01E1
:10BA8000B301C60102960E9431930F900F900F9060
:10BA90000F900F900F90009709F490CFEFEFAE1A30
:10BAA000BE0A8A0D9B1DAC010196FA01208120324D
:10BAB000D1F362E18AE192E00E945D707FCF1123B1
:10BAC00009F483CF82E08093E0301092E23010924C
:10BAD000E130F092E430E092E33040EE50E362E196
:10BAE00082E492E00E945D7070CF912C10E0D7CE7E
:10BAF00060960FB6F894DEBF0FBECDBFDF91CF9139
:10BB00001F910F91FF90EF90DF90CF90BF90AF907B
:10BB10009F907F906F905F904F9008958115910551
:10BB200011F00197F1F70895E091A135F091A23558
:10BB300090818091A03589230895E0919E35F09100
:10BB40009F3590818091A035892B8083E091A3352A
:10BB5000F091A43590818091A035892B8083089540
:10BB60001F93CF93DF93E0919E35F0919F359081A5
:10BB70008091A035809589238083E091A335F09151
:10BB8000A43590818091A035892B80838FE897E040
:10BB90000E948E5D1FB7F894E091A335F091A43513
:10BBA00090818091A03580958923808389E091E000
:10BBB0000E948E5DE091A135F091A235D081C091B7
:10BBC000A0351FBF789485E896E00E948E5DE091D5
:10BBD000A135F091A23580819091A035982319F07C
:10BBE0008D2F8C2301C081E0DF91CF911F910895AB
:10BBF0005093A4354093A33570939F3560939E3541
:10BC00009093A2358093A13581E001C0880F2A95D9
:10BC1000EAF78093A0350C94B05DCF93DF93C82FE3
:10BC2000DFB7F894E091A335F091A435908180912D
:10BC3000A035892B808387E090E00E948E5DCC2325
:10BC400051F0E091A335F091A43590818091A03519
:10BC500080958923808384E390E00E948E5DE0914B
:10BC6000A135F091A23590818091A035892309F406
:10BC7000C0E085EB90E00E948E5DE091A335F091ED
:10BC8000A43590818091A035809589238083DFBF82
:10BC900088E790E00E948E5D8C2FDF91CF91089510
:10BCA000CF93DF93C82FD8E08C2F81700E940D5E58
:10BCB000C6958111C068D150B9F78C2FDF91CF9113
:10BCC00008958FEF0C94505EDF92EF92FF920F93E6
:10BCD0001F93CF93DF93E82E8B010E94B05D8111FB
:10BCE00035C080EF0E94505ED0E0C0E488EFD82ECF
:10BCF000DC0E81E00E940D5EF82E81E00E940D5E58
:10BD0000882319F0FF2071F023C0F1100BC0CE156D
:10BD100030F0F801808180FF05C0EC1619F0DC2FAF
:10BD2000FF24F3948F2D0E940D5EF801908196956B
:10BD3000FF2011F09068F8019083C150CD11D9CF48
:10BD40000F5F1F4FC111D2CF8D2F03C08FEF01C0E6
:10BD50008EEFDF91CF911F910F91FF90EF90DF90C9
:10BD60000895EF92FF921F93CF93DF93182FEB016B
:10BD70000E94B05D209771F085E50E94505E7E01C3
:10BD800088E0E80EF11C89910E94505ECE15DF0517
:10BD9000D1F703C08CEC0E94505E812FDF91CF91D0
:10BDA0001F91FF90EF900C94505E0F931F93CF93D1
:10BDB000DF93DB01EC9111969C911197F0E0F92B48
:10BDC000803179F4EE7F63E0EE0FFF1F6A95E1F7B3
:10BDD00016969C9116976CE070E0691B7109E60F4E
:10BDE000F71FF7FF07C091E0EA019883F195E1950D
:10BDF000F10902C0EA011882883279F414968C9114
:10BE0000982F9076903649F086FF02C0EE7F05C0ED
:10BE100085FF02C0EC7F01C0E87FCF0144E096952A
:10BE200087954A95E1F7D9018C93EF70E801E88393
:10BE300080E0DF91CF911F910F9108950F931F9391
:10BE4000CF93DF93EC018B01B80188810E94645E7F
:10BE500088839FEF980F9D3F30F4F80190819832CE
:10BE600011F0903189F7DF91CF911F910F910895D3
:10BE7000CF93DF93EC010E94B05DBE0184EB0E9482
:10BE8000B15E81E00E940D5EC82F0E94B05D81E02E
:10BE9000C11101C080E0DF91CF9108951F93CF932E
:10BEA000DF931F921F92CDB7DEB7182F69837A8375
:10BEB0000E94B05D0E94945D69817A81882341F07F
:10BEC00084E40E94B15E113029F00E949D5D02C0A1
:10BED00082E001C080E00F900F90DF91CF911F9121
:10BEE00008955F926F927F928F929F92AF92BF92CE
:10BEF000CF92DF92EF92FF920F931F93CF93DF9336
:10BF0000CDB7DEB729970FB6F894DEBF0FBECDBF11
:10BF10005C014B013A0189010E94B05DB5018EEBD5
:10BF20000E94B15ECE0101967C016C0199E0592E10
:10BF30005E0C0E94615EF60181936F015E12F9CF83
:10BF400069E070E0C7010E945579D82E811108C0C0
:10BF50009301A401B701F50180810E94D55E02C062
:10BF600083E0D82E8D2D29960FB6F894DEBF0FBE34
:10BF7000CDBFDF91CF911F910F91FF90EF90DF9098
:10BF8000CF90BF90AF909F908F907F906F905F9079
:10BF900008950F931F93CF93DF93CDB7DEB72B9701
:10BFA0000FB6F894DEBF0FBECDBF182F092F682F34
:10BFB000792F88E0810F0E944E5F882319F084E377
:10BFC00091E243C06CE872E88EE190E00E9430603C
:10BFD0009E01275F3F4FAE01465F5F4FBE01655F29
:10BFE0007F4F812F902F0E94715F8111E8CF88E0F1
:10BFF000E1EEF2E0DE01119601900D928A95E1F7F3
:10C00000298541E752E0249FC001259F900D11240E
:10C0100064E670E00E9461888A8594E6899F600DDD
:10C02000711D1124FE01319688E08E0F9191291324
:10C0300003C06F5F7F4F02C08E13F8CF8B858823BC
:10C0400019F0719561957109CB012B960FB6F89493
:10C05000DEBF0FBECDBFDF91CF911F910F9108952D
:10C06000DC01CB0181159105A105B10529F08150B5
:10C070009040A040B040D9F708959B01AC011092C8
:10C08000B90060E074E284EF90E00E947588DA0104
:10C09000C9014097A109B109B695A79597958795CC
:10C0A0008093B800089594EA9093BC0040EA56E863
:10C0B00061E070E09091BC0097FD07C041505109CC
:10C0C00061097109B9F781E008959091B900987FED
:10C0D000983011F09031B9F78093BB0084E88093D9
:10C0E000BC0080EA96E8A1E0B0E02091BC0027FD0A
:10C0F00005C00197A109B109C1F7E5CF8091B90049
:10C10000887F883111F08034F1F680E0089524EAC8
:10C1100034E844E92093BC009091BC0097FFFCCF29
:10C120009091B900987F983011F0903199F78093F1
:10C13000BB003093BC009091BC0097FFFCCF909166
:10C14000B900987F903211F0983539F44093BC00D3
:10C150009091BC0094FDFCCFDDCF08950C9453600A
:10C1600084E98093BC008091BC0084FDFCCF0895DD
:10C170008093BB0084E88093BC008091BC0087FF63
:10C18000FCCF9091B900987F81E0983209F480E06B
:10C19000089584EC8093BC008091BC0087FFFCCFA5
:10C1A0008091BB00089584E88093BC008091BC001E
:10C1B00087FFFCCF8091BB000895CF93DF93FC01F4
:10C1C0007096EC01A991CE01A0933F01CE17DF0735
:10C1D000C1F780913C018F7D80933C0180913C01AF
:10C1E000877F80933C01DB015096FB018191809316
:10C1F0003E01EA17FB07D1F780913C0180688093EC
:10C200003C0180913D0180FFFCCF4051510980915C
:10C210003C01806280933C0180913C01877F809348
:10C220003C01141615069CF4FB01819180933E019C
:10C23000EA17FB07D1F780913C01806880933C01AD
:10C2400080913D0180FFFCCF40515109EACFF901B7
:10C25000C901409620913E012193E817F907D1F7D3
:10C2600081E090E0DF91CF9108950F931F93CF93DA
:10C27000DF93EC018CE70E9487608CE70E94B86036
:10C280008E01005F1F4F89910E94B860C017D107CF
:10C29000D1F7DF91CF911F910F910C94B060813055
:10C2A00019F440E050E002C040EC50E060E070E083
:10C2B0008CE790E00C94AD17813019F44EE050E01B
:10C2C00002C048E050E060E070E08CE790E00C9441
:10C2D000AD1741E050E060E070E08CE790E00E9434
:10C2E000AD1764ED74E180E090E00C94306048E3B9
:10C2F00050E060E070E08CE790E00E94AD1749E309
:10C3000050E060E070E08CE790E00E94AD1744E1FF
:10C3100050E060E070E08CE790E00E94AD1748E7E5
:10C3200050E060E070E08CE790E00E94AD174EE5D1
:10C3300050E060E070E08CE790E00E94AD174DE6C1
:10C3400050E060E070E08CE790E00E94AD1768E399
:10C3500074E38CE090E00E9430604CE050E060E0DC
:10C3600070E08CE790E00E94AD1741E050E060E0A3
:10C3700070E08CE790E00E94AD1746E050E060E08E
:10C3800070E08CE790E00E94AD1764ED74E180E00E
:10C3900090E00C943060CF93DF93CDB7DEB7A297D7
:10C3A0000FB6F894DEBF0FBECDBF81E1E0E4F9E047
:10C3B000DE01529601900D928A95E1F781E1E1E567
:10C3C000F9E0DE01119601900D928A95E1F70E9445
:10C3D0007761CE0142960E94356182E00E944F61F2
:10C3E00064ED74E180E090E00E943060CE0101963F
:10C3F0000E94356160E27CE581E590E00E9430605A
:10C4000080E00E945C6160E27CE581E590E00E9452
:10C4100030604EE050E060E070E08CE790E00E9419
:10C42000AD17A2960FB6F894DEBF0FBECDBFDF9159
:10C43000CF910895CF92DF92EF92FF920F931F93C7
:10C44000CF93DF9300D0CDB7DEB7042F122F21306A
:10C4500061F0223031F0243031F0283031F493E0B3
:10C4600005C091E003C092E001C090E0E82FF0E049
:10C470008160F82E0C3009F4E0C00E3011F49460A5
:10C48000DCC0003111F49860D8C0023109F0D5C089
:10C49000613009F4B7C09C60623011F4906207C04B
:10C4A000633011F4906403C0643009F490669068BE
:10C4B000692F70E023E030E0AE014F5F5F4FCF01A6
:10C4C0000E94C51762E174E380E090E00E94306052
:10C4D0008F2D0E9453600E94C96089830E94C960A9
:10C4E0008A83023119F40E94C9608B830E94C9605B
:10C4F00087FDF1CF0E94D3600E94B06062E174E3D7
:10C5000080E090E00E9430608F2D0E9453600E9476
:10C51000C96089830E94C9608A83023119F40E942C
:10C52000D3608B830E94D3600E94B06069812A81AE
:10C53000023139F5862F90E0A0E0B0E04B81DC01BC
:10C540009927882730E0322F2227820F931FA11DC1
:10C55000B11D61FF09C0840F911DA11DB11DBC015A
:10C56000CD018C6F9F6F06C0BC01CD01640F711DA2
:10C57000811D911D0E944C8C20E83FEF4FEF57E446
:10C580001FC070E0762F6627620F711D072E000C0A
:10C59000880B990B0E944C8C0C3029F420E030EE73
:10C5A0004FEF54E40DC00E3029F420E038EF4FEF88
:10C5B00055E406C0003131F420E03EEF4FEF56E481
:10C5C0000E94988B2FE632E143E050E40E94448EB3
:10C5D0006B017C01612F70E080E090E00E944C8C48
:10C5E0009B01AC01C701B6010E94988B0F900F9080
:10C5F0000F90DF91CF911F910F91FF90EF90DF90FF
:10C60000CF9008959C68692F70E023E030E0AE0180
:10C610004F5F5F4FCF010E94C51762E174E380E076
:10C6200090E00E9430608F2D0E9453600E94C9608C
:10C6300089830E94C9608A8356CF613009F02CCF6C
:10C640009068692F70E023E030E0AE014F5F5F4FEC
:10C65000CF010E94C51762E174E380E090E00E9480
:10C6600030608F2D0E9453600E94C96089830E94B0
:10C67000C9608A833BCFCF93E6E4F1E020819081CB
:10C680008081C081C295C695C695C370207CC20FBB
:10C69000969596959073C90F82958C70C80F1F92CE
:10C6A000CF9389E093E19F938F930E94C6930F905D
:10C6B0000F900F900F908C2FCF9108951F93CF93D1
:10C6C000DF9346E069E180E00E94466680E00E94D8
:10C6D0009B660E94296504B600FE08C088EF92E1BF
:10C6E0009F938F930E94C6930F900F9004B601FE04
:10C6F00008C087EE92E19F938F930E94C6930F909C
:10C700000F9004B602FE08C086ED92E19F938F93CE
:10C710000E94C6930F900F9004B603FE08C085ECEC
:10C7200092E19F938F930E94C6930F900F9004B64F
:10C7300004FE08C088EB92E19F938F930E94C693FA
:10C740000F900F9082E699E09F938F938DE992E18D
:10C750009F938F930E94C6930E94B8700E94E96FC6
:10C7600060E070E085EB92E00E948B700E945F6D4C
:10C77000E091A609F091A70919950E943B6390E00A
:10C780000E94CC660E94907482E08093A3378093CD
:10C79000A4370E94216543EA57E3BC018DEC9BEA74
:10C7A0000E94A0690E9491640E9486690E9425658A
:10C7B0000E94AD6A0E94CF75E0911C0AF0911D0A9B
:10C7C0001995E091F409F091F5091995E091E609C0
:10C7D000F091E70919950E94AF6A182FC091280AB5
:10C7E000D091290AFE0119950F900F900F900F908C
:10C7F000892B49F0FE011995BC0180E890E00E9468
:10C800004D88EB0102C0C0E8D0E00E9483691F920E
:10C810001F93DF93CF931F928F9380911B0A8F9367
:10C8200080911A0A8F938091F3098F938091F20976
:10C830008F938BE692E19F938F930E94C6938EE530
:10C8400092E19F938F930E94C6938DE492E19F9310
:10C850008F930E94C69360E070E087ED92E00E94A3
:10C860008B708EE299E00E94EA6C85E492E19F93DE
:10C870008F930E94C6938DB79EB742960FB6F894D9
:10C880009EBF0FBE8DBFDF91CF911F91089580E8AD
:10C8900080936100109261000E945E63C3E3D2E165
:10C8A00002E212E181E1E82E82E1F82E90E0C92E49
:10C8B00092E1D92E22EFA22E21E1B22E04B600FE83
:10C8C00006C0DF93CF930E94C6930F900F9004B6DB
:10C8D00001FE06C01F930F930E94C6930F900F9006
:10C8E00004B602FE06C0FF92EF920E94C6930F901C
:10C8F0000F9004B603FE06C0DF92CF920E94C6934B
:10C900000F900F9004B604FE06C0BF92AF920E9433
:10C91000C6930F900F9014BE0E94F96F0E94BE66DE
:10C92000CDCFDF92EF92FF920F931F93CF93DF93C0
:10C93000CDB7DEB7A0970FB6F894DEBF0FBECDBF60
:10C9400083E690E00E948B96182F282F35EF380F42
:10C95000303108F0982F9095291709F463C088E1C9
:10C9600093E19F938F930E94C693EDE5F3E18E01CF
:10C970000F5F1F4F0F900F90D801D02EE12EF02E99
:10C9800088E0800F94919D9331968A13FBCFF894A1
:10C9900048E050E06FE770E0C8010E949196EFE434
:10C9A000F3E1D8018EE08F0D94919D9331968A1317
:10C9B000FBCF4EE050E061E770E0C8010E94919625
:10C9C000E5E4F3E12AE02F0D8491D8018D938D01E8
:10C9D00031962A13F9CF4AE050E067E670E08D2DDA
:10C9E0009E2D0E9491966DEC7BEA81E690E00E947C
:10C9F000A99660E070E08FE590E00E94A99660E063
:10CA00008EE590E00E949B9660E070E085E690E005
:10CA10000E94A9961AE16AE175EE83E690E00E9411
:10CA2000A9967894812FA0960FB6F894DEBF0FBE1A
:10CA3000CDBFDF91CF911F910F91FF90EF90DF90CD
:10CA400008958FE590E00C948B968EE590E00C9421
:10CA50008396F8941092B60016BC89E787BD82E0F1
:10CA600084BD95E095BD95B395BB80936E00789499
:10CA700008950F931F936091A5137091A613809151
:10CA8000A7139091A8130091A5131091A6132091BC
:10CA9000A7133091A813601771078207930759F7FE
:10CAA0001F910F9108950F931F936091AD35709171
:10CAB000AE358091AF359091B0350091AD35109184
:10CAC000AE352091AF353091B035601771078207D0
:10CAD000930759F71F910F9108951F920F920FB668
:10CAE0000F9211240BB60F922F933F934F935F93A6
:10CAF0006F937F938F939F93AF93BF93EF93FF9326
:10CB00008091A5139091A613A091A713B091A8139B
:10CB10000196A11DB11D8093A5139093A613A09318
:10CB2000A713B093A8138091A4138F5F8093A413CD
:10CB300087FF15C01092A4138091AD359091AE354A
:10CB4000A091AF35B091B0350196A11DB11D809374
:10CB5000AD359093AE35A093AF35B093B03580919D
:10CB60004C378823E1F08091A3138F5F8093A31348
:10CB700087FF15C01092A3138091A5359091A6351B
:10CB8000A091A735B091A8350196A11DB11D809344
:10CB9000A5359093A635A093A735B093A8350E94EC
:10CBA000F66E892B11F00E94176EFF91EF91BF91E5
:10CBB000AF919F918F917F916F915F914F913F9135
:10CBC0002F910F900BBE0F900FBE0F901F901895D6
:10CBD0001F920F920FB60F9211240BB60F922F9344
:10CBE0003F934F935F936F937F938F939F93AF93F5
:10CBF000BF93EF93FF938091C600E091B335F0911E
:10CC0000B435309709F01995FF91EF91BF91AF912D
:10CC10009F918F917F916F915F914F913F912F9154
:10CC20000F900BBE0F900FBE0F901F9018951F9284
:10CC30000F920FB60F9211240BB60F922F933F93C2
:10CC40004F935F936F937F938F939F93AF93BF9314
:10CC5000EF93FF938091CE00E091B135F091B23522
:10CC6000309709F01995FF91EF91BF91AF919F9186
:10CC70008F917F916F915F914F913F912F910F9085
:10CC80000BBE0F900FBE0F901F90189581110EC014
:10CC90001092C5006093C40088E98093C10040935E
:10CCA000C2001092B4351092B3350895813069F402
:10CCB0001092CD006093CC0088E98093C900409326
:10CCC000CA001092B2351092B1350895811107C093
:10CCD0008091C00085FFFCCF6093C600089581302D
:10CCE00031F48091C80085FFFCCF6093CE00089599
:10CCF000CF93C82F8A3031F46DE08091A9130E9440
:10CD0000666602C08D3029F06C2F8091A9130E94B5
:10CD1000666680E090E0CF910895811105C0709320
:10CD2000B4356093B3350895813021F47093B235F2
:10CD30006093B13508958093A91383E992E09093AD
:10CD4000F8398093F739089584B7877F84BF0FB689
:10CD5000F894A8958091600088618093600010929B
:10CD600060000FBE08959FE088E10FB6F894A89583
:10CD7000809360000FBE909360000895A895089579
:10CD80000FB6F894A8958091600088618093600048
:10CD9000109260000FBE08950C94628F0C945E8F09
:10CDA0008091BA3590E008958091390181FF09C0E2
:10CDB000809139018D7F8093390189E190E001975D
:10CDC000F1F723E040E06FE182E491E00E940A6C19
:10CDD00085E090E00197F1F708959091390191FD78
:10CDE0000AC0282F803108F02FE040E06FE085E492
:10CDF00091E00C940A6C08958091390181FD0EC078
:10CE000040E06FE181E491E00E94FF6B282F2F7ECC
:10CE100081E090E0213021F080E0089580E090E012
:10CE200008958091390181FF02C081E0089540E0BA
:10CE30006FE181E491E00E94FF6B8F3121F08F7EE2
:10CE40008150823090F780E008958091390181FD12
:10CE500004C00E9411678823C1F3089510924C37D3
:10CE60008091390181FD8BC00E9425678091390135
:10CE700081FD85C00E94D4668091390182608093D3
:10CE80003901809184378823D9F180919400909161
:10CE90009500409195375091963784179507A0F4E7
:10CEA0008091613790916237A0916337B091643778
:10CEB000875F924CAF4FBF4F80936137909362373B
:10CEC000A0936337B093643720919400309195001C
:10CED000241B350B8091613790916237A0916337A5
:10CEE000B0916437820F931FA11DB11D80936137EC
:10CEF00090936237A0936337B0936437109284376E
:10CF0000809186378823D9F1809194009091950083
:10CF10004091993750919A3784179507A0F48091E2
:10CF2000693790916A37A0916B37B0916C37875F02
:10CF3000924CAF4FBF4F8093693790936A37A0935D
:10CF40006B37B0936C372091940030919500241B7F
:10CF5000350B8091693790916A37A0916B37B0910A
:10CF60006C37820F931FA11DB11D80936937909379
:10CF70006A37A0936B37B0936C3710928637089559
:10CF800080914C37882321F00E9411670E942E6700
:10CF900080E090E0089522E0260F27FF0CC08091EA
:10CFA0004A3790914B37019690934B3780934A378D
:10CFB0008FEF9FEF0895AB01BC018AEA93E10E94D5
:10CFC000F79280E090E0089540E06FE181E491E025
:10CFD0000C94FF6B282F40E06FEF86E591E00E94F4
:10CFE0000A6C0895CF93DF9398EF980F923038F042
:10CFF000982F9F7E963019F0893109F049C09091A1
:10D00000390191FD48C0C82F0E9425670E94E4673E
:10D01000D82FC81709F442C0C83029F480913901CB
:10D020000E94D46627C0C93119F4863181F404C046
:10D03000C63169F4893159F429E040E06FE182E4B6
:10D0400091E00E940A6C85E090E00197F1F72C2FA7
:10D0500040E06FE182E491E00E940A6CD83031F444
:10D060008FEF0E94EA6781ED92E002C085E090E0D8
:10D070000197F1F70E94E4678C1781F0C63019F42C
:10D08000813079F40BC0C63161F4813151F406C0AE
:10D0900082E490E008C084E490E005C080E490E081
:10D0A00002C083E490E0DF91CF91089580919400D5
:10D0B0009091950090939A378093993781E080936F
:10D0C000863780934C379091390191FF1EC0209193
:10D0D0009400309195003093963720939537809344
:10D0E0008437809347372FB77894809139018091A6
:10D0F00039018D7F8093390180E197E23091473784
:10D10000332311F00197D1F72FBF86E10E94F26718
:10D110000C94256780914C37811102C00E9456689B
:10D1200081E090E008950F931F93CF93DF931F92B8
:10D13000CDB7DEB780914C37882361F080913901FB
:10D1400081FF02C080E07BC00E9411678823D1F379
:10D1500000E003C00E948A6801E0809194009091F1
:10D160009500909394378093933711E01093833711
:10D1700080E88093550186E00E94F2671093BB35EA
:10D180008FB789837894109247018091BB358111C4
:10D19000FCCF89818FBF8091470111E08E3008F06C
:10D1A00010E0119586E10E94F2671092550180917E
:10D1B00083378823D9F18091940090919500409114
:10D1C00093375091943784179507A0F480915D3779
:10D1D00090915E37A0915F37B0916037875F924C36
:10D1E000AF4FBF4F80935D3790935E37A0935F370B
:10D1F000B09360372091940030919500241B350B3B
:10D2000080915D3790915E37A0915F37B091603724
:10D21000820F931FA11DB11D80935D3790935E37E0
:10D22000A0935F37B09360371092833701110E944B
:10D23000C067812F8295869586958370817090E076
:10D240000F90DF91CF911F910F9108958FEF8093F1
:10D250004E0121E044E060EF8CE691E00E940A6C10
:10D2600025E041E06EE08CE691E00E940A6C80E8E7
:10D2700080936F018091460180936D0121E045E02C
:10D2800060E284E491E00C940A6CCF93DF93C9EFE1
:10D29000D7E0CE010197F1F70E94FE6B1092C135E5
:10D2A000109243361092C5361092C0351092BF3599
:10D2B000E9E3F1E080818E7F808380818D7F8083B0
:10D2C00081EC93E00197F1F780818160808323E016
:10D2D00040E06FE182E491E00E940A6C2197F1F74F
:10D2E00080915D0180915E010E94266960E070E09E
:10D2F00081EA92E00E948B700E94566881E090E083
:10D30000DF91CF91089580912B140895CF93DF93EF
:10D310001F92CDB7DEB789830E94256789818093EC
:10D320002B14282F40E06FE188E491E00F90DF910B
:10D33000CF910C940A6C0E94866986E00C94F26787
:10D34000EF92FF920F931F93CF93DF931F921F9241
:10D35000CDB7DEB78C017A017F936F931F938F93C4
:10D360008CE799E09F938F9369837A830E94B293AD
:10D3700000936201109363016981609360017A8177
:10D38000709361010F900F900F900F900F900F907E
:10D39000E114F104C9F0F701808180936B01818170
:10D3A00080936A01828180936901838180936801FF
:10D3B0008481809367018581809366018681809353
:10D3C00065018781809364010F900F90DF91CF9169
:10D3D0001F910F91FF90EF90089581EA92E00E94D3
:10D3E000AC7081E08093BA358091BC359091BD35A9
:10D3F00001969093BD358093BC3581E090E008950F
:10D400000F931F93CF932091C035C2E8C29F900124
:10D410001124F901EF53FA4C4081442309F451C01F
:10D4200047FD09C0433038F050E08A01025011092D
:10D430006017710710F4108244C0B9016E537A4C22
:10D440000E94F7928091C035C89FF0011124EF53DC
:10D45000FA4CDF01A058BF4F9C919093B5351082D4
:10D460008F5F833018F48093C03502C01092C035AE
:10D47000E091C03582E8E89FF0011124EF53FA4CA7
:10D480008081882319F00E94ED6902C01092BA359C
:10D49000809147018093B6359091B935992311F069
:10D4A000891710F48093B9356091B63570E084E047
:10D4B0000E94AB756091B53570E083E00E94AB755A
:10D4C00002C000E010E0C801CF911F910F910895B4
:10D4D0000F931F93CF93DF931F92CDB7DEB78C01CD
:10D4E000FC0180819181009709F18334954029F0F6
:10D4F000F8011182108283E02AC06238E1F40E94B0
:10D5000057758FB78983F8940E94C67460E870E0FD
:10D510000E94006A29812FBF1816190674F40E9410
:10D52000C174E091220AF091230A199583E495E0F1
:10D53000F8019183808381E00AC08091B735909192
:10D54000B83501969093B8358093B735EFCF0F90EB
:10D55000DF91CF911F910F9108950C94ED6680910A
:10D56000390181FD06C040E06FE085E491E00C9454
:10D57000FF6B80E10895EF92FF921F93CF93DF93AB
:10D580001F92CDB7DEB7182F8091390181FD07C0FA
:10D590000E94256780914C3781111CC05AC0809130
:10D5A000940090919500909396378093953781E001
:10D5B0008093843780934737809139018D7F8093A2
:10D5C000390180E197E220914737222309F301973F
:10D5D000D1F7DECF809186378823D9F180919400EE
:10D5E000909195004091993750919A3784179507FB
:10D5F000A0F48091693790916A37A0916B37B09110
:10D600006C37875F924CAF4FBF4F809369379093D1
:10D610006A37A0936B37B0936C37209194003091A8
:10D620009500241B350B8091693790916A37A09142
:10D630006B37B0916C37820F931FA11DB11D809382
:10D64000693790936A37A0936B37B0936C37109219
:10D65000863789E10E94F26786E00E94B675892BC1
:10D6600051F00E94AF6AE82E86E00E94B6758150A4
:10D670000E94ED6602C0E12CF12C80919400909103
:10D680009500909398378093973781E08093853702
:10D690008FB78983F8948091390182608093390132
:10D6A000809139018D7F8093390162E0610F8AEAB0
:10D6B00093E10E94516C89818FBF8091483790918E
:10D6C0004937019690934937809348370E942567E0
:10D6D00045E060EE82E491E00E94FF6B182F86E047
:10D6E0000E94B675892B19F08E2D0E94ED668091EF
:10D6F00085378823D9F180919400909195004091CD
:10D7000097375091983784179507A0F48091653723
:10D7100090916637A0916737B0916837875F924CD8
:10D72000AF4FBF4F8093653790936637A0936737AD
:10D73000B09368372091940030919500241B350BED
:10D740008091653790916637A0916737B0916837BF
:10D75000820F931FA11DB11D80936537909366378B
:10D76000A0936737B09368371092853780914C3714
:10D77000882371F0809194009091950090939A374E
:10D780008093993781E0809386370E94566802C063
:10D790000E942E67123028F48CE00E94B67510E0CB
:10D7A0000BC0133031F0153031F0173029F411E08F
:10D7B00003C012E001C013E0812F90E00F90DF91D1
:10D7C000CF911F91FF90EF900895CF93DF93EB01DE
:10D7D0000E94CB67009729F4CE010E94BB6A009794
:10D7E00051F020914A3730914B372F5F3F4F3093A4
:10D7F0004B3720934A37DF91CF9108950895FC016C
:10D8000080816823862F90E002C0959587954A9580
:10D81000E2F70895CF93DF931F92CDB7DEB7FC01F7
:10D82000922F8FB78983F8942081362F3095522F0D
:10D830005323292F01C0220F4A95EAF72623252BCF
:10D84000208389818FBF0F90DF91CF910895CF936F
:10D85000DF93E0917B012DEF2E0F2D3740F0FC017F
:10D860001082E058FF4F10823196108217C0EC01F1
:10D87000E993A0E8B1E020E82E0F3C91399311968E
:10D880002A13FBCFE150F0E0E058FE4F2181FC016C
:10D89000E058FF4F2083319681E08083DF91CF9164
:10D8A000089560938001E1E8F1E06158DC012D9179
:10D8B000CD01208331966E13F9CF08951F920F92F8
:10D8C0000FB60F9211240BB60F922F933F934F93E5
:10D8D0005F936F937F938F939F93AF93BF93EF93D8
:10D8E000FF93809147018093B6358091BF3522E840
:10D8F000829FC00111248F539A4C0E94276C809103
:10D90000BF358F5F833018F48093BF3502C010920B
:10D91000BF350E94ED69FF91EF91BF91AF919F914B
:10D920008F917F916F915F914F913F912F910F90C8
:10D930000BBE0F900FBE0F901F9018951F920F9265
:10D940000FB60F9211240F900FBE0F901F901895D5
:10D950001F920F920FB60F9211240F900FBE0F90CF
:10D960001F9018951F920F920FB60F9211240F90CF
:10D970000FBE0F901F9018951F920F920FB60F9227
:10D980001124109247370F900FBE0F901F901895DB
:10D990001F920F920FB60F9211241092BE350F9066
:10D9A0000FBE0F901F9018951F920F920FB60F92F7
:10D9B00011240F900FBE0F901F9018951F920F9279
:10D9C0000FB60F9211241092BB350F900FBE0F901F
:10D9D0001F901895CF93DF93EC018991999100974F
:10D9E00029F060E070E00E948B70F7CFDF91CF915B
:10D9F0000895EF92FF920F931F93CF93DF938C01C3
:10DA00007A01FC0180819181009741F08A3491056F
:10DA100011F1F8011182108283E04AC08DE294E195
:10DA20000E943671EC01209761F04E815F8168851C
:10DA30007985CE0102960E94CD6E0990D881C02DC5
:10DA4000F2CF81E080932C148AE490E0F801918376
:10DA5000808381E02DC06838E1F78DE294E10E9477
:10DA60003671EC01209781F3CE010296E816F90693
:10DA7000D9F4BE018DE294E10E945671E090E11468
:10DA8000F090E2148E859F859093E2148093E114C8
:10DA9000E889F989309719F08A899B891995F0925C
:10DAA000E214E092E114D0CF0990D881C02DDACFF2
:10DAB000DF91CF911F910F91FF90EF9008951092F9
:10DAC0002C148DE294E10E94327160E070E08BEAE8
:10DAD00092E00C948B70EF92FF920F931F93CF9371
:10DAE000DF93EC01E090E114F090E214FF86EE8603
:10DAF000398B288B1B8B0A8B80912C14882379F00F
:10DB00008BEA92E09093E2148093E114CE010296A6
:10DB10000E94CD6EF092E214E092E11404C04E83B4
:10DB20005F8368877987BE018DE294E10E94567118
:10DB3000BE018DE294E1DF91CF911F910F91FF9093
:10DB4000EF900C947571CF93DF93EC0180912C14BE
:10DB5000882329F0CE0102960E94016F04C01B8623
:10DB60001A861D861C86BE018DE294E1DF91CF915D
:10DB70000C945671CF92DF92EF92FF920F931F9306
:10DB80008091331490913414892B49F410922F14FE
:10DB900010923014109231141092321441C00E942D
:10DBA00039658B019C01E0913314F0913414448168
:10DBB00055816681778180819181A281B381840FB3
:10DBC000951FA61FB71F801B910BA20BB30B0084E0
:10DBD000F185E02D3097C1F0C480D580E680F780D4
:10DBE00040815181628173814C0D5D1D6E1D7F1DD1
:10DBF000401B510B620B730B481759076A077B07D1
:10DC000030F7DB01CA01E3CF800F911FA21FB31FC2
:10DC100080932F1490933014A0933114B093321446
:10DC20001F910F91FF90EF90DF90CF90089585EBBB
:10DC300092E00C94AC70EF92FF920F931F93CF93EE
:10DC4000DF938C01FC0180819181009799F08935E7
:10DC50009105D9F0F8011182108283E068C08285B5
:10DC600093858417950709F049C00084F185E02D5C
:10DC70003097A9F7109234141092331489E590E08C
:10DC8000F8019183808381E052C0673891F1623856
:10DC9000A9F7C0913314D0913414E12CF12C2097C2
:10DCA00069F3CE010E940771892BF1F0AE0168E89B
:10DCB0008A859B850E945D70892BA1F41B861A863C
:10DCC00088859985E114F10421F0F7019187808717
:10DCD00004C09093341480933314198618860E94DC
:10DCE000BA6DD7CF0E94176E7E010884D985C02DEA
:10DCF000D6CFE0913314F0913414BACFF0933414AA
:10DD0000E0933314A085B185109709F4B7CF1A9624
:10DD10008D919C911B978417950739F418968D91D6
:10DD20009C91199791878087EDCFFD01EBCFDF9113
:10DD3000CF911F910F91FF90EF900895CF93DF93B4
:10DD4000EC010E94176E2A853B85909133148091D7
:10DD50003414232B91F0E92FF82F309771F0EC1742
:10DD6000FD0739F48091E1149091E2149387828742
:10DD700010C00084F185E02DF0CF2091E1143091A6
:10DD8000E2143B872A8798878987D0933414C093FD
:10DD90003314DF91CF910C94BA6DCF93DF93EC01E4
:10DDA0000E94D970CE01DF91CF910C949E6ECF93DB
:10DDB000DF93EC010E94E970CE01DF91CF910C94CA
:10DDC0009E6ECF93DF93EC010E94FB70CE01DF913A
:10DDD000CF910C949E6E21E030E0FC01828593850A
:10DDE000892B11F020E030E0C901089581E090E036
:10DDF0002091331430913414232B11F480E090E0FF
:10DE00000895CF93DF93EC01E0913314F091341433
:10DE10008E179F0769F488859985909334148093B1
:10DE200033140DC0808591858C179D0721F0FC016E
:10DE30003097C1F706C088859985918780870E94B1
:10DE4000BA6D198618861B861A86DF91CF910895C0
:10DE50001F93CF93DF93DC011496ED91FC911597FE
:10DE60003097E1F0162FEC019093E2148093E114C7
:10DE700082E08887CD0106961995082E000C990B33
:10DE80000297029710F0133839F4BE01CE01DF91EA
:10DE9000CF911F910C94586F81E08887DF91CF91CB
:10DEA0001F910895FC01208520FD0C94286F089592
:10DEB000CF92DF92EF92FF920F931F93CF93DF9356
:10DEC000E090E114F090E214C090E314D090E414D8
:10DED000F601E817F90739F0309709F44BC00190C3
:10DEE000F081E02DF6CF009709F444C08B01EC01DE
:10DEF0008885882309F11886C114D10461F0CC15F6
:10DF0000DD0529F0AE0167E8C6010E94526FF601F7
:10DF1000C080D180F1CFEC81FD81309769F0C017CE
:10DF2000D10751F0D093E214C093E11440E050E0E7
:10DF300063E8CE0106961995E091E314F091E4149C
:10DF4000CE17DF0741F4888199819093E414809380
:10DF5000E3140CC0FC01309749F0808191818C174B
:10DF60009D07C1F78881998191838083F092E214A3
:10DF7000E092E114DF91CF911F910F91FF90EF900C
:10DF8000DF90CF9008951F93CF93DF9310923D14AD
:10DF9000C091E314D091E41411E0209779F08985C1
:10DFA000882341F01887198640E050E062E8CE01EE
:10DFB0000E94286F0990D881C02DEFCFDF91CF91BB
:10DFC0001F9108958091E01491E0980F9093E014D0
:10DFD00008958AE88093E0141092DE141092DF1402
:10DFE0001092E4141092E3141092E2141092E114CF
:10DFF000089580913D1481110E94C36F5091DF14E8
:10E00000552309F452C0E091DE142E2F30E085E054
:10E01000E89FF0011124E25CFB4E608160933C14A8
:10E02000A181B281B0933B14A0933A14838194816F
:10E0300090933914809338142F5F3F4F2F713327FB
:10E040002093DE1451505093DF14009731F58091E6
:10E05000E3149091E41490933714809336148091D4
:10E06000361490913714892B01F180913D14811160
:10E070000E94C36F40913A1450913B1460913C143C
:10E0800080913614909137140E94526FE0913614AB
:10E09000F091371480819181DECF613819F421E04D
:10E0A000FC012087AD010E94526F80913D142091A8
:10E0B000DF1490E0820F911D08959C019091DF1470
:10E0C0009032B9F0E091DE14E90FEF71E09335146E
:10E0D00085E0E89FF0011124E25CFB4E60835283EF
:10E0E0004183348323839F5F9093DF1480E090E02B
:10E0F000089581E090E00895CF93DF93C091E114FB
:10E10000D091E2140E94526FD093E214C093E114B4
:10E11000DF91CF910895AB013091E3142091E41485
:10E12000E32FF22FE817F907B1F0309721F00190B3
:10E13000F081E02DF7CF009771F0FC01308321834F
:10E140009093E4148093E31421E0208717821682D1
:10E1500061E80C947C700895009749F0FC012085DB
:10E160002150223020F421E0218720933D1408958E
:10E170000C94E5798091E5149091E6140097C1F034
:10E180001092E6141092E514DC0114966D917C91C6
:10E1900015971296ED91FC9113971995E091E5145E
:10E1A000F091E614309721F0808191810C94FF79F1
:10E1B0000895CF93DF93EC014C835D836E837F835F
:10E1C0000E943965688379838A839B83DF91CF912D
:10E1D0000895FC0140815181628173818481958120
:10E1E000A681B781840F951FA61FB71F80839183D7
:10E1F000A283B3830895CF93DF93EC010E94396526
:10E20000688379838A839B83DF91CF910895CF922E
:10E21000DF92EF92FF92CF93DF93EC010E9439657A
:10E22000C880D980EA80FB80DC01CB018C199D0974
:10E23000AE09BF090196A11DB11D21E030E0CC80DF
:10E24000DD80EE80FF80C816D906EA06FB0610F0D6
:10E2500020E030E0C901DF91CF91FF90EF90DF9097
:10E26000CF900895FC01118210820895FC018081F5
:10E2700091810895DC01ED91FC91309741F080810E
:10E280009181009711F0FC01FACFCF01089580E051
:10E2900090E00895DC01ED91FC911197309721F009
:10E2A000208131812D933C93CF010895DC01ED91C4
:10E2B000FC913097C9F0A0E0B0E0E617F70761F4F1
:10E2C000FB0120813181109709F4DC012D933C93EF
:10E2D000FB0111821082089520813181DF01211517
:10E2E000310511F0F901E9CF08950F931F93CF93F2
:10E2F000DF938C01EB010E94567119821882C801CC
:10E300000E943A71009711F4F80101C0FC01D18319
:10E31000C083DF91CF911F910F910895DC01ED91A2
:10E32000FC9180E090E0309729F001960190F08117
:10E33000E02DF9CF0895009721F0FC0180819181B3
:10E34000089580E090E00895CF93DF93EC014A8137
:10E350005B8160E070E08C819D810E9400932A8146
:10E360003B8188819981289FA001299F500D389F6A
:10E37000500D112460E070E08E819F81DF91CF917C
:10E380000C940093FC018281938120E030E02817F7
:10E390003907D1F0A481B581A20FB31F4C9141116F
:10E3A00010C081E08C9380819181289FA001299FDA
:10E3B000500D389F500D112486819781840F951F31
:10E3C00008952F5F3F4FE3CF80E090E00895FC0178
:10E3D000868197814281538120E030E02417350700
:10E3E000D1F08617970781F4A481B581A20FB31FDE
:10E3F0008C91181614F481508C9384819581FC01C2
:10E40000E20FF31F80810895A081B1818A0F9B1FC5
:10E410002F5F3F4FE3CF8FEF0895FC0126813781B7
:10E4200062177307A0F0A081B18142815381A49F3C
:10E43000C001A59F900DB49F900D1124280F391F86
:10E4400081E090E06217730720F080E0089580E09B
:10E4500090E008952F923F924F925F926F927F9239
:10E460008F929F92AF92BF92CF92DF92EF92FF92E4
:10E470000F931F93CF93DF93CDB7DEB768970FB697
:10E48000F894DEBF0FBECDBFEDE4F7E324A535A5BC
:10E4900046A557A550A441A432A423A4948C858CEE
:10E4A000768C678C808D8983918D9A83828D8B8306
:10E4B000938D9C8384898D8395899E8386898F83A0
:10E4C000978998878089898791899A8782898B879C
:10E4D00093899C8784858D8795859E8786858F8780
:10E4E0009785988B8085898B91859A8BB284A3843C
:10E4F000F480E580D680C78080818F8B9181988F52
:10E50000128103812B8B3C8B4D8B5E8B0E9453655C
:10E510005E895F934D894F933C893F932B892F935D
:10E520002F923F924F925F926F927F928F929F9223
:10E530002C812F932B812F932A812F9329812F9325
:10E5400028852F932F812F932E812F932D812F9309
:10E550002C852F932B852F932A852F9329852F93F5
:10E5600028892F932F852F932E852F932D852F93D9
:10E57000AF92BF922A892F9329892F93CF92DF924E
:10E58000EF92FF920F931F93288D2F932F892F9334
:10E590009F938F937F936F93E3EAF7E381811F92B9
:10E5A0008F9380811F928F9385E693E19F938F9342
:10E5B0000E94C6930FB6F894DEBF0FBECDBF68961B
:10E5C0000FB6F894DEBF0FBECDBFDF91CF911F9184
:10E5D0000F91FF90EF90DF90CF90BF90AF909F9002
:10E5E0008F907F906F905F904F903F902F90089505
:10E5F000EF92FF920F931F93CF93DF938C01EB0168
:10E600007A010E948E73F801F086E78265ED79E069
:10E61000CE01DF91CF911F910F91FF90EF900C945D
:10E62000B2730C9496730C944A74DC011796ED91B6
:10E63000FC9118970190F081E02D309709F0199422
:10E640000895DC011796ED91FC9118970280F381F3
:10E65000E02D309709F019940895DC011996ED9199
:10E66000FC911A970280F381E02D309709F01994FC
:10E6700008950F931F93CF93DF931F921F92CDB7EF
:10E68000DEB78C0188E10E94C975BC01CE010196FC
:10E690000E947874D8011996ED91FC911A97019017
:10E6A000F081E02D309729F0BE016F5F7F4FC801E8
:10E6B00019950F900F90DF91CF911F910F910895B1
:10E6C000EF92FF920F931F93CF93DF938C01EB0197
:10E6D0007A0147ED59E00E94F872F801F286E1866E
:10E6E0006BED79E0CE01DF91CF911F910F91FF90FB
:10E6F000EF900C94B2730C941173CF93DF93EC01F1
:10E7000063EA77E388E10E94BF75CE01DF91CF9184
:10E710000C94137387EE94E10C943271FC017383B3
:10E720006283BC0187EE94E10C947571BC0187EEA5
:10E7300094E10C945671CF93DF93EC0187EE94E152
:10E740000E943671009749F0FC01228133812C1719
:10E750003D0729F00E949B71F5CF80E090E0DF91AA
:10E76000CF9108950F931F93CF93DF938B010E9456
:10E770009B73EC01892B31F01D830C83C8010E942F
:10E78000B2838E83DF91CF911F910F910895CF9225
:10E79000DF92EF92FF920F931F93CF93DF937C0151
:10E7A0008B016A0189EE94E10E943671EC01892B9C
:10E7B00051F0EC81FD81309711F0C8011995CE011F
:10E7C0000E949B71F3CFA601B801C701DF91CF91E1
:10E7D0001F910F91FF90EF90DF90CF900C942173D9
:10E7E0000F931F93CF93DF931F921F92CDB7DEB786
:10E7F0000E9484838C0189EE94E10E943671009717
:10E8000079F0DC011296ED91FC911397309729F085
:10E8100089839A8319959A8189810E949B71EFCF90
:10E820000115110549F0C8010F900F90DF91CF91AC
:10E830001F910F910C9415730F900F90DF91CF9152
:10E840001F910F910895CF92DF92EF92FF920F9355
:10E850001F930E94CF750E9457750E9419820E94D3
:10E860008283C12C88E0D82E87E0E82EF12C00E0CE
:10E870001EE120E030E040E052E060E070E082E045
:10E8800090E00E9449831F910F91FF90EF90DF90DD
:10E89000CF900895CF93DF93EC010E949783009768
:10E8A00061F00E94DF74E091F609F091F709BE0172
:10E8B00087EC93E7199581E090E0DF91CF9108957F
:10E8C000E0911E0AF0911F0A1994E091E809F09175
:10E8D000E9091994E091240AF091250A1994E0912C
:10E8E000260AF091270A199480E090E0089508958F
:10E8F000FB0120813181FC0131832083089542E0B6
:10E9000050E00E94EA9221E030E0892B11F020E0F3
:10E9100030E0C9010895BC0183EA97E30C94787450
:10E92000E091A609F091A7091995E0911C0AF091D0
:10E930001D0A1995E091F409F091F5091995E091F6
:10E94000E609F091E70919942091A2153091A315D9
:10E950002817390798F04091A0155091A115480F3C
:10E96000591F5093A1154093A015281B390B3093C4
:10E97000A3152093A21581E090E0089580E090E037
:10E9800008959093A3158093A21508958091A015E2
:10E990009091A115835E9A4E089580919F1590E005
:10E9A00083519B4E089581E090E02091EB143091CB
:10E9B000EC142D51354111F480E090E008950E944F
:10E9C000D374892B61F06091EB147091EC14409139
:10E9D000A2155091A3158DE195E10C94F792209129
:10E9E000A0153091A11521153105B9F08091A2151E
:10E9F0009091A315C096EDE1F5E1AF014D5E544154
:10EA00004817590734F4DF01A20FB31F4C9141930B
:10EA1000F4CF1092A1151092A01508958091A2151F
:10EA20009091A315089580919F1590E3981B2091D4
:10EA3000A2153091A315A901490F511DCA010895CE
:10EA40000F931F93CF938C01C0919F158C2F90E053
:10EA5000801791076CF00E941375800F911F813809
:10EA6000910530F4C01BC0939F1581E090E002C077
:10EA700080E090E0CF911F910F910895CF93DF93A5
:10EA8000EDEAF7E31192119287E3ED3DF807D1F734
:10EA9000C5EAD7E360E07AE0CE010E94787422965E
:10EAA00087E3CD3AD807B1F7DF91CF91089510925F
:10EAB000A1151092A0151092A3151092A21580E333
:10EAC00080939F158DE195E19093EC148093EB1466
:10EAD0000C943E75EF92FF920F931F93CF93DF93A9
:10EAE0001F921F92CDB7DEB78C0169837A830E9493
:10EAF00057756981E62E7A81F72E81E8E816F104D0
:10EB000018F080E8E82EF12CA701B8018091EB14F1
:10EB10009091EC140E94F792F092A315E092A21546
:10EB2000C7010F900F90DF91CF911F910F91FF9030
:10EB3000EF900895FC0190E3ADEAB7E301900D92E8
:10EB40009A95E1F788E0FB01A5EAB7E301900D9201
:10EB50008A95E1F70895E82FF0E0EE0FFF1FE355E7
:10EB6000F84C7183608381E090E00895E82FF0E035
:10EB7000EE0FFF1FE355F84C80819181089590E0DE
:10EB8000880F991F8B58984C0E94787481E090E010
:10EB9000089590E0880F991F8B58984C08958FEB3B
:10EBA00092E00E94A4718FEC92E00E94A47187EC25
:10EBB00092E00C94A4710F931F93CF93DF93EC0119
:10EBC000BC018FEC92E00E940D72892BA9F0099094
:10EBD000D881C02DFE0161917191CF010E946A75AB
:10EBE000BE016E547F4FCE018E579F4FDF91CF9164
:10EBF0001F910F910C949A75BE0187EC92E00E94D0
:10EC00000D72892BD1F00E945775688179818A81B4
:10EC10009B810E946A758CA990E00E9420750CA9C6
:10EC200010E00E94CD74BE016C5F7F4FA801DF91A0
:10EC3000CF911F910F910C94F792DF91CF911F917B
:10EC40000F91089587E19CE10E94EB6E892B21F0E2
:10EC500087E19CE10C94E16E0895E091031CF09132
:10EC6000041C309709F0199480E00895EF92FF9208
:10EC70000F931F93CF93DF938C01EA01FC018081F6
:10EC80009181009741F08A33934081F1F80111821C
:10EC9000108283E0F8C080E024E0829FF00111241C
:10ECA000EB5FF34E118210828F5F8430A9F780935F
:10ECB000021C8091E1149091E2149093161C8093B1
:10ECC000151C0E94E26F8093DD3740E450E060E065
:10ECD00070E087E19CE10E94CD6E0E94C67A8AE3D3
:10ECE00093E0F8019183808381E0CDC06230D9F454
:10ECF0008091DE379091DF37892B89F38091EF3750
:10ED0000863029F48091073881FD0E94227681E0C7
:10ED10000E940D7B8091DE379091DF37892BF9F2CD
:10ED20000E949077DCCF633060F5611114C02097AA
:10ED3000B1F2D093DC38C093DB3883E00E940D7BC6
:10ED40008091DE379091DF37892B11F00E942D766C
:10ED50000E942276C4CF613011F6209709F4BFCF0C
:10ED6000D093D838C093D73885E00E940D7B80912E
:10ED7000DE379091DF37892B09F4B1CF0E942D76D1
:10ED8000AECF673809F040C01092011C85E0E82E34
:10ED90008CE1F82E8091011C8430C0F4F70182814F
:10EDA00093818C179D0749F4808191810E94F27AAA
:10EDB000F7011182108213821282F4E0EF0EF11C2F
:10EDC0008091011C8F5F8093011CE4CFE6EFF8E394
:10EDD000838194818C179D0719F414821382108209
:10EDE000B09629E3E637F20799F7E3E7F9E381857F
:10EDF00092858C179D0711F4158214823D9689E344
:10EE0000E53FF807A1F76BCF683809F068CFC75125
:10EE1000DC4109F064CF87E19CE10E94EB6E892B15
:10EE200009F45DCF1092011CE091011CE43008F060
:10EE300056CF20E2E29FF0011124E352F74C818D7E
:10EE40008823D9F087E19CE10E94E16E8091011C4A
:10EE5000E0E28E9FC00111248352974C9093DC38DE
:10EE60008093DB3882E00E940D7B8091DE379091A9
:10EE7000DF37892B11F00E942D768091011C8F5F66
:10EE80008093011CD1CFDF91CF911F910F91FF9003
:10EE9000EF900895CF93DF93A091DB38B091DC38E9
:10EEA000109719F0ED016C9605C0C091D738D0913C
:10EEB000D83829968091D63886FF23C01092001C3E
:10EEC00080E0E5E0FCE18430C1F04081518114969E
:10EED0002D913C9115974217530761F4228133819C
:10EEE0002115310539F08093001C398328831B825A
:10EEF0001A8205C034968F5FE6CF8093001C0E9473
:10EF0000227688819981009741F04A815B816091E6
:10EF1000DD37DF91CF910C947C70DF91CF91089514
:10EF20000F931F93CF93DF938091EF37863009F0D3
:10EF30007AC08091DE379091DF37803F910508F4E9
:10EF400072C08897EC01D695C7959E01220F331F9A
:10EF50008E012817390710F40F5F1F4FCE018896D6
:10EF60009093DF378093DE379093E8378093E937CB
:10EF700010920B3810920A380E94C07A80959095B2
:10EF800090930B3880930A381092F1371092F03733
:10EF90000E94AF7A809590959093F1378093F037E7
:10EFA0000E942D76C80188969093DF378093DE37D4
:10EFB0009093E8378093E9378091D9389091DA3887
:10EFC000BC016C0F7D1FA8010E94F792BE018EEF5D
:10EFD00097E30E945C7A8091E2378093FE378091BC
:10EFE000E3378093FF378091E43780930038809136
:10EFF000E5378093013810920B3810920A380E943E
:10F00000C07A8095909590930B3880930A3810922F
:10F01000F1371092F0370E94AF7A809590959093D7
:10F02000F1378093F037DF91CF911F910F910C94BE
:10F030002D76E091B609F091B709199480E090E03F
:10F040000895AF92BF92CF92DF92EF92FF920F930B
:10F050001F93CF93DF93CDB7DEB7E1970FB6F89448
:10F06000DEBF0FBECDBF7C016B01CE0101965C01FE
:10F0700081E3F50111928A95E9F781E089838CE0BB
:10F080000E94B6758C831D821F828091231C91E0A3
:10F09000980F9093231C898713E018878DEC9BEAC7
:10F0A0009B878A8789E10E94C97560E07AE00E94A7
:10F0B0007F74892B31F082E08E838FEF8C878D8770
:10F0C00009C089E10E94C975BC01CE010C960E945D
:10F0D00078741E838DEC9BEA9D8B8C8B63EA77E3BF
:10F0E000CE0146960E9478740E94C6749FA78EA790
:10F0F0000E940E7599AB88ABC5010E94FA838C0102
:10F100001127C8010E942075892B31F10E94CD740E
:10F11000A801BC01C5010E941D840091AC09109199
:10F12000AD090E9413755C010E94CD74B501F80110
:10F130001995E114F10481F0009739F0019761F419
:10F1400041E050E064E070E004C041E050E060E085
:10F1500070E0C601F7011995E1960FB6F894DEBF8D
:10F160000FBECDBFDF91CF911F910F91FF90EF9018
:10F17000DF90CF90BF90AF9008950F931F93CF93E0
:10F18000DF934115510579F0FA018B01EC01828181
:10F1900093810E94DB75B801CE01DF91CF911F9161
:10F1A0000F910C942178DF91CF911F910F910895C9
:10F1B0000F931F93CF93DF93CDB7DEB7E1970FB6D1
:10F1C000F894DEBF0FBECDBF0E940E758C010E9469
:10F1D000C674AE014F5F5F4FB8010E941085892B46
:10F1E00009F443C088A999A99801281B390BC901C2
:10F1F0000E94A474892BC9F18E8181110CC0BE01BB
:10F200006A5E7F4F88E10E94BF75E091F809F09136
:10F21000F90919952AC02A853B852D3C9BEA3907B7
:10F2200019F02F3F3F4F09F5823019F088E090E048
:10F2300002C082E090E0019710F3E1E0F0E0EC0F13
:10F24000FD1FE80FF91F23852F3FA9F3BE01645F5F
:10F250007F4F89E10E94BF7589E10E94C97563EA09
:10F2600077E30E947F74892B51F6E1960FB6F894EC
:10F27000DEBF0FBECDBFDF91CF911F910F910895DB
:10F280000E94CE668093231CE091B609F091B709E5
:10F290001994892B29F0E091B609F091B70904C0BF
:10F2A000E091B809F091B9091994FC01680F791F30
:10F2B00080E048E1E617F70781F0219198E0322FCE
:10F2C0003827532F517030FD84278695513009F42B
:10F2D00080682695915099F7EDCF08951F920F926F
:10F2E0000FB60F9211240BB60F922F933F934F93AB
:10F2F0005F936F937F938F939F93AF93BF93EF939E
:10F30000FF93809194009091950090939037809313
:10F310008F3781E08093813780917100807D809369
:10F3200071000E94BA70809181378823D9F1809151
:10F3300094009091950040918F37509190378417A9
:10F340009507A0F48091553790915637A091573783
:10F35000B0915837875F924CAF4FBF4F809355376E
:10F3600090935637A0935737B09358372091940015
:10F3700030919500241B350B80915537909156376D
:10F38000A0915737B0915837820F931FA11DB11D1F
:10F390008093553790935637A0935737B09358378B
:10F3A00010928137FF91EF91BF91AF919F918F9113
:10F3B0007F916F915F914F913F912F910F900BBE75
:10F3C0000F900FBE0F901F9018959FB7F894E1E72C
:10F3D000F0E08081807D808388B38F6288BB10924B
:10F3E0009000E1E9F0E010821092920010929500F6
:10F3F000109294008081856080839FBF08959C0156
:10F400009FB7F894309399002093980088B38F6247
:10F4100088BBE1E7F0E08081826080839FBF089530
:10F42000FB0141505109460F571FE417F50778F4C7
:10F43000208130E0322F22276181260F311D820F7B
:10F44000931F8217930708F401963296EECFE417C4
:10F45000F50751F4208130E0322F2227820F931FCD
:10F460008217930708F401960895CF93DF93C09114
:10F47000E937D0E064972091E83730E0322F222737
:10F48000C20FD31F48E050E062EF77E39E01280FE0
:10F49000311DC9010E94107AAE016AEF77E30E9424
:10F4A000107A009721F098278927982702C08FEFBC
:10F4B0009FEFDF91CF910895FC012381260F2093C8
:10F4C000E537A72FBB2792819A0F9093E4373181BC
:10F4D0003093E33740814093E237E92FF0E0EA17B9
:10F4E000FB0748F481E0830F8093E337811103C069
:10F4F0004F5F4093E23730E077272617370788F4CD
:10F500009F5F9093E43791110CC08091E3378F5F38
:10F510008093E337811105C08091E2378F5F80933C
:10F52000E23708952091DB383091DC38BC01C90105
:10F5300008960E945C7AE091DB38F091DC38A2EE0C
:10F54000B7E38C91808711968C91119781871296E1
:10F550008C911297828713968C918387089544E14A
:10F5600050E066EE77E380E090E00E94107A00972A
:10F5700021F098278927982708958FEF9FEF089506
:10F5800086E00C94357A81E10C94357A80E0E82F9E
:10F59000F0E0EE0FFF1FE35AF64C118210828F5FEE
:10F5A0008430A9F780E090E2899FF0011124E352B2
:10F5B000F74C118E8F5F8430B1F780E094E0909328
:10F5C000291C8093281C80E09DE0989FF001112465
:10F5D000ED58F64C158214828F5F8A30B1F7809314
:10F5E000271C08959C0190E09430A1F0E92FF0E0F1
:10F5F00081E0890FEE0FFF1FE35AF64C40815181E5
:10F600004217530729F49093271C11821082089502
:10F61000982FEACF9093271C0895AF92BF92CF9274
:10F62000DF92EF92FF920F931F93CF93DF93C091DE
:10F63000DB38D091DC38843009F4DBC12EE038E3CC
:10F640003093DA382093D9383093E1372093E0377C
:10F65000833059F4898D8F70833009F06AC08889AE
:10F660009989892B09F0D4C67EC0823009F07FC009
:10F6700080912D1C8F5F80932D1C811113C0809170
:10F680002C1C8F5F80932C1C81110CC080912B1C33
:10F690008F5F80932B1C811105C080912A1C8F5F86
:10F6A00080932A1C1092DF371092DE371092723945
:10F6B00010927139898D982F9D7F953041F48A8DF4
:10F6C0008F5F8A8F843109F0A3C6198EA1C6882363
:10F6D00009F49EC628893989232B09F440C09A8DE4
:10F6E0002FEF290F2A8F911193C69B8D983031F0FF
:10F6F0002FEF280F223048F4953039F4198E80E826
:10F700008093D6380E944A773DC5953038F423E07F
:10F71000092E01C0220F0A94EAF701C020E32A8FC4
:10F720009F5F9B8F8F708330A1F048F4813009F484
:10F7300044C3823009F06CC61092073841C386304A
:10F7400009F4BCC4883009F4B9C4843009F060C637
:10F75000B5C484E08093D6380E944A7745C58F703F
:10F76000833009F055C688E08093D63800C58530CF
:10F7700019F5E091D738F091D83884819581892B9B
:10F7800009F446C61092DC381092DB3882E098E328
:10F790009093DA388093D9389093E1378093E037AB
:10F7A00010927239109271391092DF371092DE3751
:10F7B00088E08093D6381BC18091E637853409F004
:10F7C00027C60091E83710E0102F00278091E93715
:10F7D000080F111D8091DE379091DF378017910758
:10F7E00008F416C61093DF370093DE378091EC37AC
:10F7F0008F7309F00DC6F090ED37F11009C68091B6
:10F800006D3990916E39C0912A0AD0912B0A8C17CC
:10F810009D0759F440916F395091703920912C0A0D
:10F8200030912D0A42175307A1F02091F6373091FD
:10F83000F7372817390709F0EBC52091F8373091D1
:10F84000F93780916F39909170392817390709F08D
:10F85000DFC50E94AF7A019609F0DAC58091EF37D3
:10F86000863009F429C18131E9F1813009F0D0C530
:10F870008091FA37883009F0CBC51092FA37809121
:10F88000FC379091FD37873F6FEF960710F0099690
:10F8900001C008969093FD378093FC378091F23732
:10F8A0009091F337A091F437B091F5378093F63704
:10F8B0009093F737A093F837B093F93780916D396B
:10F8C00090916E39A0916F39B09170398093F23771
:10F8D0009093F337A093F437B093F53780E4809397
:10F8E000EE3773C50C5111091093DF370093DE37E3
:10F8F00082E098E39093DA388093D9388091003889
:10F9000090910138892B29F00E94C37A019609F061
:10F910007FC52091FC373091FD372115310509F461
:10F9200077C583E799E39093D8388093D738A09030
:10F93000FA37B090FB3740912E0A50912F0A609110
:10F94000300A7091310AA091F237B091F3370091EB
:10F95000F4371091F537E0902C0AF0902D0AE091E1
:10F96000D738F091D83889E3E53FF80708F050C55B
:10F9700084819581009721F12817390709F586813F
:10F980009781009719F0A816B906D1F4808191816A
:10F990008C179D0729F4C280D380CE14DF04B1F008
:10F9A0008417950729F4C280D380C616D70671F054
:10F9B000A817B90729F4828193810817190731F034
:10F9C0003D96F093D838E093D738C9CF1092DC3801
:10F9D0001092DB3882E08093D63882E098E39093EF
:10F9E000E1378093E03710927239109271390E949A
:10F9F0004A778091713990917239009709F408C55E
:10FA00009C01245E3F4F3093DF372093DE373093E5
:10FA1000E8372093E937E091D738F091D83820853E
:10FA20002093EE3721E12093EF3708969827892716
:10FA300098279093FF378093FE37109201381092E9
:10FA40000038848195819093FB378093FA378681C3
:10FA500097819093FD378093FC3780916D39909119
:10FA60006E39A0916F39B09170398093F2379093CD
:10FA7000F337A093F437B093F53780819181A28159
:10FA8000B3818093F6379093F737A093F837B0930C
:10FA9000F9378EE098E39093DA388093D9380E9452
:10FAA000C37A80959095009711F48FEF9FEF909314
:10FAB00001388093003889C40E94C07A019609F009
:10FAC000A7C44091FC375091FD374115510509F409
:10FAD0009FC48091FA379091FB37009709F498C43E
:10FAE0006091F2377091F337E091F437F091F53788
:10FAF000CDEDD8E3298D2223A9F0AC81BD814A1731
:10FB00005B0781F4AE81BF818A179B0759F4A881F6
:10FB1000B9816A177B0731F4AA81BB81EA17FB0719
:10FB200009F466C1A09629E3CD35D20719F7809173
:10FB300007388F738230D9F45093251C4093241CCE
:10FB400080E0843091F0E82FF0E0EE0FFF1FE35AE1
:10FB5000F64C208131818F5F4217530791F7109245
:10FB6000271C80E0C0E0D0E07CC08093271C8091FF
:10FB7000073882FD4DC484E18093073888E290E025
:10FB80009093DF378093DE3780E58093063830919D
:10FB90000138809105388093013820910038809198
:10FBA000043880930038209304389091FF37809177
:10FBB00003388093FF37909303388091FE3780930A
:10FBC000271C409102384093FE37809302383F5FF4
:10FBD0003093053831110DC02F5F20930438211167
:10FBE00008C09F5F90930338911103C08F5F80938B
:10FBF00002388091FA379091FB379093251C8093BF
:10FC0000241C2091FC373091FD373093FB37209333
:10FC1000FA379093FD378093FC378091F2379091BB
:10FC2000F337A091F437B091F5378093F63790937E
:10FC3000F737A093F837B093F93780916D399091E9
:10FC40006E39A0916F39B09170398093F2379093EB
:10FC5000F337A093F437B093F5379CC3973089F00E
:10FC60008F5F8430C1F060E2869F90011124F9011A
:10FC7000E352F74C918D9111F1CF8093271CEF0146
:10FC80000CC0209721F0428D9A8D941748F7E90116
:10FC9000C352D74CE5CF8093271C209709F4B8C3F3
:10FCA000D093DC38C093DB3883E08A8F888F1E8A3C
:10FCB00084E08F8B1B8E8091FC379091FD379D8364
:10FCC0008C838091FA379091FB379F838E8380914C
:10FCD000F2379091F337A091F437B091F5378883DC
:10FCE0009983AA83BB8381E0898F80912A1C8C87AA
:10FCF00080912B1C8D8780912C1C8E8780912D1CD0
:10FD00008F8781E090E0998B888B809101388B8779
:10FD1000809100388A878091FF3789878091FE37EC
:10FD2000888781E090E00E94927A80910638982F2F
:10FD3000907F913508F441C082958F7090E00597CF
:10FD4000880F991F880F991F2091261CEF2DF0E036
:10FD5000E817F90774F5EA51F84C20A5211103C002
:10FD60001092261C28C0213011F4F394EFCF2230DA
:10FD7000D9F431A53430C1F42093261CF092271C0D
:10FD800082A590E0982F882723A5822B9093251C8D
:10FD90008093241C893C910510F088EC90E09B8BAB
:10FDA0008A8B9D8B8C8B09C031A5332311F0F30E08
:10FDB000CDCF2093261CF092271C80E1809307383A
:10FDC0008091073882608093073882E080930E38F4
:10FDD00084E080930F381092103888EC80931138AB
:10FDE0008CE290E09093DF378093DE3780E680C22C
:10FDF000D093DC38C093DB381092D6388091073826
:10FE0000782F7470F72E82FF03C0198E80E219C21A
:10FE10009091063892959F70990F990F9093271C97
:10FE2000091B1109045111091093DF370093DE37C4
:10FE3000922F9F70923029F4982F9F73923139F44A
:10FE40001FC0913021F4982F9F739230C9F0012B7D
:10FE500019F4982F9370A1F02091FE3798852913FB
:10FE60003DC22091FF379985291338C2209100386F
:10FE70009A85291333C2209101389B8529132EC2FC
:10FE800084FF49C0688979896115710509F443C007
:10FE9000CE010C960E945C7A309102388091E23754
:10FEA000381339C0209103388091E337281333C0C9
:10FEB000909104388091E43798132DC080910538D3
:10FEC0004091E537841327C03C872D879E878F8715
:10FED0008B8D811119C09E89888D2A8D821B292FB7
:10FEE000269526952695821B980F9E8B87FD8195DA
:10FEF0002F89322F36953695231B820F8F8B96953F
:10FF000096959695890F888F81E08093D638888D55
:10FF10008A8F198A188A298DE22FEF708E2F90E030
:10FF2000FC013197E830F10508F072C28827E656E7
:10FF3000FF4F8F4F0C94B6888091D63880FF14C045
:10FF400083E0898F80E48093D638198A188A80915B
:10FF5000DE379091DF37009709F405C122E4209342
:10FF6000D6380E94927AFFC0809107388F73823012
:10FF700009F04EC222CF8091D63880FF6AC08091AE
:10FF800007388F73823109F064C080910638982F4A
:10FF9000907F913508F441C082958F7090E005976D
:10FFA000880F991F880F991F2091261CEF2DF0E0D4
:10FFB000E817F90774F5EA51F84C20A5211103C0A0
:10FFC0001092261C28C0213011F4F394EFCF223078
:10FFD000D9F431A53430C1F42093261CF092271CAB
:10FFE00082A590E0982F882723A5822B9093251C2B
:10FFF0008093241C893C910510F088EC90E09B8B49
:020000021000EC
:100000008A8B9D8B8C8B09C031A5332311F0F30EA5
:10001000CDCF2093261CF092271C83E0898F8091FE
:10002000FE3788878091FF378987809100388A87DB
:10003000809101388B8781E090E00E94927A82E47F
:100040008093D638198A188A1092DF371092DE37DB
:100050008AC080E28093D6380E944A77E091DB38EC
:10006000F091DC38118E83CD8091073880FF28C055
:1000700024FD26C088899989892B09F0C9C18091FE
:10008000DE379091DF3701960E94927A8091D638C0
:10009000982F90619093D6382091DE373091DF37DA
:1000A000232B19F082618093D6380E944A7781E031
:1000B00090E0998B888B88E0898F1B8E81E10FC13E
:1000C00085FF1DC080910C3890E0982F88273091D3
:1000D0000D38832B4091D9385091DA38480F591F89
:1000E0005093DA384093D9384091DE375091DF375A
:1000F000BA01681B790B7093DF376093DE3740914C
:10010000DE375091DF374115510551F024FD08C00D
:100110009091D63892609093D638CA010E94927A14
:100120008091083890E0982F882720910938820F15
:10013000911D9093251C8093241C2C893D892817A0
:10014000390710F0892B21F43093251C2093241CAF
:100150008091241C9091251C9B8B8A8B8091D63892
:10016000837009F455C110927239109271390E944E
:100170004A778091D63885FF07C010927239109265
:100180007139198E84E1ABC084FF0AC010927239B4
:100190001092713981E090E0998B888B84E08CCF4C
:1001A000209171393091723921153105E1F080FFCC
:1001B00002C0198A188A88899989009781F48A89E6
:1001C0009B898217930720F4909372398093713939
:1001D0008091713990917239998B888B04C090937A
:1001E0007239809371391B8E8091E0379091E1379D
:1001F0009093DA388093D93880917139909172391F
:10020000892B59F088899989009739F088969093BD
:10021000DF378093DE3788E10BC08091D63881FFCD
:10022000F7C088E290E09093DF378093DE3780E17B
:10023000809307385CC08091D63880FFE9C0198E62
:1002400080E18093D6380E944A77E2C08091DE3701
:100250009091DF37009711F00E94927A90910738C1
:100260008091D63890FF0BC080FF06C087E0898F51
:100270001A8E198A188A19C086E0898F16C080FFE5
:100280001EC085E0898F198A188AC2C08091DE3726
:100290009091DF37009711F00E94927A8091073891
:1002A00080FF0DC087E0898F1A8E81E090E00E9468
:1002B000927A80E18093D6380E944A770FC080916D
:1002C000DE379091DF37892B49F4A2C08091D63870
:1002D00080FF9EC087E0898F1A8E9AC080E180934C
:1002E000073888E290E09093DF378093DE3780E52F
:1002F00080930638888580930238898580930338F7
:100300008A85809304388B85809305388C8580930B
:10031000FE378D858093FF378E85809300388F85DB
:100320008093013886E08093EF378C819D81909394
:10033000FB378093FA378E819F819093FD378093AE
:10034000FC3780916D3990916E39A0916F39B091E1
:1003500070398093F2379093F337A093F437B093CA
:10036000F53788819981AA81BB818093F637909374
:10037000F737A093F837B093F937898D84FF05C01C
:10038000109209381092083805C01092083888EC8D
:100390008093093880E48093EE378091DE37909126
:1003A000DF379093E8378093E93710920D38109239
:1003B0000C3810920B3810920A380E94C07A80953F
:1003C000909590930B3880930A3885E48093E637B4
:1003D0001092E7371092ED371092EC3780912E1C77
:1003E00090912F1C019690932F1C80932E1C90931C
:1003F000EA378093EB371092F1371092F0370E9472
:10040000AF7A809590959093F1378093F03704C040
:100410001092DF371092DE371092D638DF91CF91ED
:100420001F910F91FF90EF90DF90CF90BF90AF9012
:10043000089582E39CE10C9432719093311C809377
:10044000301C089582E39CE10C943671EF92FF9288
:100450000F931F93CF93DF938C01EB017A0182E31B
:100460009CE10E9436710097D9F0DC0112962D9123
:100470003C9113972C173D0781F41696ED91FC9152
:100480001797309769F09701AE01B801DF91CF91CE
:100490001F910F91FF90EF9019940E949B71E3CFF1
:1004A000DF91CF911F910F91FF90EF9008950895E4
:1004B0000F931F93CF93DF93C3E7DCE1488159810A
:1004C0006A817B8100E010E022E832E883E59CE16C
:1004D0000E946B6D0E94CE66BC0180E090E0288196
:1004E00039814A815B810E947588AB01BC0127EA92
:1004F00032E88FE39CE10E946B6DDF91CF911F91F9
:100500000F9108958091731C9091741CA091751C9B
:10051000B091761C40916F1C5091701C6091711CC1
:100520007091721C880F991FAA1FBB1F481759078B
:100530006A077B0710F4DB01CA018093731C909358
:10054000741CA093751CB093761C0C945882CF93A6
:10055000DF930E9457750E94C674EC0119821882BD
:100560000E94228228813981009719F1FC0140857F
:100570004423F9F0FC0142815381F901EE0FFF1F82
:10058000EE0FFF1FEC0FFD1F53834283FC014481DC
:1005900055812F5F3F4FF901EE0FFF1FEE0FFF1F39
:1005A000EC0FFD1F51834083398328830E949B7188
:1005B000D9CFC901880F991F880F991F02960E94F1
:1005C000C17488819981892B31F084E39CE1DF91AA
:1005D000CF910C947D73DF91CF910895AF92BF922C
:1005E000CF92DF92EF92FF920F931F93CF93DF93FF
:1005F0001F921F92CDB7DEB75B010E94C6748C01BB
:10060000FC01E080F180FA82E9820E940E75970178
:10061000220F331F220F331F2E5F3F4F8217930786
:1006200098F0C12CD12CCE14DF0471F0F801448174
:10063000558162817381C5010E942682FFEFCF1A26
:10064000DF0A0C5F1F4FEFCF0F900F90DF91CF911C
:100650001F910F91FF90EF90DF90CF90BF90AF90E0
:1006600008950F93013099F48091671C9091681C54
:10067000A091691CB0916A1C8093731C9093741CA8
:10068000A093751CB093761C0F910C9458820F9117
:1006900008954F925F926F927F928F929F92AF9246
:1006A000BF92CF92DF92EF92FF920F931F932A0196
:1006B0003B014801590142E35AE0BC0184E39CE15B
:1006C0000E946073E4E3FCE143AA54AA65AA76AAF7
:1006D00087AA90AEA1AEB2AEC3AED4AEE5AEF6AED2
:1006E00081E393E81F910F91FF90EF90DF90CF90FF
:1006F000BF90AF909F908F907F906F905F904F9042
:100700000C941D820C948A73CF93DF93E091360A88
:10071000F091370A1995EC01892B29F06A817B81C8
:1007200081E00E94AB75CE01DF91CF9108950F93C8
:100730001F93CF93DF93EC01E091380AF091390ACF
:1007400019958C016A817B8181E00E94AB7581E003
:1007500090E0012B11F480E090E0DF91CF911F91A8
:100760000F910895E0913A0AF0913B0A1994CF93C2
:10077000DF93FC01DB0185E0EB0119928A95E9F733
:100780008581837011F082E08C938781837021F0E2
:1007900082E012968C9312978581837081F0878115
:1007A000837069F0238934898185928528173907F8
:1007B00031F481E0848312961C92129701C0148256
:1007C00085818370823029F0833011F488E001C084
:1007D00080E011968C93119787818370823029F085
:1007E000833011F488E001C080E013968C93DF9190
:1007F000CF910895CF93DF9300D01F921F92CDB772
:10080000DEB7BE016F5F7F4F0E94B783898190E0A2
:1008100003962A81820F911D2B81820F911D2C81BD
:10082000820F911D2D81820F911D0F900F900F90BF
:100830000F900F90DF91CF9108953F924F925F926A
:100840006F927F928F929F92AF92BF92CF92DF92E0
:10085000EF92FF920F931F93CF93DF9300D01F92DD
:100860001F92CDB7DEB78C017B013A01BE016F5FED
:100870007F4F0E94B78369817A81472F50E0EB81D7
:100880003C80232D30E0862F90E00396840F951F47
:100890008E0F911D820F931FAD818A0F911D6816D7
:1008A00079060CF4A4C0D80111968C91119780FBA5
:1008B000882480F8912C83E0880C991C8A95E1F7B4
:1008C00012968C91129780FBAA24A0F8B12C94E088
:1008D000AA0CBB1C9A95E1F78A288C918770882A0C
:1008E00013968C91139780FBCC24C0F8D12CF5E0A3
:1008F000CC0CDD1CFA95E1F7C82814968C9180FB8E
:10090000442440F8512CA6E0440C551CAA95E1F76C
:100910004C28D7014C92D80115968C918370B4E085
:100920008B9F60011124D80116969C919370B0E1C1
:100930009B9FC00111248C29D8011796FC9190E44B
:10094000F99FD00111248A2BD70111968C93D801DD
:1009500018968C91D70112968C93623071F4D8015D
:1009600019968C91D70113968C93D8011A968C9175
:10097000D70114968C9385E001C083E0780F872F10
:10098000972F941B4115510561F041505109D80131
:10099000A40FB51F1B968C91D701A90FB11D8C9385
:1009A000EECFE23071F4D701A70FB11DF8019389A2
:1009B0009C9391E0970FD701A90FB11D8E5F948989
:1009C0009C93F32DF80F8F2F821B2115310561F0B9
:1009D00021503109D801A20FB31F55969C91D70120
:1009E000A80FB11D9C93EFCF8F2F90E002C080E045
:1009F00090E00F900F900F900F900F90DF91CF919C
:100A00001F910F91FF90EF90DF90CF90BF90AF902C
:100A10009F908F907F906F905F904F903F90089540
:100A2000AF92BF92CF92DF92EF92FF920F931F93FC
:100A3000CF93DF93633071050CF4B3C0EA016B010F
:100A40007C01FC01908196FBAA24A0F88181282FCB
:100A5000269526952370B82EB294B694B69453E09A
:100A6000B522392F3770388393FB332730F9398318
:100A700094FB332730F93A8395FB992790F99B83B0
:100A8000AC822D83829583708E83BF82828188871A
:100A9000222379F13381848190E0982F8827830F76
:100AA000911D9A87898787010B5F1F4F223071F450
:100AB00060E07AE0CE010B960E947874F70186819F
:100AC0008B8785818C870E5F1F4F1EC02330E1F41A
:100AD000F7013D96DE011B969E012D5E3F4F9E2F36
:100AE0008F2F42914D93A217B307D9F7092F182FD3
:100AF0000BC087010D5F1F4F60E07AE0CE010B96BF
:100B00000E9478741A861986BB20A1F1A1100DC02D
:100B1000F8012081818190E0982F8827820F911D14
:100B20009C8B8B8B0E5F1F4F04C089859A859C8B95
:100B30008B8BF2E0BF120EC060E07AE0CE014596EA
:100B40000E947874F80181818D8B80818E8B0E5F7D
:100B50001F4F18C0F3E0BF1215C0085F1F4FD80128
:100B6000FE017596CE014D962E912193E817F90757
:100B7000D9F708C060E07AE0CE0145960E9478740B
:100B80001C8A1B8A98012E193F09C601821B930BF0
:100B900098AB8FA71EA70DA7C216D30614F0C901E4
:100BA00002C080E090E0DF91CF911F910F91FF9004
:100BB000EF90DF90CF90BF90AF90089520E030E0AD
:100BC0000296FC0132974081442331F0FC013197B9
:100BD0004081240F311DF4CFC9010895FC0120810B
:100BE00030E0322F22278181282B02C0220F331FB1
:100BF0006A95E2F7232F3327FA01E45CF54F8081F1
:100C000090E08223932328E030E0241B350B02C0C0
:100C1000969587952A95E2F708956F927F928F9225
:100C20009F92AF92BF92CF92DF92EF92FF920F937B
:100C30001F93CF93DF937C018B015A01E901283088
:100C4000310544F4A901B501C8010E94EE85F70100
:100C5000808346C0690183E0D594C7948A95E1F703
:100C6000452B21F04701612C712C06C0FB01D701F7
:100C7000CB018C0D9D1D1FC048E050E0B501C8019F
:100C8000860D971D0E94EE85F40181934F01FFEFC1
:100C90006F1A7F0A6C147D0479F7AE0147705527EF
:100CA00041155105E9F0E701C60DD71DB501C80191
:100CB000860D971D12C0E817F90719F021912D93A1
:100CC000FACFAE01477055274115510549F0E701AC
:100CD000CC0DDD1D60E070E0CF010E94EE858883C1
:100CE000DF91CF911F910F91FF90EF90DF90CF9008
:100CF000BF90AF909F908F907F906F9008958F924C
:100D00009F92AF92BF92CF92DF92EF92FF920F939A
:100D10001F93CF93DF931F921F92CDB7DEB70E9430
:100D2000C6748C0182E090E00E94A474892B19F4AF
:100D300080E090E05FC0F801218130E0322F22276F
:100D40008081A901480F511DCA010E949B737C013B
:100D5000892B71F30E94C6744C01F7019681292FEB
:100D600026952695269530E0977041E050E011F4E5
:100D700040E050E0C901840F951F0E94A474892BA4
:100D8000B9F2F70104811581A12CB12CF801808101
:100D9000882379F1F801C180D12CA501477055272E
:100DA000B50193E0759567959A95E1F7680D791D02
:100DB000883168F09601CE0101960E940D86BE0131
:100DC0006F5F7F4FF80180810E94BF750DC01A824E
:100DD00019829601CE0101960E940D8669817A8161
:100DE000F80180810E94AB75AC0CBD1C0E5F1F4FDB
:100DF000CDCFC7010F900F90DF91CF911F910F9131
:100E0000FF90EF90DF90CF90BF90AF909F908F902A
:100E10000895DC0150E0E0E1F0E0CF01861B970B84
:100E2000821B930B02C0440F551F8A95E2F78C91E9
:100E3000852B8C9311968C911197482B11964C937E
:100E400008956F927F928F929F92AF92BF92CF92AE
:100E5000DF92EF92FF920F931F93CF93DF9328308F
:100E600031051CF4FA0140815AC05901E3E0B59400
:100E7000A794EA95E1F76115710541F03901EA019E
:100E80008B017C014A01C12CD12C05C0EA01FC0177
:100E90004A0D5B1D2AC0F40141914F0128E030E06A
:100EA000B801C7018C0D9D1D0E940987FFEFCF1A65
:100EB000DF0ACA14DB0479F7930127703327211561
:100EC0003105E9F1CC0DDD1D488150E0021B130B0B
:100ED000085F1F4F02C0559547950A95E2F760E0FD
:100EE00070E0C7018C0D9D1D1AC0C417D50719F0FD
:100EF00069916193FACF2770332721153105F9F0F5
:100F0000488150E068E070E0621B730B02C05595A9
:100F100047956A95E2F760E070E08A0D9B1DDF91CE
:100F2000CF911F910F91FF90EF90DF90CF90BF90E6
:100F3000AF909F908F907F906F900C940987DF9176
:100F4000CF911F910F91FF90EF90DF90CF90BF90C6
:100F5000AF909F908F907F906F9008956F927F9247
:100F60008F929F92AF92BF92CF92DF92EF92FF92B9
:100F70000F931F93CF93DF931F921F92CDB7DEB7CE
:100F80007C01FC018681082F069506950695202F89
:100F900030E0877001E010E011F400E010E0020F93
:100FA000131FC80102960E942075009709F448C0DB
:100FB0000E94CD74F7012281FC012083F701238177
:100FC000FC0121830E94CD7402965C01A80160E0BF
:100FD00070E00E940093F701048115810F5F1F4F9D
:100FE000812C912CF80131978081882339F1F80107
:100FF000C080D12C3401F7E06F227724740193E094
:10100000F594E7949A95E1F7EA0CFB1C883128F0F7
:101010000E94C9759601AC0108C00E94B6759A83FA
:1010200089839601AE014F5F5F4FB301C7010E94F4
:1010300021878C0C9D1C0E5F1F4FD4CF81E090E068
:101040000F900F90DF91CF911F910F91FF90EF9034
:10105000DF90CF90BF90AF909F908F907F906F90D8
:101060000895DB018F939F930E94DC88BF91AF911D
:10107000A29F800D911DA39F900DB29F900D1124F2
:101080000895991B79E004C0991F961708F0961BE4
:10109000881F7A95C9F780950895AA1BBB1B51E15B
:1010A00007C0AA1FBB1FA617B70710F0A61BB70BD8
:1010B000881F991F5A95A9F780959095BC01CD017D
:1010C000089597FB072E16F4009407D077FD09D0FA
:1010D0000E944D8807FC05D03EF4909581959F4F66
:1010E0000895709561957F4F0895A1E21A2EAA1B6D
:1010F000BB1BFD010DC0AA1FBB1FEE1FFF1FA217C8
:10110000B307E407F50720F0A21BB30BE40BF50BC4
:10111000661F771F881F991F1A9469F7609570954D
:10112000809590959B01AC01BD01CF010895052EDE
:1011300097FB1EF400940E94AE8857FD07D00E94D2
:10114000758807FC03D04EF40C94AE8850954095FA
:10115000309521953F4F4F4F5F4F08959095809563
:10116000709561957F4F8F4F9F4F0895EE0FFF1F32
:10117000881F8BBF0790F691E02D19940E94C688B6
:10118000332312F48A1B9B0B0C94D788A29FB001C7
:10119000B39FC001A39F700D811D1124911DB29FAB
:1011A000700D811D1124911D08950E94C688B7FFFE
:1011B0000895821B930B08950E94C688A59F900DE9
:1011C000B49F900DA49F800D911D11240895B7FF29
:1011D0000C94DC880E94DC88821B930B0895DF93BB
:1011E000CF931F930F939A9DF02D219FF00D8B9D10
:1011F000F00D8A9DE02DF10D039FF00D029FE00D93
:10120000F11D4E9DE00DF11D5E9DF00D4F9DF00D09
:101210007F936F93BF92AF925F934F93D5010E94DC
:10122000C6888B01AC01D7010E94C688EB01E80F8C
:10123000F91FD6010E943F892F913F91D6010E944C
:10124000C688C60FD71FE81FF91FAF91BF910E9434
:101250003F892F913F910E94C688C60FD71FE81F74
:10126000F91FD6010E94C688E60FF71F9801BE013C
:10127000CF0111240F911F91CF91DF9108950E940A
:10128000C688460F571FC81FD91F08F43196089506
:10129000E894DF93CF93FC01DB010E94C6887F9323
:1012A0006F93E9019A01AC01BF93AF933F932F93E2
:1012B000DF010E94C68826F46C1B7D0B820B930B0A
:1012C0009E01EB01FC010E943F89AF91BF912F91DC
:1012D0003F910E943F89BE01CF01F9012F913F91BB
:1012E000CF91DF910895689401C0E894F92FF12B14
:1012F00012F00C94A789A0E0B0E0E1E8F9E80C94C2
:10130000198A092E059422F40E94038A112392F46B
:10131000F0E80F26FFEFE094F09400951095B0945C
:10132000C094D094A194BF0ACF0ADF0AEF0AFF0A43
:101330000F0B1F0B0E94B28907FC0E94038ACDB7D6
:10134000DEB7ECE00C94358A689401C0E8948F9283
:101350009F92CF93DF930E94B289DF91CF919F90AC
:101360008F90089588249924F401E401B0E49F93B8
:10137000AA279A158B049C04ED05FE05CF05D0071E
:10138000A10798F4AD2FDC2FCF2FFE2FE92D982C3D
:10139000892E982F872F762F652F542F432F322F8A
:1013A0002227B85031F7BF9127C01B2EBF91BB2712
:1013B000220F331F441F551F661F771F881F991F59
:1013C000881C991CEE1FFF1FCC1FDD1FAA1FBB1F0F
:1013D0008A149B04EC05FD05CE05DF05A007B107C7
:1013E00048F08A189B08EC09FD09CE09DF09A00B1B
:1013F000B10B21601A94E1F62EF49401AF01BE0105
:10140000CD01000C0895609570958095909530956C
:101410004095509521953F4F4F4F5F4F6F4F7F4FF6
:101420008F4F9F4F08952F923F924F925F926F92EE
:101430007F928F929F92AF92BF92CF92DF92EF9264
:10144000FF920F931F93CF93DF93CDB7DEB7CA1BE5
:10145000DB0B0FB6F894DEBF0FBECDBF19942A8800
:10146000398848885F846E847D848C849B84AA84B8
:10147000B984C884DF80EE80FD800C811B81AA8145
:10148000B981CE0FD11D0FB6F894DEBF0FBECDBF10
:10149000ED0108950F93083090F0982F872F762F45
:1014A000652F542F432F322F22270850F4CF220FBD
:1014B000331F441F551F661F771F881F991F0A95EA
:1014C000B2F70F91089597FB10F8169400080F9348
:1014D000083098F00850232F342F452F562F672FB0
:1014E000782F892F902DF4CF059497958795779530
:1014F000679557954795379527950A95AAF70F91C0
:1015000008952A0D3B1D4C1D5D1D6E1D7F1D801F06
:10151000911F08950024A7FD00942A0F301D401D3F
:10152000501D601D701D801D901D08952A193B09D6
:101530004C095D096E097F09800B910B08952A15EE
:101540003B054C055D056E057F05800791070895F5
:101550000024A7FD00942A173005400550056005BA
:1015600070058005900508955058BB27AA270E9452
:10157000CC8A0C94378D0E94298D38F00E94308DD2
:1015800020F039F49F3F19F426F40C94EF8C0EF4FC
:10159000E095E7FB0C94E98CE92F0E94488D58F305
:1015A000BA17620773078407950720F079F4A6F548
:1015B0000C946A8D0EF4E0950B2EBA2FA02D0B0122
:1015C000B90190010C01CA01A0011124FF27591B88
:1015D00099F0593F50F4503E68F11A16F040A22F8E
:1015E000232F342F4427585FF3CF469537952795FF
:1015F000A795F0405395C9F77EF41F16BA0B620BFE
:10160000730B840BBAF09150A1F0FF0FBB1F661F44
:10161000771F881FC2F70EC0BA0F621F731F841F87
:1016200048F4879577956795B795F7959E3F08F0AD
:10163000B0CF9395880F08F09927EE0F979587956F
:1016400008950E94298D60F080E891E009F49EEFF2
:101650000E94308D28F040E851E071F45EEF0CC03C
:101660000C94EF8C0C946A8DE92FE0780E94488DE1
:1016700040F3092E052AB1F3261737074807590703
:1016800038F00E2E07F8E02569F0E025E0640AC086
:10169000EF6307F8009407FADB01B9019D01DC0153
:1016A000CA01AD01EF930E94AF8B0E94378D0E945B
:1016B000648B5F91552339F02BED3FE049E450FDF9
:1016C00049EC0C94B58A0895DF93DD27B92FBF77D5
:1016D00040E85FE31616170648075B0718F4D92F92
:1016E0000E94768D9F938F937F936F930E94018FBB
:1016F000E4E4F1E00E94028D0E94378D2F913F912A
:101700004F915F910E94578EDD2351F09058A2EACD
:101710002AED3FE049EC5FE3D0785D270E94CC8A58
:10172000DF910C94378D0E94C58C08F481E00895F8
:101730000E94AC8B0C94378D0E94308D58F00E9423
:10174000298D40F029F45F3F29F00C94E98C511168
:101750000C946B8D0C94EF8C0E94488D68F3992348
:10176000B1F3552391F3951B550BBB27AA2762179D
:101770007307840738F09F5F5F4F220F331F441FAA
:10178000AA1FA9F335D00E2E3AF0E0E832D09150DE
:101790005040E695001CCAF72BD0FE2F29D0660FCB
:1017A000771F881FBB1F261737074807AB07B0E80E
:1017B00009F0BB0B802DBF01FF2793585F4F3AF014
:1017C0009E3F510578F00C94E98C0C946B8D5F3F33
:1017D000E4F3983ED4F3869577956795B795F7959A
:1017E0009F5FC9F7880F911D9695879597F9089582
:1017F000E1E0660F771F881FBB1F6217730784071E
:10180000BA0720F0621B730B840BBA0BEE1F88F72C
:10181000E095089529F416F00C94E98C0C946A8DE7
:101820000C94EF8C0E94508DA8F39638A0F707F81F
:101830000F92E8942BE33AEA48EB5FE70E945A8E56
:101840000F920F920F924DB75EB70F920E94108EBB
:10185000E1E7F1E00E94028D4F915F91EF91FF91DE
:10186000E595EE1FFF1F49F0FE57E0684427EE0F95
:10187000441FFA95E1F74195550B0E94828D0F9018
:1018800007FE0C94768D089597FB16F40E94F28C57
:101890000C94888CE89409C097FB3EF49095809551
:1018A000709561957F4F8F4F9F4F9923A9F0F92F26
:1018B00096E9BB279395F695879577956795B795A4
:1018C000F111F8CFFAF4BB0F11F460FF1BC06F5F8A
:1018D0007F4F8F4F9F4F16C0882311F096E911C09C
:1018E000772321F09EE8872F762F05C0662371F0BD
:1018F00096E8862F70E060E02AF09A95660F771FD1
:10190000881FDAF7880F9695879597F90895E894D8
:10191000F92F96EBFF2381F0121613061406440BE1
:101920009395F69587957795679557954040FF2352
:10193000B9F71BC099270895882351F49850D2F71E
:10194000872B762F652F542F432F322F20E0B1F3B2
:10195000121613061406440B88233AF09A95440F86
:10196000551F661F771F881FCAF755234AF4440F77
:10197000551F11F460FF04C06F5F7F4F8F4F9F4F63
:10198000880F9695879597F90895990F0008550F38
:10199000AA0BE0E8FEEF16161706E807F907C0F0F5
:1019A00012161306E407F50798F0621B730B840BFD
:1019B000950B39F40A2661F0232B242B252B21F4D7
:1019C00008950A2609F4A140A6958FEF811D811D77
:1019D000089597F99F6780E870E060E008959FEFB1
:1019E00080EC089590958095709560955095409500
:1019F000309521953F4F4F4F5F4F6F4F7F4F8F4F28
:101A00009F4F0895DF93CF931F930F93FF92EF9211
:101A1000DF927B018C01689406C0DA2EEF010E94F0
:101A2000578EFE01E894A5912591359145915591E8
:101A3000A6F3EF010E94CC8AFE019701A801DA9477
:101A400069F7DF90EF90FF900F911F91CF91DF9199
:101A5000089500240A941616170618060906089514
:101A600000240A9412161306140605060895092E7A
:101A70000394000C11F4882352F0BB0F40F4BF2BE9
:101A800011F460FF04C06F5F7F4F8F4F9F4F089529
:101A900057FD9058440F551F59F05F3F71F047951F
:101AA000880F97FB991F61F09F3F79F08795089504
:101AB000121613061406551FF2CF4695F1DF08C023
:101AC000161617061806991FF1CF86957105610540
:101AD00008940895E894BB2766277727CB0197F9E8
:101AE00008950E94C58C08F48FEF08959B01AC0106
:101AF00060E070E080E89FE30C94988B0C94E98C94
:101B00000C94058F0E94508DD8F39923C9F3940F3C
:101B1000511DA3F39150504094F059F0882332F0B6
:101B2000660F771F881F91505040C1F79E3F5105A7
:101B30002CF7880F911D9695879597F908955F3F2B
:101B4000ACF0983E9CF0BB27869577956795B79546
:101B500008F4B1609395C1F7BB0F58F711F460FF1B
:101B6000E8CF6F5F7F4F8F4F9F4FE3CF0C946B8D0C
:101B70000E94C88D29ED3BE54EED5EE30C94448E4A
:101B800016F00C94058F0C94EF8C68940C94E98CEF
:101B90000E94508DA8F39923C1F3AEF3DF93CF9346
:101BA0001F930F93FF92C92FDD2788232AF02197D7
:101BB000660F771F881FDAF720E030E040E85FEB20
:101BC0009FE3883920F0803E38F021968F770E947D
:101BD000B58AE9E9F1E004C00E94B58AE6ECF1E0DB
:101BE0000E94028D8B01BE01EC01FB2E6F57710923
:101BF0007595771F880B990B0E944C8C28E132E772
:101C000041E35FE30E94578EAF2D9801AE01FF9034
